:100000000C942C320C9426350C9451350C947C3580
:100010000C94A7350C94D2350C94FD350C942836ED
:100020000C9453360C945D320C945D320C945D321A
:100030000C945D320C945D320C945D320C945D3204
:100040000C945D320C9457F90C945D320C945D3233
:100050000C945D320C945D320C9429E70C945F3261
:100060000C945D320C943CBD0C94E8BD0C945D3254
:100070000C945D320C945D320C945D320C945D32C4
:100080000C945D320C945D320C945D320C945D32B4
:100090000C945D320C945D320C945D320C945D32A4
:1000A0000C945D320C945D320C945D320C945D3294
:1000B0000C945D320C945D320C945D320C945D3284
:1000C0000C945D320C945D320C945D320C945D3274
:1000D0000C945D320C945D320C945D320C945D3264
:1000E0000C945D329C33A133A633B033BA3333342E
:1000F000C433CC33D433DE33E833F23301340B343E
:10010000333415341F34293457345A3449344D3478
:10011000533491345E34623468346C3470347634E1
:100120007A347E349134843488348C349E707E707A
:100130008470817087708A708D7099709070AB70C8
:100140009370967077BA75BA99BA96BA94BACBBAD0
:10015000C8BAC6BA24BBF2BAEFBAEDBA6FBD75BD64
:1001600086BD91BD99BDAEBD9DBDAEBDA1BDA5BDB8
:10017000AEBDABBDE5CDEACDEFCDF7CDFCCD01CE2B
:1001800006CE0BCE28CE28CE10CE28CE15CE1ACE37
:1001900023CE43CE48CE4DCE55CE5ACE5FCE64CE82
:1001A00069CE86CE86CE6ECE86CE73CE78CE81CE0A
:1001B000A1CEA6CEABCEB3CEB8CEBDCEC2CEC7CE2C
:1001C000E4CEE4CECCCEE4CED1CED6CEDFCEFFCEC2
:1001D00004CF09CF11CF16CF1BCF20CF25CF42CFD1
:1001E00042CF2ACF42CF2FCF34CF3DCF09D00ED030
:1001F00019D024D02FD03AD045D050D084D084D03C
:1002000084D084D05BD0A2D0ADD0BED0CFD0E0D04F
:10021000F1D002D113D14BD14BD14BD14BD121D104
:100220006AD176D187D198D1A9D1BAD1CBD1DCD13D
:1002300014D214D214D214D2EAD133D23CD24BD23B
:1002400056D261D26CD277D281D2B0D2B0D2B0D2F3
:10025000B0D289D2EAD2F0D2FAD206D312D329D3BD
:1002600039D31BD449D31BD459D31BD46AD376D3E7
:100270008BD397D3D6D3E0D3E8D3F4D300D40FD421
:100280003AD443D450D45FD46ED488D49BD4A7D569
:10029000AED4A7D5C1D4A7D5D5D4E7D4FFD411D532
:1002A00053D560D56BD57AD589D59BD5C6D5CFD555
:1002B000DCD5EBD5FAD514D627D633D73AD633D7F3
:1002C0004DD633D761D673D68BD69DD6DFD6ECD636
:1002D000F7D606D715D727D752D758D760D76AD7BA
:1002E00072D789D797D76AD8A5D76AD8B3D76AD82B
:1002F000C2D7D1D7E5D7F0D732D83AD842D84AD8E2
:1003000052D861D8084AD73B3BCE016E84BCBFFDB2
:10031000C12F3D6C74319ABD56833DDA3D00C77FD5
:1003200011BED9E4BB4C3E916BAAAABE000000806E
:100330003F05A84CCDB2D44EB93836A9020C50B9FD
:10034000918688083CA6AAAA2ABE000000803F0029
:100350000D94357E0D94BA360D946B5C0D942A8302
:100360004E414E494E495459494E46CDCCCC3D0A9A
:10037000D7233C17B7D13877CC2B329595E6241F7D
:10038000B14F0A000020410000C84200401C462036
:10039000BCBE4CCA1B0E5AAEC59D7400000A0B02AF
:1003A000090C0D0E08070304010000000000000006
:1003B000000000000000000000000000000000003D
:1003C00000000000000000121110000000000000FA
:1003D000000000000000000000000000000000001D
:1003E0000001021020200808102040102040800248
:1003F000010201080402010102040810204080806B
:1004000040201008040201800402018040201008EE
:1004100004020108040201010204081020408001C6
:100420000204081020408005050505070508080896
:1004300008020202020A0A08080404040401010175
:10044000010101010103030303030303030407077D
:10045000070C0C0C0C0C0C0C0C020202020606061B
:1004600006060606060B0B0B0B0B0B0B0B000020F6
:10047000002300260029002C002F0032000001007C
:100480000003010601090100002200250028002BBD
:10049000002E003100340002010000050108010BAC
:1004A0000100002100240027002A002D0030003325
:1004B0000001010000040107010A0101060D00FE10
:1004C00009016602D620FFFE0BFE0AFE0D00602227
:1004D0001969808080808080800080183363A0A0AC
:1004E000A00357675050F850F850500259692078CF
:1004F000A0A0702828F02002596948A85010204078
:1005000050A89002586840A0A040A0989068281376
:1005100063808080113B6B204040808080808040E1
:100520004020113B6B804040202020202040408014
:1005300006556520A870A8200455652020F82020C5
:10054000113363604080065161F811336340E0402D
:100550000259690808101020404080800259692023
:1005600050888888888850200259692060A02020FF
:10057000202020F80259697088880810204080F8EF
:10058000025969F80810207008088870025969102B
:100590001030505090F81010025969F88080B0C89F
:1005A0000808887002596970888080F0888888708F
:1005B000025969F808101020204040400259697023
:1005C00088888870888888700259697088888878D7
:1005D0000808887011386840E040000040E0401191
:1005E000386840E0400000604080025969081020EF
:1005F000408040201008045464F80000F802596953
:1006000080402010081020408002596970888808B6
:10061000102020002002596970888898A8A8B0800E
:10062000780259692050888888F888888802596932
:10063000F048484870484848F002596970888080FE
:100640008080808870025969F04848484848484886
:10065000F0025969F8808080F0808080F802596942
:10066000F8808080F0808080800259697088808066
:10067000809888887002596988888888F88888886E
:1006800088123969E040404040404040E0025969EA
:10069000381010101010109060025969888890A0CE
:1006A000C0A0908888025969808080808080808086
:1006B000F80259698888D8A8A88888888802596962
:1006C00088C8C8A8A89898888802596970888888B6
:1006D0008888888870025969F0888888F0808080CE
:1006E00080015A6A70888888888888A870080259AA
:1006F00069F0888888F0A09088880259697088809D
:10070000807008088870025969F820202020202075
:1007100020200259698888888888888888700259CA
:1007200069888888885050502020025969888888B4
:1007300088A8A8A8A850025969888850502050500D
:10074000888802596988885050202020202002592A
:1007500069F808101020404080F8113B6BE0808061
:1007600080808080808080E00259698080404020C5
:1007700010100808113B6BE02020202020202020B2
:1007800020E0085363205088015161F82A226280DA
:10079000400256667008788898680259698080809F
:1007A000F088888888F00256667088808088700299
:1007B0005969080808788888888878025666708899
:1007C000F880887002596930484040F0404040400D
:1007D0000058687088888878088870025969808015
:1007E00080B0C8888888881238684000C04040407F
:1007F00040E0004A6A100030101010109090600223
:10080000596980808090A0C0A09088123969C0404A
:10081000404040404040E0025666D0A8A8A8A888C2
:10082000025666B0C88888888802566670888888AC
:100830008870005868F0888888F080808000586848
:100840007888888878080808025666B0C880808052
:10085000800256667088601088700258684040F0C8
:10086000404040483002566688888888986802561A
:10087000668888885050200256668888A8A8A850A4
:1008800002566688502020508800586888888898CA
:1008900068088870025666F810204080F8015B6B8B
:1008A0001820202020C020202020182219698080B4
:1008B00080808080808080015B6BC0202020201899
:1008C00020202020C008536348A890FFFFFFFFFFAF
:1008D000FFFFFFFFFFFFFFFFFFFFFFFFFFFFFFFF28
:1008E000FFFFFFFFFFFFFFFFFFFFFFFF0D00602285
:1008F0001969800080808080808080035868207023
:10090000A8A0A0A8702002596930484040E04040AB
:1009100048B00356668870505070880259698888BC
:100920005050F820F82020221969808080800080B3
:10093000808080124A6A6090806090906010906021
:100940001A3262A0A00359697088A8D8C8D8A888AC
:1009500070045767700878887800F8035666285046
:10096000A0A05028045363F80808163161E0035929
:10097000697088E8D8D8E8D888700A5161F81744B7
:1009800064609090600357672020F8202000F807EB
:10099000356540A02040E007356540A04020C02AD2
:1009A000226240800058688888888898E8808002A1
:1009B000596978E8E8E8E868282828262161C020F5
:1009C0002262408007356540C04040E004576770B0
:1009D0008888887000F8035666A050282850A00226
:1009E0005A6A40C04040E00818283808025A6A4055
:1009F000C04040E01028081038025A6A40A0402049
:100A0000A048182838080259692000202040808812
:100A10008870025A6A40200020508888F88888022E
:100A20005A6A10200020508888F88888025A6A3054
:100A3000480020508888F88888025A6A2850002088
:100A4000508888F88888025A6A5050002050888858
:100A5000F88888025A6A20502020508888F88888B0
:100A600002596958A0A0A0B0E0A0A0B8005B6B70CC
:100A700088808080808088702040025A6A402000F0
:100A8000F88080F08080F8025A6A102000F8808098
:100A9000F08080F8025A6A304800F88080F0808048
:100AA000F8025A6A505000F88080F08080F8123ABC
:100AB0006A804000E04040404040E0123A6A2040F6
:100AC00000E04040404040E0124A6A609000E04050
:100AD00040404040E0123A6AA0A000E04040404060
:100AE00040E0025969F0484848E8484848F0025A4E
:100AF0006A2850008888C8A8988888025A6A4020C6
:100B00000070888888888870025A6A10200070886F
:100B10008888888870025A6A304800708888888877
:100B20008870025A6A285000708888888888700205
:100B30005A6A505000708888888888700355658884
:100B400050205088015B6B08709898A8A8A8C8C866
:100B50007080025A6A4020008888888888887002DD
:100B60005A6A10200088888888888870025A6A30FB
:100B7000480088888888888870025A6A505000889F
:100B8000888888888870025A6A10200088885020D7
:100B900020202002596980F0888888F080808002B7
:100BA0005969609090A0A0908888B002596940204F
:100BB00000700878889868025969102000700878D9
:100BC00088986802596930480070087888986802E7
:100BD00059692850007008788898680259695050FF
:100BE00000700878889868025A6A304830007008A7
:100BF00078889868025666702870A0A850005868D7
:100C00007088808088702040025969402000708878
:100C1000F88088700259691020007088F880887008
:100C20000259693048007088F8808870025969500C
:100C300050007088F8808870123969804000C04088
:100C4000404040E0123969204000C040404040E050
:100C5000124969609000C040404040E0123969A0EC
:100C6000A000C040404040E0025A6A50206010702E
:100C70008888888870025969285000B0C888888898
:100C800088025969402000708888888870025969F4
:100C90001020007088888888700259693048007078
:100CA00088888888700259692850007088888888E8
:100CB000700259695050007088888888700357679F
:100CC000202000F8002020015868087098A8A8C8C3
:100CD0007080025969402000888888889868025985
:100CE000691020008888888898680259693048000F
:100CF0008888888898680259695050008888888850
:100D00009868005B6B102000888888986808887055
:100D1000005A6A8080B0C88888C8B08080005B6B49
:100D2000505000888888986808887001050700FE80
:100D30000500FB01F220FFFE05FE05FE0200400259
:100D400015258080800080053242A0A002556550A4
:100D5000F850F8500146562070C030E0200255652A
:100D60009010204048025565608068906805122206
:100D700080800225354080808040022535804040BB
:100D80004080043343A040A003334340E0400122AD
:100D9000324080043141E002112180025565081083
:100DA0002040800245556090909060022535C040FB
:100DB000404040024555E0106080F0024555E0108B
:100DC0006010E00245552060A0F020024555F080FB
:100DD000E010E00245556080E09060024555F0105B
:100DE00020404002455560906090600245556090FB
:100DF0007010600313238000800214248000808020
:100E00000235452040804020033343E000E00235B6
:100E1000458040204080024555E01060004002556A
:100E2000657088B8A870024555609090F0900245B2
:100E300055E090E090E0023545608080806002459A
:100E400055E0909090E0023545E080E080E002358A
:100E500045E080E080800245557080B0907002458A
:100E6000559090F09090023545E0404040E00245BA
:100E700055301010906002455590A0C0A0900235EA
:100E80004580808080E002556588D8A88888024522
:100E90005590D0B09090024555609090906002457A
:100EA00055E09090E080014656609090906010026E
:100EB0004555E09090E09002455570806010E0024A
:100EC0003545E0404040400245559090909060028A
:100ED00045559090A0A04002556588A8A8A850024A
:100EE000455590906090900245559090701060022A
:100EF0003545E0204080E0022535C0808080C0027A
:100F000055658040201008022535C0404040C0058E
:100F1000324240A0024151F0052232804002445446
:100F20007090907002455580E09090E002344460EB
:100F3000808060024555107090907002445460B0FB
:100F4000C0600235452040E0404000465670909019
:100F500070106002455580E0909090021525800049
:100F60008080800027374000404040408002455547
:100F70008090A0E0900215258080808080025464DB
:100F8000F0A8A8A8024454E09090900244546090C5
:100F90009060004656E09090E08080004656709049
:100FA00090701010023444A0C0808002445470C07D
:100FB00030E002354540E04040200244549090909B
:100FC000700244549090A040025464A8A85050026B
:100FD0003444A04040A000465690909070106002AB
:100FE0004454F02040F002354560408040600215D6
:100FF000258080808080023545C0402040C0054269
:101000005250A0FFFFFFFFFFFFFFFFFFFFFFFFFFAB
:10101000FFFFFFFFFFFFFFFFFFFFFFFFFFFFFFFFE0
:10102000FFFFFFFF020040FFFFFFFFFFFFFFFFFF8B
:10103000FFFFFFFFFFFFFFFFFFFFFFFFFFFFFFFFC0
:10104000FFFFFFFFFFFFFFFFFFFFFFFFFFFFFFFFB0
:10105000FFFFFFFFFFFFFFFFFFFFFFFFFFFFFFFFA0
:10106000FFFFFFFFFFFFFFFFFFFFFFFFFFFFFFFF90
:10107000FFFFFFFFFFFFFFFFFFFFFFFFFFFFFFFF80
:10108000FFFFFFFFFFFF01050800FF0601210235FA
:1010900020FFFF07FF06FF090050221656808080C0
:1010A000800080153353A0A0A00257575050F8502D
:1010B000F850500257572070A070287020133555F3
:1010C00080A040A02002475740A0A040A0A05025EB
:1010D00013538080801226564080808080401226E4
:1010E000568040404040800245559060F06090023C
:1010F00055552020F8202011335360408004415181
:10110000F011335340E040024656101020408080DA
:1011100012365640A0A0A0A04012365640C0404013
:1011200040E00246566090106080F0024656F02083
:10113000601090600246562060A0F02020024656C3
:10114000F080E01090600246566080E0909060026F
:101150004656F01020204040024656609060909025
:1011600060024656609090701060122555C0C00015
:10117000C0C0113656606000604080123656204074
:1011800080804020034353F000F012365680402008
:1011900020408012365640A0204000400158583070
:1011A0004898A8A8904030024656609090F09090E1
:1011B000024656E090E09090E002465660908080B3
:1011C0009060024656E090909090E0024656F08083
:1011D000E08080F0024656F080E080808002465633
:1011E000609080B090600246569090F0909090127F
:1011F0003656E040404040E002465670202020A095
:101200004002465690A0C0A0A09002465680808022
:101210008080F002465690F0F090909002465690F2
:10122000D0F0B0B090024656609090909060024628
:1012300056E09090E08080014757609090D0B06079
:1012400010024656E09090E0909002465660904022
:10125000209060123656E040404040400246569092
:1012600090909090600246569090909060600246F8
:1012700056909090F0F0900246569090606090905A
:10128000025656888850202020024656F0102040F2
:1012900080F0123656E080808080E00246568080E2
:1012A00040201010123656E020202020E016325246
:1012B00040A0014151F016225280400244547090E7
:1012C00090700246568080E09090E0123454608026
:1012D000806002465610107090907002445460B0C6
:1012E000C060024656205040E040400145556090A5
:1012F0007010600246568080E09090901236564002
:1013000000C04040E01137572000202020A04002BC
:101310004656808090E09090123656C04040404043
:10132000E0025454D0A8A8A8024454E0909090023F
:10133000445460909060014555E090E08080014504
:10134000557090701010024454A0D0808012345414
:1013500060C020C00246564040E040502002445445
:1013600090909070123454A0A0A04002545488A8C9
:10137000A850024454906060900145559090709040
:1013800060024454F02040F0024757304020C02013
:101390004030221656808080808080024757C020CF
:1013A00040304020C006425250A0FFFFFFFFFFFF29
:1013B000FFFFFFFFFFFFFFFFFFFFFFFFFFFFFFFF3D
:1013C000FFFFFFFFFFFFFFFFFFFFFF090050221697
:1013D000568000808080800146562070A0A070203A
:1013E0000246562050E04050A0025555887050707B
:1013F000880256568850F820F8202217578080809F
:10140000008080800247577080E0907010E01731B4
:1014100051A002565670A8C8C8A87014355560A0CF
:101420006000E003435350A050123353E0202014D7
:101430003151E002565670E8D8E8D870173151E0C3
:1014400015335340A04012355540E04000E01435BC
:101450005540A02040E0143555C020C020C01622C1
:10146000524080014555909090E08002565678E8B1
:10147000E8682828241151801122524080143555E3
:1014800040C04040E014355540A04000E0034353C5
:10149000A050A0024757808080A060F020024757EC
:1014A0008080A0D010207002475780408060A0F05C
:1014B0002012365640004080A0400247574020602E
:1014C00090F0909002475720406090F09090024733
:1014D0005760906090F0909002475750A06090F055
:1014E000909002475790006090F0909002475760AC
:1014F000906090F0909002465670A0A0F0A0B001CD
:101500004757609080809060400247574020F080AD
:10151000E080F00247572040F080E080F00247571B
:101520006090F080E080F00247579000F080E0800B
:10153000F01237578040E0404040E01237572040DB
:10154000E0404040E012375740A0E0404040E01209
:101550003757A000E0404040E00256567048E84847
:10156000487002475750A090D0B090900247574023
:10157000206090909060024757204060909090606B
:101580000247576090609090906002475750A0606B
:101590009090906002475790006090909060123356
:1015A00053A040A002465670B0B0D0D0E0024757DA
:1015B00040209090909060024757204090909090EB
:1015C000600247576090909090906002475790005B
:1015D0009090909060025757102088502020200251
:1015E000465680E09090E0800246566090A0A09021
:1015F000A00247574020007090907002475720404B
:1016000000709090700247572050007090907002C8
:10161000475750A00070909070024656500070904E
:10162000907002475760906070909070025454F030
:1016300068B078113555608080604002475740207F
:101640000060B0C06002475720400060B0C0600238
:10165000475760900060B0C060024656500060B0CE
:10166000C060123757804000C04040E0123757201A
:101670004000C04040E012375740A000C04040E06A
:10168000123656A000C04040E0024757A040A010CC
:1016900070906002475750A000E09090900247572A
:1016A000402000609090600247572040006090907A
:1016B000600247576090006090906002475750A0CA
:1016C00000609090600246569000609090601235E5
:1016D000554000E0004002445470B0D0E00247574B
:1016E00040200090909070024757204000909090CA
:1016F000700247576090009090907002465690009C
:101700009090907001485820400090907090600137
:1017100047578080E090E08080014757900090908C
:1017200070906025753A2530327500253032753A53
:101730002530327500202020200025202000252083
:1017400000253164002532640025336400253464AB
:101750000025356400253664000000007E0060002E
:10176000600060F87ECC60CC60CC60F860CC00CCCF
:1017700000CC00CC00000000000000FE7F0E7026B0
:1017800064724E7A5E324C8241324C7A5E724E26E0
:10179000640E70FE7F000000000000FE7F0E70C629
:1017A00063C24382411A58BA5D1A588241C243C685
:1017B000630E70FE7F00000000000088088808109B
:1017C0001120222022101188088808101100000022
:1017D000000000000000000000000020221011881E
:1017E000088808101120222022101188080000000B
:1017F00000000000000000000000000000000000E9
:10180000000000000000000000000000000000FEDA
:101810007FFE7F06600000000000000000F00FF86F
:101820001FF81FF81FF00FF00FF81FF81FF81FE048
:1018300007C0038001000000003048483045727244
:101840003A207574663820666F6E74206E6F74204F
:10185000696E697469616C697A65642E004572729B
:101860003A207574663820666F6E74206E6F74202F
:10187000696E697469616C697A65642E004572727B
:101880003A207574663820666F6E74206E6F74200F
:10189000696E697469616C697A65642E00506C6563
:1018A000617365207265736574005052494E5445EA
:1018B000522048414C544544007F80FFC0FFC0FF88
:1018C000C07F807F80FFC0FFC0FFC03F001E000CB4
:1018D00000FFFFFF0E000E000E000E000E000E00B7
:1018E0000E000E007FC03F801F000E0004000400A9
:1018F0000E001F003F807FC00E000E000E000E0085
:101900000E000E000E000E0000FE0003FF80078395
:10191000C00E01C00E00E01C00E07F00E03E00E0D1
:101920001C00E00800E00000E00001C00E01C00F54
:10193000078007FF0001FC0001FC0007FF000F0704
:10194000800E01C00001C00000E00800E01C00E0C3
:101950003E00E07F00E01C00E00E00E00E01C0074A
:1019600083C003FF8000FE0000060C00FE07022675
:1019700003BC017FFE08FE08FE05080806000040C3
:10198000F0C88888987810050808060000C0F88814
:1019900088888888F80505050600012030F8302081
:1019A0000508080600002070F820202020E0050926
:1019B000090600FF2070A8A8B888887020050606D0
:1019C000060001E08CEA8C8A0A0509090600FFF886
:1019D000A88888888888A8F8050A0A0600FE20508A
:1019E00050505088A8A8887003030306000340A045
:1019F00040FFFFFFFFFFFFFFFFFFFFFFFFFFFFFFB6
:101A0000FFFFFFFFFFFFFF0000000605FF010707C4
:101A100006020080808080800080030303060105A9
:101A2000A0A0A005060606000050F85050F850058A
:101A300009090600FF2070A8A07028A870200507DB
:101A400007060000C8C81020409898050707060040
:101A50000040A0A040A89068010303060205808012
:101A6000800309090601FF2040408080804040201B
:101A70000309090601FF80404020202040408005E6
:101A8000070706000020A8702070A820050505069D
:101A900000012020F820200203030601FFC040803F
:101AA000050101060003F8020202060100C0C0059C
:101AB00007070600000810102040408005070706B1
:101AC0000000708898A8C8887003070706010040C6
:101AD000C040404040E0050707060000708808103D
:101AE0002040F8050707060000F808103008887045
:101AF00005070706000010305090F8101005070782
:101B0000060000F880F00808887005070706000046
:101B1000304080F0888870050707060000F808103C
:101B2000102020200507070600007088887088882C
:101B300070050707060000708888780810600205A5
:101B400005060100C0C000C0C00206060601FFC0B5
:101B5000C000C040800305050601012040804020F0
:101B6000050303060002F800F803050506010180DD
:101B700040204080050707060000708810202000E4
:101B8000200507070600007088B8A8B88070050710
:101B900007060000708888F888888805070706000F
:101BA00000F04848704848F00507070600007088B4
:101BB0008080808870050707060000F04848484884
:101BC00048F0050707060000F88080F08080F805DF
:101BD0000707060000F88080F08080800507070670
:101BE00000007088808098887005070706000088CC
:101BF0008888F8888888030707060100E04040408D
:101C00004040E005070706000038101010109060F3
:101C10000507070600008890A0C0A0908805070768
:101C2000060000808080808080F80507070600009D
:101C300088D8A8888888880507070600008888C88B
:101C4000A898888805070706000070888888888813
:101C500070050707060000F08888F080808005077F
:101C60000706000070888888A890680507070600A6
:101C700000F08888F0A090880507070600007088AB
:101C80008070088870050707060000F820202020D3
:101C90002020050707060000888888888888700546
:101CA0000707060000888888885050200507070627
:101CB000000088888888A8A85005070706000088C3
:101CC0008850205088880507070600008888502023
:101CD000202020050707060000F80810204080F8A3
:101CE0000309090601FFE080808080808080E00594
:101CF000070706000080404020101008030909066D
:101D000001FFE020202020202020E0050303060022
:101D1000052050880501010600FEF80303030601B3
:101D200005804020050505060000700878887805C4
:101D300007070600008080F0888888F00505050602
:101D4000000070808088700507070600000808788A
:101D5000888888780505050600007088F080700581
:101D60000707060000304840E040404005070706EE
:101D700000FE7088888878087005070706000080D4
:101D800080F0888888880307070601004000C0406B
:101D90004040E00409090601FE1000301010101048
:101DA000906005070706000080808890E090880317
:101DB0000707060100C04040404040E00505050619
:101DC0000000D0A8A8A8A8050505060000B0C8888E
:101DD0008888050505060000708888887005070753
:101DE0000600FEF0888888F080800507070600FE60
:101DF00078888888780808050505060000B0C8803E
:101E0000808005050506000078807008F00507074A
:101E10000600002020F820202018050505060000F7
:101E200088888898680505050600008888885020FD
:101E30000505050600008888A8A8500505050600C8
:101E40000088502050880507070600FE88888850C3
:101E5000204080050505060000F8102040F8030921
:101E6000090601FF20404040804040402001090910
:101E70000602FF80808080808080808003090906C0
:101E800001FF8040404020404040800503030600A1
:101E90000248A890FF1FFFFFFFFFFFFF6000000048
:101EA0000001FF400000000000FF80000000000073
:101EB0007F83CF00000C303F87FF80000C301F86EF
:101EC0007980000C000F8C30C7838C30E78C30CFCA
:101ED000C7CC31F38C30DCECEC33B98C30D86C6C83
:101EE00033198C30D06C0C33198C30D86C0C3319FE
:101EF0008C30DC6C0E3B198C30CF7C079F198C30FA
:101F0000C77C038F19400000000000026000000041
:101F10000000061FFFFFFFFFFFF8000000000000A9
:101F200000000000000000000000000000000000B1
:101F3000000000000000000000000000000C000095
:101F400000000000000C0000000000000012000073
:101F5000000000000023000000000000002100003D
:101F600000000000004C800000000000005E8000C7
:101F700000000000009240000000000000A14000AE
:101F8000000000000121200000000000027F9000FE
:101F900000000000020010000000000007FFF80031
:101FA0000000000004000800000000000800040019
:101FB0000000000008000600000000001000020001
:101FC00000000000301E010000000000207F8100A2
:101FD0000000000041FFE0800000000043FCF080B2
:101FE00000000000873B7840000000018EDBFC60B1
:101FF000000000010FEBCC20000000021FEDB61026
:10200000000000021FDEB6100000000439CD7F087A
:102010000000000436E0FF08000000087EC0BB841A
:10202000000000187F005D86000000107FC0ED8278
:10203000000000203CC07301000000203B337F0102
:10204000000000701BE77E03800000C81DEEDE0468
:10205000C00000880FDEDC04400001240FDF3C09D3
:102060002000012607DBF8192000027203E7F013B5
:102070009000025101FFE02290000489007F80243B
:1020800048000904801E004824000BFE400000DFC9
:10209000F40010004000008002001FFFFFFFFFFF60
:1020A000FE00000000000000000000000000000032
:1020B000000000000000000000001022103C3C0E58
:1020C0001F001022100422110400102210082211F7
:1020D0000400102210083C110400102210102211DC
:1020E000040010221020221104001E1C1E3C3C0E75
:1020F00004000000000000000000000000000000DC
:1021000000000000000000000000000000000000CF
:1021100000000000000000000000000000000000BF
:1021200000000000000000000000000000000000AF
:10213000000000000000000000000000000000009F
:10214000000000000000000000000000000000008F
:10215000000000000000000000060900FE060189E2
:1021600002FE20FFFE07FE06FE000000060007013B
:1021700006060602008080808000800303030601BB
:1021800003A0A0A00507070600FF5050F850F85024
:10219000500509090600FE2070A8A07028A870202C
:1021A0000608080600FF40A8481020485408050704
:1021B000070600FF60909060989068010303060294
:1021C000038080800207070602FF408080808080B5
:1021D000400207070602FF8040404040408005055E
:1021E000050600008850F850880505050600002007
:1021F00020F820200204040602FEC04040800501B1
:1022000001060002F8020202060200C0C00406062F
:1022100006010010102040808004060606010060C0
:10222000909090906003060606010040C040404038
:10223000E00406060601006090102040F004060647
:10224000060100F020601010E005060606000010F0
:10225000305090F810040606060100F080E01010DF
:10226000E00406060601006080E090906004060627
:10227000060100F010102040400406060601006030
:1022800090609090600406060601006090907010C7
:1022900060020505060200C0C000C0C002070706B4
:1022A00002FEC0C000C040408005050506000018C1
:1022B00060806018050303060001F800F8050505B5
:1022C000060000C0300830C0040707060100609017
:1022D00010604000400506060600007090A8B0801F
:1022E00070050606060000205088F8888805060656
:1022F000060000F088F08888F004060606010060F9
:102300009080809060040606060100E09090909016
:10231000E0040606060100F080E08080F004060676
:10232000060100F080E0808080040606060100605F
:102330009080B090600406060601009090F09090A6
:1023400090030606060100E040404040E005060616
:102350000600003810101090600406060601009078
:10236000A0C0A090900406060601008080808080B6
:10237000F005060606000088D8A8A8888804060686
:1023800006010090D0B090909005060606000070FF
:102390008888888870040606060100E09090E08036
:1023A000800407070601FF609090D0B0601004061B
:1023B00006060100E09090E09090040606060100F9
:1023C000609040209060050606060000F82020205E
:1023D000202004060606010090909090906004066C
:1023E00006060100909090F0606005060606000069
:1023F0008888A8A8D88805060606000088502020EE
:102400005088050606060000888850202020040613
:1024100006060100F010204080F0030606060100C9
:10242000E080808080E00406060601008080402075
:102430001010030606060100E020202020E005031E
:10244000030600032050880501010600FEF8020281
:10245000020602048040040404060100709090709B
:102460000406060601008080E09090E00404040663
:102470000100708080700406060601001010709044
:10248000907004040406010060B0C07004060606E3
:102490000100205040E040400406060601FE609026
:1024A000907010600406060601008080E090909015
:1024B0000306060601004000C04040E0030808068D
:1024C00001FE200060202020A04004060606010036
:1024D0008080A0C0A090030606060100C0404040D6
:1024E00040E0050404060000D0A8A88804040406FF
:1024F0000100E09090900404040601006090906058
:102500000406060601FEE09090E0808004060606C0
:1025100001FE709090701010040404060100A0D019
:10252000808004040406010070C030E00406060642
:1025300001004040E0405020040404060100909057
:102540009070040404060100909060600504040685
:10255000000088A8A8500404040601009060609060
:102560000406060601FE9090907090600404040634
:102570000100F02040F003070706010020404080E2
:102580004040200107070602FF8080808080808015
:1025900003070706010080404020404080040202FB
:1025A00006010350A0FFFFFFFFFFFFFFFFFFFFFF3C
:1025B000FFFFFFFFFFFFFFFFFFFFFFFFFFFFFFFF2B
:1025C000FFFFFFFFFFFF00000006000701060606F1
:1025D00002008000808080800406060601FF2070D3
:1025E000A0A070200507070600FF304840F04040DB
:1025F000F8050505060000A8508850A8050606063F
:1026000000008850F820F8200107070602FF8080AC
:1026100080008080800407070601FF708060906062
:1026200010E0030101060105A00607070600007877
:102630008494A494847803050506010160A06000D9
:10264000E00505050600002850A0502804030306F5
:102650000100F01010040101060102F00607070650
:1026600000007884B4A4A48478040101060105F074
:102670000403030601026090600507070600FF20BF
:1026800020F8202000F803050506010140A02040A5
:10269000E0030505060101C0204020C00202020639
:1026A000020440800405050601FF9090B0D080052B
:1026B000060606000078E8E86828280101010602FD
:1026C00002800202020602FE4080030505060101A7
:1026D00040C04040E003050506010140A04000E085
:1026E000050505060000A0502850A00508080600B2
:1026F000FF40C04050703078100508080600FF40C9
:10270000C04050680810380508080600FFC0204087
:1027100030F03078100407070601002000206080A8
:10272000906005070706000040202050708888054B
:10273000070706000010202050708888050707064C
:1027400000002050205070888805070706000028E8
:102750005020507088880507070600005000205060
:102760007088880507070600002050205070888870
:1027700005060606000078A0F0A0A0B80408080628
:1027800001FE6090808090602040040707060100F1
:102790004020F080E080F00407070601002040F0B0
:1027A00080E080F00407070601002050F080E08000
:1027B000F00407070601005000F080E080F00307F6
:1027C000070601008040E0404040E00307070601A3
:1027D000002040E0404040E003070706010040A021
:1027E000E0404040E0030707060100A000E0404051
:1027F00040E00506060600007048E84848700407F7
:102800000706010050A090D0B09090040707060181
:10281000004020609090906004070706010020406F
:10282000609090906004070706010020506090902F
:10283000906004070706010050A06090909060042B
:10284000070706010050006090909060050505069E
:10285000000088502050880408080601FF1070B05E
:10286000B0D0D0E08004070706010040209090908F
:10287000906004070706010020409090909060044B
:10288000070706010020509090909060040707060B
:10289000010050009090909060050707060000101E
:1028A00020885020202004060606010080E0909039
:1028B000E0800406060601006090A0A090A0040736
:1028C0000706010040200070909070040707060181
:1028D000002040007090907004070706010020500F
:1028E000007090907004070706010050A0007090DF
:1028F0009070040606060100500070909070040766
:102900000706010020502070909070050404060016
:102910000070A8B0780406060601FE708080702062
:102920004004070706010040200060B0C0700407A3
:102930000706010020400060B0C0700407070601D0
:102940000020500060B0C070040606060100500070
:1029500060B0C070030707060100804000C040401F
:10296000E0030707060100204000C04040E00307E5
:102970000706010040A000C04040E0030606060133
:1029800000A000C04040E0040707060100306010CE
:102990007090906004070706010050A000E090903E
:1029A0009004070706010040200060909060040733
:1029B00007060100204000609090600407070601B0
:1029C000002050006090906004070706010050A0AE
:1029D0000060909060040606060100500060909030
:1029E000600505050600002000F800200404040628
:1029F000010070B0D0E004070706010040200090FD
:102A0000909070040707060100204000909090709D
:102A100004070706010020500090909070040606FD
:102A20000601005000909090700409090601FE20F4
:102A300040009090907090600408080601FE80802D
:102A4000E09090E080800408080601FE500090901D
:102A500090709060536E346B3300496E766164659C
:102A6000727300427269636B6F7574004D61696EB9
:102A7000005072696E742066726F6D20534400506E
:102A800072696E742066726F6D20534400022E2EA0
:102A9000004D61696E005072696E740043616E632F
:102AA000656C005374617274207072696E742000DA
:102AB0003F00536D6F6F7468696E6700536D6F6F81
:102AC0007468696E67005A005A005900590058002E
:102AD0005800436F7272656374696F6E00436F7262
:102AE00072656374696F6E004D61696E0046696C52
:102AF000616D656E7400544D432064726976657231
:102B000073004261636B6C6173680053746570732A
:102B10002F6D6D004A65726B00416363656C657271
:102B20006174696F6E0056656C6F636974790043F8
:102B30006F6E66696775726174696F6E0045737454
:102B40006570732F6D6D004573746570732F6D6DB7
:102B5000005A73746570732F6D6D005A73746570CD
:102B6000732F6D6D005973746570732F6D6D0059FF
:102B700073746570732F6D6D005873746570732F67
:102B80006D6D005873746570732F6D6D00416476C0
:102B9000616E6365642053657474696E6773005673
:102BA000652D6A65726B0056652D6A65726B0056FD
:102BB0007A2D6A65726B00567A2D6A65726B0056C3
:102BC000792D6A65726B0056792D6A65726B0056B5
:102BD000782D6A65726B0056782D6A65726B0041BC
:102BE0006476616E6365642053657474696E67739F
:102BF00000416D6178204500416D617820450041BC
:102C00006D6178205A00416D6178205A00416D61F4
:102C100078205900416D6178205900416D6178201C
:102C20005800416D6178205800412D7472617665BD
:102C30006C00412D74726176656C00412D72657473
:102C40007261637400412D72657472616374004136
:102C50006363656C00416363656C00416476616E1B
:102C60006365642053657474696E677300565472AB
:102C70006176206D696E005654726176206D696EC2
:102C800000566D696E00566D696E00566D61782054
:102C90004500566D6178204500566D6178205A00D8
:102CA000566D6178205A00566D6178205900566D36
:102CB0006178205900566D6178205800566D617812
:102CC000205800416476616E6365642053657474B6
:102CD000696E6773004C6F6164206D6D004C6F61AD
:102CE00064206D6D00556E6C6F6164206D6D0055D4
:102CF0006E6C6F6164206D6D00416476616E63651A
:102D0000204B00416476616E6365204B0041647620
:102D1000616E6365642053657474696E6773004403
:102D2000697361626C65207374657070657273009D
:102D30004D3834004175746F2D63616C6962726146
:102D40007465004D313137205374617274696E6758
:102D5000204175746F2D43616C6962726174696F93
:102D60006E0A54300A4D32313820543120583433F1
:102D7000205930205A300A4732380A4D3131372035
:102D80004C6576656C696E67205820417869730AD6
:102D90004732380A473020583135302046393939E2
:102DA000390A4730205A352046363030300A473904
:102DB000310A4D3231312053300A4D3430300A4D12
:102DC000393036205A3630300A4730205A2D3135C6
:102DD00020463530300A4730205A352046353030CD
:102DE0000A4739300A4D3430300A4D393036205ACE
:102DF0003936300A4D3231312053310A4732380AE0
:102E00004D313137204C6576656C696E6720646F93
:102E10006E652E0A4731320A4D3131372043616CDD
:102E20006962726174696E672E2E2E0A47343235DC
:102E30000A4D3530300A4D3131372043616C6962BB
:102E4000726174696F6E206461746120736176656C
:102E500064004C6576656C20582041786973004D9C
:102E6000313137204C6576656C696E67205820419A
:102E70007869730A4732380A473020583135302094
:102E800046393939390A4730205A352046363030EC
:102E9000300A4739310A4D3231312053300A4D342E
:102EA00030300A4D393036205A3630300A4730201B
:102EB0005A2D313520463530300A4730205A3520DA
:102EC000463530300A4739300A4D3430300A4D39F2
:102ED0003036205A3936300A4D3231312053310ADA
:102EE0004732380A4D313137204C6576656C696E52
:102EF0006720646F6E652E0A004175746F20686FDD
:102F00006D6500473238004D6F76652061786973D2
:102F1000004D61696E0045787472756465722000B9
:102F20004175746F20686F6D6500473238004D6FD2
:102F30007665205A004D6F76652059004D6F766595
:102F40002058004D6F76656D656E7400457874721B
:102F50007564657220004D6F766520302E316D6D81
:102F6000004D6F766520316D6D004D6F76652031B7
:102F7000306D6D004D6F7665206178697300486F24
:102F800074656E6420746F6F20636F6C64004578A5
:102F900074727564657220004D6F7665205A004D1D
:102FA0006F76652059004D6F76652058004D6F761D
:102FB00065205A004D6F76652059004D6F7665206B
:102FC00058005761697420666F720066696C616DA4
:102FD000656E742070757267650000506C65617372
:102FE0006520776169742E00507265737320627575
:102FF00074746F6E00746F20726573756D652070E8
:1030000072696E74005761697420666F7200666938
:103010006C616D656E74206C6F616400496E7365E0
:1030200072742066696C616D656E7400616E6420F7
:10303000707265737320627574746F6E00746F20A4
:10304000636F6E74696E756500507265737320628C
:103050007574746F6E00746F2068656174206E6F94
:103060007A7A6C65004E6F7A7A6C65206865617457
:10307000696E6700506C6561736520776169742EB5
:103080002E2E005761697420666F720066696C614C
:103090006D656E7420756E6C6F6164005761697444
:1030A00020666F720066696C616D656E742063687E
:1030B000616E676500746F20737461727400506193
:1030C000726B696E672E2E2E004368616E67696EA3
:1030D000672046696C616D656E7400554E4C4F41BA
:1030E000442046494C414D454E54004C4F414420EC
:1030F00046494C414D454E540020204E6F7A7A6C23
:10310000653A20002000456E642066696C616D653B
:103110006E74206368616E67650050757267652024
:103120006D6F726500004368616E67652066696C4B
:10313000616D656E7400556E6C6F61642066696CBC
:10314000616D656E74004C6F61642066696C616DC1
:10315000656E74004D3630302042302054256400B6
:103160004D373032203B2564004D37303220542516
:1031700064004D3730312054256400507265686515
:10318000617420437573746F6D005072656865617A
:103190007420437573746F6D005072656865617457
:1031A00020414253005072656865617420504C4163
:1031B000004261636B004E6F205344206361726470
:1031C000005072696E742066726F6D205344004324
:1031D00068616E67652053442063617264004D32FC
:1031E000310041626F7574205072696E74657200AF
:1031F0004368616E67652066696C616D656E740019
:103200004368616E67652066696C616D656E740008
:103210004D36303020423000436F6E6669677572FC
:103220006174696F6E0054656D706572617475725A
:1032300065004D6F76656D656E7400526573756DD2
:1032400065207072696E740054756E650053746FFA
:1032500070207072696E74005061757365207072B1
:10326000696E7400496E666F2073637265656E00E7
:1032700053746F70004261636B0053746F70207001
:1032800072696E74003F005072696E742061626FE3
:1032900072746564004D3234004D323520500A4D51
:1032A0003234005061757365207072696E7400501D
:1032B000726F6265205A204F6666736574004261C2
:1032C0006279737465702059004261627973746524
:1032D00070205800466C6F7700466C6F770046612F
:1032E0006E2073706565640046616E20737065655D
:1032F000640042656400426564004E6F7A7A6C65D2
:10330000004E6F7A7A6C6500537065656400537087
:10331000656564004D61696E004261627973746530
:1033200070205900426162797374657020580047BB
:10333000616D6573005072696E74657220537461BB
:103340007473004669726D77617265205665727399
:10335000696F6E004D61696E002569730025696DA6
:1033600020256973002569682025696D202569730A
:1033700000256964202569682025696D2025697309
:103380000025697920256964202569682025696DF3
:1033900020256973003E2000457874727564656469
:1033A00020746F74616C3A00256C642E25696D0081
:1033B0003E20004C6F6E67657374206A6F622074E4
:1033C000696D653A003E2000546F74616C20707224
:1033D000696E742074696D653A00436F6D706C6539
:1033E0007465643A20005072696E7420436F756E84
:1033F000743A2000436F6F6C646F776E0046616EA5
:103400002073706565640046616E20737065656445
:103410000042656400426564004E6F7A7A6C650014
:103420004E6F7A7A6C65004D61696E006F6F6F0048
:1034300000001FC07FF0DDD8FFF87FF044402480FB
:1034400000003180000024804440107CFEFEFE0419
:10345000000E000E007FC0FFE0FFE0FFE0FFE0068F
:10346000000F001F8036C03FC009001680294006AB
:10347000000F001F8036C03FC01680204010801013
:103480004008801FC037607FF05FD050500D801023
:103490004048905FD077707FF01FC0104020200F11
:1034A000007FE0FFF0E670FFF0198036C0C0300FFB
:1034B000007FE0FFF0E670FFF0198036C01980470A
:1034C000414D45204F56455200526573746F7265E9
:1034D000206661696C73616665004C6F616420737E
:1034E000657474696E67730053746F7265207365D9
:1034F0007474696E67730050726F6265205A204F52
:10350000666673657400416476616E63656420531A
:10351000657474696E6773004D61696E0050726FF7
:103520006265205A204F6666736574004D6F766938
:103530006E672E2E2E005374657070696E67206D55
:103540006F64650053656E736F726C65737320688A
:103550006F6D696E67004879627269642074687281
:103560006573686F6C640044726976657220637578
:103570007272656E7400436F6E74726F6C00486F88
:1035800074656E64004F6666004F6E00486F746528
:103590006E64005A004F6666004F6E005A00590074
:1035A0004F6666004F6E00590058004F6666004F28
:1035B0006E005800544D4320647269766572730042
:1035C000537465616C746843686F7020656E6162E6
:1035D0006C6564005900590058005800544D432050
:1035E0006472697665727300486F74656E64004832
:1035F0006F74656E64005A005A00590059005800F3
:103600005800544D43206472697665727300486FA8
:1036100074656E6400486F74656E64005A005A00E9
:103620005900590058005800544D4320647269767F
:10363000657273004D696E6920322072656164792C
:103640002E005072696E74696E672E2E2E005072B5
:10365000696E7420706175736564004361726420E3
:1036600072656D6F766564004361726420696E7384
:103670006572746564004D33310043616E6E6F7422
:1036800020656E746572207375626469723A2000F9
:103690002E0A006F70656E206661696C65642C206F
:1036A00046696C653A20006175746F25632E67006A
:1036B0006572726F722077726974696E6720746FB9
:1036C0002066696C650A004E6F7420534420707246
:1036D000696E74696E670A005344207072696E7473
:1036E000696E67206279746520002E0A0044656C5B
:1036F0006574696F6E206661696C65642C2046692B
:103700006C653A200046696C652064656C6574657B
:10371000643A0057726974696E6720746F20666935
:103720006C653A20002E0A006F70656E2066616934
:103730006C65642C2046696C653A20002E0A006F87
:1037400070656E206661696C65642C2046696C65E5
:103750003A200046696C652073656C656374656426
:103760000A002053697A653A200046696C65206F2B
:1037700070656E65643A20002066696C653A2000C9
:10378000667265736800646F696E67004E6F7720BC
:1037900000454E4420535542524F5554494E450A18
:1037A000002220706F73002220706172656E743A7F
:1037B0002200535542524F5554494E452043414CE7
:1037C0004C207461726765743A2200747279696E74
:1037D0006720746F2063616C6C207375622D676362
:1037E0006F64652066696C657320776974682074FE
:1037F0006F6F206D616E79206C6576656C732E201D
:103800004D4158206C6576656C2069733A310A0029
:103810004D3234004D323320257300534420636110
:103820007264206F6B0A006F70656E526F6F742048
:103830006661696C65640A00766F6C756D652E69EA
:103840006E6974206661696C65640A00534420697E
:103850006E6974206661696C0A00286E6F20666963
:103860006C65290043616E6E6F74206F70656E2009
:1038700073756264697220007C3C3E5E2B3D3F2F75
:103880005B5D3B2C2A225C0066616C736500747280
:103890007565004F4646004F4E006563686F3A00FD
:1038A0004572726F723A004572726F722077726958
:1038B00074696E6720746F20454550524F4D210A40
:1038C00000507265737320627574746F6E20286F78
:1038D00072204D3130382920746F20686561742062
:1038E0006E6F7A7A6C650A00507265737320627528
:1038F00074746F6E20286F72204D31303829207417
:103900006F20726573756D650A00496E7365727418
:103910002066696C616D656E7420616E64207072E2
:1039200065737320627574746F6E20286F72204DFA
:10393000313038290A004D3630303A20546F6F202C
:10394000636F6C6400486F74656E6420746F6F20E1
:10395000636F6C640A00486F74656E6420746F6FE7
:1039600020636F6C640A00496E7365727420666927
:103970006C616D656E7420616E6420707265737326
:1039800020627574746F6E20286F72204D3130384C
:10399000290A004C4F570048494748004F4B004503
:1039A00072726F723A20416C6C200020636F6E6EF1
:1039B000656374696F6E2E2E2E20005465737469D2
:1039C0006E6720004C4F570048494748004F4B0056
:1039D0004572726F723A20416C6C200020636F6EEA
:1039E0006E656374696F6E2E2E2E2000546573749D
:1039F000696E6720004C4F570048494748004F4BBD
:103A0000004572726F723A20416C6C200020636F27
:103A10006E6E656374696F6E2E2E2E200054657372
:103A200074696E6720004C4F570048494748004F63
:103A30004B004572726F723A20416C6C200020631B
:103A40006F6E6E656374696F6E2E2E2E2000546546
:103A50007374696E672000544D4320434F4E4E45AA
:103A60004354494F4E204552524F52004452565FE4
:103A7000535441545553090050574D5F5343414CE3
:103A800045090050574D434F4E460900434F4F4C98
:103A9000434F4E46090043484F50434F4E4609009E
:103AA000544849474809090054434F4F4C54485221
:103AB0005309005450574D5448525309005453541D
:103AC000455009090054504F574552444F574E092D
:103AD00000494F494E090900475354415409090010
:103AE00049484F4C445F4952554E090047434F4E99
:103AF000460909000900092042616420726573705B
:103B00006F6E7365210009204261642072657370D5
:103B10006F6E7365210009204261642072657370C5
:103B20006F6E7365210009204261642072657370B5
:103B30006F6E73652100303D2E33323500313D2EDE
:103B40003138006D6178002F3331002F3331002F71
:103B5000333100303D2E33323500313D2E313800C7
:103B60006D6178002F3331002F3331002F33310056
:103B7000303D2E33323500313D2E3138006D6178C5
:103B8000002F3331002F3331002F333100303D2EE1
:103B900033323500313D2E3138006D6178002F33DE
:103BA00031002F3331002F33310044726976657252
:103BB000207265676973746572733A0A006F7409DD
:103BC000006F7470770900733267610900733267A0
:103BD0006209006F6C6109006F6C62090073747395
:103BE0007409006673616374697665090073675FC1
:103BF000726573756C7409007374616C6C677561C0
:103C0000726409004452565354415455530053743E
:103C1000616C6C67756172642074687273002D73D7
:103C2000746172740900687973746572657369737D
:103C30000A2D656E640900626C616E6B2074696D9B
:103C400065006F66662074696D6509004F542070C9
:103C500072657761726E206861730A6265656E20B5
:103C6000747269676765726564004F54207072658D
:103C70007761726E005B6D6D2F735D090070776DFB
:103C80000A7468726573686F6C6409007473746594
:103C90007009006D73746570730900737465616CED
:103CA000746843686F70007673656E7365090050C1
:103CB000574D207363616C650043532061637475D5
:103CC000616C0900486F6C642063757272656E7474
:103CD0000052756E2063757272656E74004D4158A6
:103CE0002063757272656E7400524D532063757255
:103CF00072656E74005365742063757272656E74BC
:103D000000456E61626C6564090009006178697341
:103D10003A70776D5F7363616C652F63757272655E
:103D20006E745F7363616C652F6D6563685F6C6F44
:103D300061647C666C6167737C7761726E636F75BA
:103D40006E740A006D41290A0020647269766572FA
:103D5000206F76657274656D7065726174757265D9
:103D6000207761726E696E67212028003A2000205A
:103D700063757272656E74206465637265617365E4
:103D80006420746F20006D41290A002064726976F6
:103D90006572206F76657274656D70657261747599
:103DA0007265207761726E696E67212028003A2063
:103DB000002063757272656E74206465637265615C
:103DC00073656420746F20006D41290A00206472BD
:103DD00069766572206F76657274656D7065726163
:103DE00074757265207761726E696E672120280094
:103DF0003A20002063757272656E74206465637288
:103E0000656173656420746F20002575642025301A
:103E100032753A25303275006D41290A00206472EE
:103E200069766572206F76657274656D7065726112
:103E300074757265207761726E696E672120280043
:103E40003A20002063757272656E74206465637237
:103E5000656173656420746F2000447269766572D1
:103E6000206572726F7200636F696C2073686F7285
:103E70007420636972637569740A006F7665727481
:103E8000656D70657261747572650A00206472698F
:103E9000766572206572726F7220646574656374F2
:103EA00065643A2030780063616E63656C0072650A
:103EB00073756D656400726573756D65007061750D
:103EC00073656400706F7765726F6666002F2F618F
:103ED0006374696F6E3A0020573A0020573A0048E1
:103EE0006F74656E6420436F6F6C696E672E2E2E43
:103EF00000486F74656E642048656174696E672E52
:103F00002E2E00202F002042403A0020403A00543C
:103F10006865726D616C2052756E617761790048D9
:103F20006F74656E6420544845524D414C20525583
:103F30004E415741590042454420544845524D4155
:103F40004C2052554E4157415900202D20496E7644
:103F5000616C6964206578747275646572206E7531
:103F60006D62657220210A0048656174696E672080
:103F70006661696C656400426564206865617469A6
:103F80006E67206661696C656400546865726D6176
:103F90006C2052756E617761790042454420544827
:103FA00045524D414C2052554E41574159004865AC
:103FB0006174696E67206661696C656400486F743E
:103FC000656E642048656174696E67206661696C1E
:103FD000656400546865726D616C2052756E61771E
:103FE000617900486F74656E6420544845524D41B4
:103FF0004C2052554E41574159004D494E54454D64
:10400000502074726967676572656400486F7465F3
:104010006E64204572723A204D494E54454D500011
:104020004572723A204D494E54454D502042454408
:10403000004D415854454D50207472696767657250
:10404000656400486F74656E64204572723A204D55
:10405000415854454D50004572723A204D415854D4
:10406000454D502042454400626564002C20737920
:104070007374656D2073746F70706564212048657A
:10408000617465725F49443A200023646566696E15
:10409000652044454641554C545F004B6420004B1D
:1040A0006920004B70200000626564005049442084
:1040B0004175746F74756E652066696E69736865A5
:1040C00064212050757420746865206C61737420BD
:1040D0004B702C204B6920616E64204B6420636F11
:1040E0006E7374616E74732066726F6D2062656C9E
:1040F0006F7720696E746F20436F6E6669677572A3
:104100006174696F6E2E680A0050494420417574CD
:104110006F74756E65206661696C656421207469D1
:104120006D656F75740A00546865726D616C20521C
:10413000756E6177617900486F74656E64205448CC
:1041400045524D414C2052554E4157415900424530
:104150004420544845524D414C2052554E41574100
:10416000590048656174696E67206661696C6564B1
:1041700000486F74656E642048656174696E6720DD
:104180006661696C65640042656420686561746994
:104190006E67206661696C65640050494420417512
:1041A000746F74756E65206661696C656421205456
:1041B000656D706572617475726520746F6F2068CB
:1041C0006967680A00204B643A2000204B693A2056
:1041D00000204B703A20000A20436C6173736963BE
:1041E00020504944200A002054753A2000204B7585
:1041F0003A2000206D61783A2000206D696E3A20E7
:104200000020643A200020626961733A200050491E
:1042100044204175746F74756E6520737461727497
:104220000A00504944204175746F74756E652066AC
:1042300061696C6564212054656D70657261747587
:10424000726520746F6F20686967680A001000AD9E
:104250000330016A0150022B0170030A019004F53A
:1042600000B005E500D006D800F007CE001009C563
:1042700000300ABE00500BB700700CB100900DABBF
:1042800000B00EA600D00FA200F0109D00101299F1
:1042900000301395005014920070158E0090168B0C
:1042A00000B0178700D0188400F0198100101B7E21
:1042B00000301C7B00501D7900701E7600901F732B
:1042C00000B0207000D0216E00F0226B0010246935
:1042D0000030256600502663007027610090285E3C
:1042E00000B0295C00D02A5900F02B5600102D5444
:1042F00000302E5100502F4E0070304B009031484E
:1043000000B0324500D0334200F0343E0010363B5E
:1043100000303737005038330070392E00903A297A
:1043200000B03B2300D03C1B00F03D1100103F01CA
:1043300000F03F00001000C90210012C01400122D2
:104340000170011801B0010E01F00104015002FAE0
:1043500000B002F0003003E600D003DC009004D28D
:10436000007005C800A006BE000008B400B009AA8D
:1043700000D00BA000600E960060118C000015822A
:104380000020197800C01D6E00A0226400B0275ADA
:1043900000902C500000314600E0343C00103832D0
:1043A00000903A2800603C1E00A03D1400803E0AA8
:1043B00000203F00006F70656E005452494747452A
:1043C000524544003A20007A5F6D6178007A5F6D53
:1043D000696E00795F6D617800785F6D696E00527B
:1043E00065706F7274696E6720656E6473746F7048
:1043F000207374617475730A00456E6473746F7012
:104400007320256320256320256320256300205A1F
:104410003A0020593A0020583A00656E6473746F70
:104420007073206869743A2000486F6D696E672068
:104430006661696C6564000A53746174733A20465E
:10444000696C616D656E7420757365643A20002C2B
:10445000204C6F6E67657374206A6F623A20005457
:104460006F74616C2074696D653A200053746174D7
:10447000733A20002C204661696C65643A20002C58
:104480002046696E69736865643A20005072696EEF
:1044900074733A200053746174733A2000496E7645
:1044A000616C69642065787472756465720A0020B5
:1044B0005A3A0020593A0020436F756E7420583ADA
:1044C00000C23100001C260000F4190000D80F00C3
:1044D00000EB080000C0040000750200004001006D
:1044E0000024F4D43050C38E20C2A24017828B70B7
:1044F00011127A910D816CD90AA861E108C758663A
:1045000007615143061E4B5D05C145A7041A4111C1
:1045100004093D9803713931034036DB026533915C
:1045200002D4305402802E1D02632CEE01752AC580
:1045300001B028A001102781018F2564012B244B95
:1045400001E0223401AC211F018D200D01801FFCF0
:1045500000841EED00971DDF00B81CD200E61BC6CC
:1045600000201BBC00641AB200B219A8000A19A0EE
:10457000006A189900D117910040178B00B5168476
:104580000031167E00B31579003A157300C7146F19
:104590000058146A00EE1366008813630025135E4A
:1045A00000C7125B006C12570015125400C1115164
:1045B0000070114F0021114B00D61049008D10479B
:1045C000004610440002104200C00F4000800F3E21
:1045D00000420F3C00060F3B00CB0E3800930E3715
:1045E000005C0E3500270E3400F30D3200C10D3192
:1045F00000900D3000600D2E00320D2D00050D2CA9
:1046000000D90C2B00AE0C2900850C29005C0C276E
:1046100000350C27000E0C2600E80B2400C40B24E8
:1046200000A00B23007D0B23005A0B2100390B2126
:1046300000180B2000F80A1F00D90A1E00BB0A1E32
:10464000009D0A1D00800A1D00630A1C00470A1B0A
:10465000002C0A1B00110A1A00F7091A00DD0919BB
:1046600000C4091900AB091900920917007B091849
:1046700000630917004C09160036091600200916B8
:10468000000A091500F5081500E0081400CC08140C
:1046900000B8081400A4081400900813007D081244
:1046A000006B081300580812004608120034081165
:1046B00000230811001208110001081100F0071072
:1046C00000E0071000D0071000C0071000B0070F6F
:1046D00000A107100091070E0083070F0074070F59
:1046E0000065070E0057070E0049070E003B070D37
:1046F000002E070E0020070D0013070D0006070D02
:1047000000F9060C00ED060D00E0060C00D4060CC6
:1047100000C8060C00BC060C00B0060C00A4060B7A
:104720000099060C008D060B0082060B0077060B25
:10473000006C060B0061060A0057060B004C060AC7
:104740000042060A0038060A002E060A0024060A5D
:10475000001A060A001006090007060A00FD0509EE
:1047600000F4050900EB050900E2050900D9050977
:1047700000D0050900C7050900BE050900B50508F8
:1047800000AD050800A50509009C05080094050872
:10479000008C050800840508007C050800740508E5
:1047A000006C050700650508005D05070056050853
:1047B000004E0507004705070040050800380507BB
:1047C00000310507002A050700230507001C050620
:1047D00000160507000F050700080506000205077B
:1047E00000FB040600F5040700EE040600E80406DA
:1047F00000E2040700DB040600D5040600CF04062F
:1048000000C9040600C3040600BD040600B7040680
:1048100000B1040500AC040600A6040600A00405CF
:10482000009B04060095040500900406008A040518
:104830000085040500800406007A0405007504055F
:1048400000700405006B04050066040500610405A2
:10485000005C04050057040500520405004D0405E2
:104860000048040500430405003E0404003A040522
:104870000035040500300404002C0405002704045E
:1048800000230405001E0404001A04040016040595
:1048900000110404000D04040009040500040404CC
:1048A0000000040400FC030400F8030400F4030403
:1048B00000F0030400EC030400E8030400E4030434
:1048C00000E0030400DC030400D8030400D4030464
:1048D00000D0030400CC030400C8030300C5030395
:1048E0000024F404D9201BC40C5C0E9804C4095F96
:1048F0000265077101F405F900FB04B30048048761
:1049000000C10369005803550003034500BE023A85
:10491000008402310053022A0029022500040220EB
:1049200000E4011C00C8011900AF01170098011430
:104930000084011300710110006101100051010E8B
:104940000043010D0036010B002B010B0020010B71
:1049500000150109000C01090003010800FB000813
:1049600000F3000800EB000700E4000600DE00068C
:1049700000D8000600D2000600CC000500C70005E4
:1049800000C2000500BD000400B9000400B5000429
:1049900000B1000400AD000400A9000400A500035C
:1049A00000A20003009F0004009B00030098000386
:1049B000009500020093000300900003008D0002A8
:1049C000008B0003008800020086000200840003C0
:1049D00000810002007F0002007D0002007B0002D7
:1049E00000790002007700010076000200740002E6
:1049F0000072000100710002006F0002006D0001F2
:104A0000006C0002006A00010069000200670001FA
:104A10000066000100650001006400020062000100
:104A20000061000100600001005F0002005D000104
:104A3000005C0001005B0001005A00010059000108
:104A40000058000100570001005600010055000108
:104A50000054000100530000005300010052000107
:104A60000051000100500001004F0001004E000005
:104A7000004E0001004D0001004C0001004B000001
:104A8000004B0001004A00010049000100480000FD
:104A900000480001004700010046000000460001F8
:104AA00000450000004500010044000100430000F3
:104AB00000430001004200000042000100410000EC
:104AC0000041000100400001003F0000003F0001E4
:104AD000003E0000003E0001003D0000003D0001DE
:104AE000003C0000003C0000003C0001003B0000D6
:104AF000003B0001003A0000003A000100390000CC
:104B000000390001003800000038000000380001C2
:104B100000370000003700010036000000360000BA
:104B200000360001003500000035000000350001AE
:104B300000340000003400000034000100330000A5
:104B4000003300000033000100320000003200009A
:104B5000003200010031000000310000003100018E
:104B6000003000000030000000300001002F000085
:104B7000002F0000002F0000002F0001002E000079
:104B8000002E0000002E0001002D0000002D00006E
:104B9000002D0000002D0001002C0000002C000062
:104BA000002C0000002C0001002B0000002B000056
:104BB000002B0000002B0001002A0000002A00004A
:104BC000002A0000002A000100290000002900003E
:104BD0000029000000290000002900010028000031
:104BE0000028000000280000002800000028000124
:104BF0000027000000270000002700000027000019
:104C0000002700010026000000260000002600000A
:104C100000260000002600010025000000250000FD
:104C200000250000002500000025000000250001EF
:104C300000240000002400000024000000240000E4
:104C400000240001002300000023000000230000D6
:104C500000230000002300000023000000230001C7
:104C600000220000002200000022000000220000BC
:104C700000220000002200010021000000210000AD
:104C800000210000002100000021000000210000A0
:104C90000021000100200000002000000020000092
:104CA0000020000000200000002000000020000084
:104CB00000200001001F0000001F0000001F000076
:104CC000001F0000001F0000001F0000001F000167
:104CD000001E0000001E0000001E0000001E00005C
:104CE0000020204D363033200020204D3931340053
:104CF00020204D3931330020204D393036003A0A1A
:104D00000020286D6D2900205300205A00205900F2
:104D100020580020204D3432352046004261636B1C
:104D20006C61736820636F6D70656E736174696F19
:104D30006E3A0A002055004C0046696C616D656E44
:104D400074206C6F61642F756E6C6F6164206C658C
:104D50006E677468733A0A0020204D393030204B5A
:104D6000004C696E65617220416476616E63653ADC
:104D70000A005430204500205A00205900205800D5
:104D8000447269766572207374657070696E67200D
:104D90006D6F64653A0A00205900205800544D4355
:104DA00032313330205374616C6C4775617264200A
:104DB0007468726573686F6C643A0A00205430201E
:104DC0004500205A00205900205800487962726935
:104DD00064205468726573686F6C643A0A002054EA
:104DE00030204500205A0020590020580053746597
:104DF0007070657220647269766572206375727274
:104E0000656E743A0A0020204D383531205A005A18
:104E10002D50726F6265204F666673657400204482
:104E20000020490020204D33303420500020440021
:104E300020490020204D333031205000504944207B
:104E400073657474696E67733A0A002046002042E5
:104E50000020480020204D3134352053004D61742E
:104E6000657269616C20686561747570207061722B
:104E7000616D65746572733A0A0020204D343230DA
:104E80002053004175746F20426564204C6576653F
:104E90006C696E673A0A00204500205A00205900CC
:104EA00020580020540020530020204D323035205F
:104EB000420020453C6D61785F655F6A65726B3EBC
:104EC0000020583C6D61785F785F6A65726B3E20A8
:104ED000593C6D61785F795F6A65726B3E205A3C20
:104EE0006D61785F7A5F6A65726B3E0041647661DE
:104EF0006E6365643A20423C6D696E5F7365676DF1
:104F0000656E745F74696D655F75733E20533C6DAB
:104F1000696E5F66656564726174653E20543C6DC0
:104F2000696E5F74726176656C5F666565647261F7
:104F300074653E0020540020520020204D32303451
:104F4000205000416363656C65726174696F6E2007
:104F500028756E6974732F7332293A20503C707231
:104F6000696E745F616363656C3E20523C72657468
:104F7000726163745F616363656C3E20543C74725C
:104F80006176656C5F616363656C3E0A0020450075
:104F9000205A0020590020204D3230312058004D39
:104FA0006178696D756D20416363656C65726174CC
:104FB000696F6E2028756E6974732F7332293A0AEF
:104FC00000204500205A0020590020204D32303367
:104FD0002058004D6178696D756D20666565647255
:104FE000617465732028756E6974732F73293A0A8A
:104FF0000053746570732070657220756E69743A21
:105000000A0020204D3134392043203B20556E6961
:10501000747320696E2043656C736975730A002090
:1050200020473231202020203B20556E69747320A8
:10503000696E206D6D0020204D35363920533100CA
:1050400048617264636F6465642044656661756C71
:10505000742053657474696E6773204C6F61646566
:10506000640A002823000028230000C8000000E88C
:1050700003000000009643000096430000964300A2
:105080000020420000C8420000C84200004843001F
:1050900000D243454550524F4D20496E69746961B5
:1050A0006C697A65640A00290A0020627974657364
:1050B0003B2063726320002073746F7265642073F9
:1050C000657474696E67732072657472696576655C
:1050D00064202800202863616C63756C61746564CA
:1050E00029210A0020213D2000454550524F4D20E6
:1050F000435243206D69736D61746368202D2028CD
:1051000073746F7265642920002053697A653A20B0
:1051100000496E6465783A2000204D61726C696EBA
:105120003D563637290A00454550524F4D20766589
:105130007273696F6E206D69736D61746368202886
:10514000454550524F4D3D00290A00206279746553
:10515000733B20637263200053657474696E6773D8
:105160002053746F7265642028000A003B20454577
:1051700050524F4D20496E6465783A200055706456
:105180006174696E67207A6F666673657420696EF4
:1051900020454550524F4D3A2000454550524F4D05
:1051A000206461746173697A65206572726F722E12
:1051B0000A004175746F6C6576656C206661696C78
:1051C00065640A004175746F6C6576656C20666174
:1051D000696C6564005761726E696E673A20486F4A
:1051E0006D696E672042756D702044697669736FD2
:1051F00072203C20310A00020204486F6D652025B0
:105200007325732573206669727374002066697252
:1052100073740A00486F6D65200020746F6F206CF6
:105220006F6E6720657874727573696F6E20707227
:105230006576656E7465640A0020636F6C64206532
:105240007874727573696F6E2070726576656E74AE
:1052500065640A0020453A00205A3A0020593A0075
:10526000583A00000048420000484200002042FF37
:1052700001010000000000000000000000400000EC
:1052800030430000454300003743000040C00000A9
:1052900040430000374300002D430000404300001E
:1052A0003743000040C00000A0C000000000207490
:1052B0006F6F206C6F6E6720657874727573696F9D
:1052C0006E2070726576656E7465640A0020636F87
:1052D0006C6420657874727573696F6E2070726586
:1052E00076656E7465640A00627573793A20706140
:1052F0007573656420666F7220696E7075740A003C
:10530000627573793A2070617573656420666F7297
:1053100020757365720A00627573793A2070726F36
:1053200063657373696E670A004D313137205072BF
:105330006F6265207375636365737366756C0A00CD
:1053400020496E76616C6964206578747275646555
:10535000722000205A3A200020593A200042656409
:1053600020583A200050726F6265205A204F6666BE
:105370007365743A20003F5A206F7574206F662061
:1053800072616E676520282D3220746F2035290ADE
:10539000004D31343520533C696E6465783E206F92
:1053A0007574206F662072616E67652028302D311C
:1053B000290A00436C69636B20746F2072657375F2
:1053C0006D652E2E2E00220A00556E6B6E6F776E65
:1053D00020636F6D6D616E643A2022004545505226
:1053E0004F4D204F4B0A004E6F206D6F76652E009B
:1053F0004543484F00494E464F004552524F525385
:105400000044525952554E00434F4D4D554E49435D
:105410004154494F4E006F666600F053F553FA53FE
:105420000154085444454255473A004C756C7A4241
:105430006F74204D696E692032204F46462E002041
:105440005A00205900580020204D61783A20002051
:105450005A00205900580020204D696E3A20005310
:105460006F667420656E6473746F70733A200050B9
:1054700072696E742074696D653A20004D31313364
:105480002053002F2F20004361703A004348414DC4
:105490004245525F54454D50455241545552450086
:1054A0004D4F54494F4E5F4D4F444553005448456E
:1054B000524D414C5F50524F54454354494F4E005A
:1054C0004155544F5245504F52545F53445F5354CB
:1054D000415455530050524F4D50545F5355505006
:1054E0004F525400454D455247454E43595F504138
:1054F0005253455200434153455F4C494748545F1E
:105500004252494748544E45535300544F47474C25
:10551000455F4C494748545300534F4654574152F6
:10552000455F504F574552004255494C445F5045E6
:105530005243454E54004C4556454C494E475F44F6
:10554000415441005A5F50524F4245004155544F1B
:105550004C4556454C005052494E545F4A4F42000C
:1055600050524F4752455353004155544F524550A6
:105570004F52545F54454D5000564F4C554D455475
:1055800052494300454550524F4D0042494E415209
:10559000595F46494C455F5452414E53464552006F
:1055A00053455249414C5F584F4E5F584F46460055
:1055B0004649524D574152455F4E414D453A4D6126
:1055C000726C696E20204649524D574152455F56D4
:1055D000455253494F4E3A322E302E302E3132380A
:1055E0002045585452554445525F545950453A53FA
:1055F0006D616C6C4C6179657220534F5552434517
:105600005F434F44455F55524C3A68747470733A27
:105610002F2F636F64652E616C6570686F626A65B9
:105620006374732E636F6D2F646966667573696F3B
:105630006E2F4D41524C494E2050524F544F434FC4
:105640004C5F56455253494F4E3A312E30204D4112
:105650004348494E455F545950453A4C756C7A421F
:105660006F74204D696E692032204558545255445C
:1056700045525F434F554E543A3120555549443AAF
:1056800065353530323431312D643436642D343261
:1056900031642D626133612D6132303132366437CD
:1056A000393330660A0020284E6F742079657420E3
:1056B0006D6561737572656429002020417665729D
:1056C000616765206D6561737572656420626163F1
:1056D0006B6C61736820286D6D293A002020536D32
:1056E0006F6F7468696E6720286D6D293A202020DD
:1056F0002020202020202020202020202020530097
:1057000020204261636B6C6173682044697374612B
:105710006E636520286D6D293A20202020202020EE
:105720002000202846312E30203D2066756C6C2CE0
:105730002046302E30203D206E6F6E65290A0020F5
:1057400020436F7272656374696F6E20416D6F756F
:105750006E742F466164652D6F75743A2020202089
:105760002046006163746976653A0A00696E0042FA
:1057700061636B6C61736820436F727265637469F7
:105780006F6E2000205A0020506F736974696F6E2D
:10579000616C204572726F723A0A004E6F7A7A6CB1
:1057A0006520546970204F757465722044696D6579
:1057B0006E73696F6E733A0A002020546F703A203E
:1057C00000202046726F6E743A200020204C6566DF
:1057D000743A20004261636B6C6173683A0A00207E
:1057E0005A0043656E7465723A0A00202046726F53
:1057F0006E743A200020204C6566743A2000202008
:10580000546F703A200053696465733A0A00426528
:1058100064204C6576656C696E6720004661696C32
:10582000656420746F20656E61626C6520426564FA
:10583000204C6576656C696E670A00426564204C91
:105840006576656C20436F7272656374696F6E2054
:105850004D61747269783A000A0A426564204C65A9
:1058600076656C20436F7272656374696F6E204D4C
:1058700061747269783A00202B000A436F72726576
:1058800063746564204265642048656967687420B4
:1058900076732E2042656420546F706F6C6F677949
:1058A0003A0A00202B000A4265642048656967684F
:1058B0007420546F706F6772617068793A0A2020A3
:1058C000202B2D2D2D204241434B202D2D2B0A2006
:1058D00020207C20202020202020202020207C0A26
:1058E000204C207C20202020282B29202020207CB8
:1058F00020520A2045207C2020202020202020200B
:1059000020207C20490A2046207C20282D29204E5A
:1059100020282B29207C20470A2054207C2020206E
:1059200020202020202020207C20480A2020207CAD
:1059300020202020282D29202020207C20540A20CF
:1059400020207C20202020202020202020207C0AB5
:105950002020204F2D2D2046524F4E54202D2D2BF0
:105960000A2028302C30290A003474682070726FA5
:10597000626520706F696E742C2064697374616E47
:1059800063652066726F6D20706C616E653A2000F1
:10599000202844525952554E29004732392041752A
:1059A000746F20426564204C6576656C696E670093
:1059B0003F20284C2C522C462C4229206F757420F5
:1059C0006F6620626F756E64732E0A003F50726FAF
:1059D000626520706F696E7473202859292069737D
:1059E00020696D706C61757369626C652028322D59
:1059F00032292E0A003F50726F626520706F696E07
:105A000074732028582920697320696D706C617542
:105A10007369626C652028322D32292E0A003F28D6
:105A200056296572626F7365206C6576656C2069B6
:105A30007320696D706C61757369626C65202830C4
:105A40002D34292E0A0043757272656E74206669C2
:105A50006C653A2000456E642066696C65206C694F
:105A600073740A00426567696E2066696C65206C14
:105A70006973740A00416476616E6365204B3D0072
:105A80003F4B2076616C7565206F7574206F6620C2
:105A900072616E67652028302D3130292E0A004D45
:105AA00031313720486F7420456E64204865617439
:105AB000696E672E2E2E0A4D313034205331373027
:105AC0002054300A473238204F310A4731205932AA
:105AD00035205A31302046353030300A4D3131379B
:105AE000205265776970696E67206E6F7A7A6C658F
:105AF0000A54300A47312058313135205931373472
:105B00002046353030300A4D31303920523137306F
:105B10002054300A4731205A310A47312058313158
:105B20003520593137342046343030300A4731205F
:105B300058343520593137342046343030300A4714
:105B40003120583131352059313734204634303006
:105B5000300A473120583435205931373420463403
:105B60003030300A473120583131352059313734FF
:105B70002046343030300A473120583435205931EE
:105B800037342046343030300A47312058313135EF
:105B900020593137342046343030300A47312058CC
:105BA000343520593137342046343030300A4731CB
:105BB0002058313135205931373420463430303097
:105BC0000A47312058343520593137342046343093
:105BD00030300A473120583131352059313734209F
:105BE00046343030300A4731205834352059313767
:105BF000342046343030300A4731205A31350A4D8E
:105C00003130362053323535200A47302058302085
:105C100059300A4D31303920523136302054300A53
:105C20004D3130370A007370726561644379636C7B
:105C30006500737465616C746843686F70002064FC
:105C40007269766572206D6F64653A0900737072CF
:105C50006561644379636C6500737465616C746835
:105C600043686F700020647269766572206D6F649E
:105C7000653A09007370726561644379636C65000D
:105C8000737465616C746843686F70002064726936
:105C9000766572206D6F64653A0900737072656194
:105CA000644379636C6500737465616C7468436800
:105CB0006F700020647269766572206D6F64653A5A
:105CC000090020686F6D696E672073656E73697473
:105CD00069766974793A200020686F6D696E672073
:105CE00073656E73697469766974793A20002073FC
:105CF0007465616C746843686F70206D617820739F
:105D0000706565643A200020737465616C74684343
:105D1000686F70206D61782073706565643A20004B
:105D200020737465616C746843686F70206D61786E
:105D30002073706565643A200020737465616C742B
:105D40006843686F70206D61782073706565643A90
:105D50002000207072657761726E20666C6167202A
:105D6000636C65617265640A0020707265776172A8
:105D70006E20666C616720636C65617265640A0001
:105D8000207072657761726E20666C616720636C4B
:105D900065617265640A00207072657761726E20B9
:105DA000666C616720636C65617265640A002074CB
:105DB000656D70657261747572652070726577616A
:105DC000726E207472696767657265643A2000209C
:105DD00074656D7065726174757265207072657737
:105DE00061726E207472696767657265643A20003B
:105DF0002074656D7065726174757265207072656E
:105E00007761726E207472696767657265643A20A3
:105E1000002074656D7065726174757265207072B2
:105E2000657761726E207472696767657265643A3E
:105E30002000206472697665722063757272656EE7
:105E4000743A2000206472697665722063757272FC
:105E5000656E743A200020647269766572206375FD
:105E60007272656E743A20002064726976657220E1
:105E700063757272656E743A20004D6163726F20B3
:105E8000746F6F206C6F6E672E0A0020466C6F7700
:105E90003A200020643A0020693A0020703A00203D
:105EA0004500205A00205900204D39322058004327
:105EB000290A0061626C656420286D696E20746532
:105EC0006D70200064697300656E00436F6C642020
:105ED0006578747275646573206172652000205462
:105EE00000205200416363656C65726174696F6E76
:105EF0003A205000496E76616C696420657874724E
:105F0000756465720A0020643A0020693A002070C6
:105F10003A00536C6565702E2E2E0047322F4733A2
:105F20002062616420706172616D65746572730ACC
:105F30000050726F6265205A204F66667365743A2E
:105F40002000446F6E6520736176696E6720666914
:105F50006C652E0A0053442072656164206572727C
:105F60006F720A00446F6E65207072696E74696E9C
:105F7000672066696C650A004D32390053544F50F2
:105F80005045442E20005072696E746572207374FF
:105F90006F707065642064756520746F206572721F
:105FA0006F72732E2046697820746865206572725E
:105FB0006F7220616E6420757365204D3939392008
:105FC000746F20726573746172742E202854656D2D
:105FD000706572617475726520697320726573658E
:105FE000742E205365742069742061667465722074
:105FF00072657374617274696E67290A004E6F204E
:10600000436865636B73756D2077697468206C698C
:106010006E65206E756D6265722C204C6173742004
:106020004C696E653A20004E6F20436865636B7360
:10603000756D2077697468206C696E65206E756D6A
:106040006265722C204C617374204C696E653A2035
:1060500000636865636B73756D206D69736D617442
:1060600063682C204C617374204C696E653A200083
:106070004C696E65204E756D626572206973206E85
:106080006F74204C617374204C696E65204E756D81
:106090006265722B312C204C617374204C696E65E3
:1060A0003A20004D31313000526573656E643A20FC
:1060B000002042002050006F6B00220A00656E71C4
:1060C00075657565696E67202200504944204175E9
:1060D000746F74756E65206661696C656421204219
:1060E0006164206578747275646572206E756D6286
:1060F00065720A0042656420636F6F6C696E672E7B
:106100002E2E004265642068656174696E672E2ECC
:106110002E006F6B00307800473238205A0A473023
:106120002058383020593139302046333030300A49
:106130004D313137205072696E742061626F727414
:1061400065642E002020506C616E6E65724275662B
:1061500066657242797465733A20002046726565FF
:10616000204D656D6F72793A2000436F6D70696CD8
:1061700065643A204A756E20313020323031390A58
:1061800000207C20417574686F723A2028416C654C
:106190007068204F626A6563747320496E632E2CA9
:1061A000204C756C7A426F74204769742052657078
:1061B0006F7369746F7279290A0000204C617374DF
:1061C00020557064617465643A2000322E302E30A0
:1061D0002E3132380A004D61726C696E0020536FA7
:1061E0006674776172652052657365740A00205782
:1061F00061746368646F672052657365740A002078
:1062000042726F776E206F75742052657365740AE1
:10621000002045787465726E616C205265736574F8
:106220000A00506F77657255700A0073746172745A
:106230000A004B494C4C45442E20005072696E7444
:1062400065722068616C7465642E206B696C6C28C3
:10625000292063616C6C6564210A004B494C4C2019
:10626000636175736564206279204B494C4C2062F0
:106270007574746F6E2F70696E0A004B494C4C2018
:1062800063617573656420627920746F6F206D752A
:10629000636820696E6163746976652074696D65F1
:1062A000202D2063757272656E7420636F6D6D6151
:1062B0006E643A20004D3130342053313730205451
:1062C000300A4D313137204C6576656C696E672038
:1062D0005820417869730A4732380A4730205831CC
:1062E00035302046393939390A4730205A35204669
:1062F000363030300A4739310A4D3231312053308F
:106300000A4D3430300A4D393036205A3630300A92
:106310004730205A2D313520463530300A4730205D
:106320005A3520463530300A4739300A4D3430303E
:106330000A4D393036205A3936300A4D3231312043
:1063400053310A4732380A4D313137204C65766572
:106350006C696E6720646F6E652E0A4731320A4D94
:1063600031303920523136300A4D313137205072B8
:106370006F62696E67206265640070726F62655F4C
:10638000726577697065004175746F6C6576656CD0
:10639000206661696C6564004D3131372042656467
:1063A000206C6576656C696E67206661696C6564F2
:1063B0002E0A4730205A31300A47302045300A4DE6
:1063C0003330302050323520533838300A4D333096
:1063D00030205035302053300A4D33303020503289
:1063E0003520533838300A4D333030205035302086
:1063F00053300A4D33303020503235205338383046
:106400000A47342053310070726F62655F666169BC
:106410006C65640050726F746563746564205069C4
:106420006E0A0025311D402924301C4527232F1BCF
:106430000A0743222B1A42043803FF3604080606D3
:106440000001EE53A89AB4A4E3C0C6F038F8AA013C
:10645000AC01A801AE01D4A411241FBECFEFD1E23C
:10646000DEBFCDBF00E00CBF14E0A0E0B2E0ECEA7C
:10647000FFE103E00BBF02C007900D92A43BB10700
:10648000D9F729E1A4EBB4E001C01D92AE3CB207FC
:10649000E1F712E3CBE2D2E300E006C02197010965
:1064A000802FFE010F949087C132D10780E008074A
:1064B000A9F70E942C470D94C48F0C9400001F92E2
:1064C0000F920FB60F9211242F933F938F939F93A8
:1064D000AF93BF938091B5049091B604A091B70497
:1064E000B091B8043091B40423E0230F2D3720F489
:1064F0000196A11DB11D05C026E8230F0296A11D1E
:10650000B11D2093B4048093B5049093B604A09376
:10651000B704B093B8048091B9049091BA04A091E3
:10652000BB04B091BC040196A11DB11D8093B904B8
:106530009093BA04A093BB04B093BC04BF91AF91F5
:106540009F918F913F912F910F900FBE0F901F90B1
:1065500018952FB7F8946091B5047091B6048091A6
:10656000B7049091B8042FBF08953FB7F894809175
:10657000B9049091BA04A091BB04B091BC0426B5B3
:10658000A89B05C02F3F19F00196A11DB11D3FBF6B
:10659000BA2FA92F982F8827820F911DA11DB11DF9
:1065A000BC01CD0142E0660F771F881F991F4A95F5
:1065B000D1F708958F929F92AF92BF92CF92DF92C0
:1065C000EF92FF926B017C01D0DF4B015C01C114A3
:1065D000D104E104F104F1F091D3C7DFDC01CB0178
:1065E00088199909AA09BB09883E9340A105B105FC
:1065F00070F321E0C21AD108E108F10888EE880E94
:1066000083E0981EA11CB11CC114D104E104F10463
:1066100021F7DDCFFF90EF90DF90CF90BF90AF904C
:106620009F908F900895789484B5826084BD84B5DE
:10663000816084BD85B5826085BD85B5816085BD7D
:10664000EEE6F0E0808181608083E1E8F0E0108296
:10665000808182608083808181608083E0E8F0E0D7
:10666000808181608083E1EBF0E0808184608083C1
:10667000E0EBF0E0808181608083E1E9F0E08081FF
:1066800082608083808181608083E0E9F0E08081A6
:1066900081608083E1EAF0E0808182608083808194
:1066A00081608083E0EAF0E0808181608083E1E2C4
:1066B000F1E0808182608083808181608083E0E27C
:1066C000F1E0808181608083EAE7F0E0808184608E
:1066D00080838081826080838081816080838081EB
:1066E000806880831092C10008951F93CF93DF9339
:1066F000182FEB0161E016D1209711F460E004C07F
:10670000CF3FD10531F461E0812FDF91CF911F910F
:1067100045C1E12FF0E0E556FC4FE4914E2F50E0EB
:10672000FA013197E231F10508F09DC08827EE5853
:10673000FF4F8F4F0D94908784B5806884BDC7BD8F
:1067400097C084B5806284BDC8BD92C0809180002E
:10675000806880938000D0938900C093880088C0AF
:1067600080918000806280938000D0938B00C093E2
:106770008A007EC080918000886080938000D093E2
:106780008D00C0938C0074C08091B00080688093AD
:10679000B000C093B3006CC08091B0008062809361
:1067A000B000C093B40064C0809190008068809372
:1067B0009000D0939900C09398005AC080919000A7
:1067C000806280939000D0939B00C0939A0050C049
:1067D00080919000886080939000D0939D00C0933A
:1067E0009C0046C08091A00080688093A0008091AA
:1067F000A0008F7B8093A000D093A900C093A80035
:1068000037C08091A00080628093A000D093AB003D
:10681000C093AA002DC08091A00088608093A00042
:10682000D093AD00C093AC0023C08091200180685C
:1068300080932001D0932901C093280119C0809131
:106840002001806280932001D0932B01C0932A0104
:106850000FC080912001886080932001D0932D018A
:10686000C0932C0105C0C038D1050CF04CCF46CFE9
:10687000DF91CF911F91089590E0FC013197E231B3
:10688000F10508F04EC08827EC57FF4F8F4F0D944D
:106890009087809180008F7703C0809180008F7DEA
:1068A00080938000089580918000877FF9CF84B520
:1068B0008F7702C084B58F7D84BD08958091B0002C
:1068C0008F7703C08091B0008F7D8093B0000895D2
:1068D000809190008F7707C0809190008F7D03C0DA
:1068E00080919000877F8093900008958091A00010
:1068F0008F7707C08091A0008F7D03C08091A0009A
:10690000877F8093A0000895809120018F7707C032
:10691000809120018F7D03C080912001877F80932B
:1069200020010895CF93DF9390E0FC01EF51FC4FDD
:106930002491FC01E95DFB4F8491882361F190E093
:10694000880F991FFC01EF55FB4FC591D491FC01B5
:10695000E957FB4FA591B491611109C09FB7F89415
:106960008881209582238883EC912E230BC062308E
:1069700061F49FB7F8943881822F809583238883B0
:10698000EC912E2B2C939FBF06C08FB7F894E88113
:106990002E2B28838FBFDF91CF9108951F93CF9324
:1069A000DF93282F30E0F901E556FC4F8491F9017F
:1069B000EF51FC4FD491F901E95DFB4FC491CC2319
:1069C000C1F0162F811158DFEC2FF0E0EE0FFF1F02
:1069D000E957FB4FA591B4918FB7F894111105C0F9
:1069E0009C91ED2FE095E92302C0EC91ED2BEC9307
:1069F0008FBFDF91CF911F910895CF93DF93282F01
:106A000030E0F901E556FC4F8491F901EF51FC4F5C
:106A1000D491F901E95DFB4FC491CC2389F0811138
:106A20002BDFEC2FF0E0EE0FFF1FE359FB4FA5919A
:106A3000B491EC91ED2381E090E021F480E002C07C
:106A400080E090E0DF91CF91089508951F920F921A
:106A50000FB60F9211240BB60F922F933F934F93C3
:106A60005F936F937F938F939F93AF93BF93EF93B6
:106A7000FF93E0910802F09109021995FF91EF91BF
:106A8000BF91AF919F918F917F916F915F914F9146
:106A90003F912F910F900BBE0F900FBE0F901F9044
:106AA00018951F920F920FB60F9211240BB60F92EA
:106AB0002F933F934F935F936F937F938F939F9306
:106AC000AF93BF93EF93FF93E0910A02F0910B0213
:106AD0001995FF91EF91BF91AF919F918F917F9108
:106AE0006F915F914F913F912F910F900BBE0F903F
:106AF0000FBE0F901F9018951F920F920FB60F9216
:106B000011240BB60F922F933F934F935F936F9384
:106B10007F938F939F93AF93BF93EF93FF93E091F6
:106B20000C02F0910D021995FF91EF91BF91AF9179
:106B30009F918F917F916F915F914F913F912F9195
:106B40000F900BBE0F900FBE0F901F9018951F92C5
:106B50000F920FB60F9211240BB60F922F933F9303
:106B60004F935F936F937F938F939F93AF93BF9355
:106B7000EF93FF93E0910E02F0910F021995FF91B0
:106B8000EF91BF91AF919F918F917F916F915F91A5
:106B90004F913F912F910F900BBE0F900FBE0F9012
:106BA0001F9018951F920F920FB60F9211240BB6DB
:106BB0000F922F933F934F935F936F937F938F9396
:106BC0009F93AF93BF93EF93FF93E0910402F091F3
:106BD00005021995FF91EF91BF91AF919F918F9110
:106BE0007F916F915F914F913F912F910F900BBECD
:106BF0000F900FBE0F901F9018951F920F920FB617
:106C00000F9211240BB60F922F933F934F935F93E4
:106C10006F937F938F939F93AF93BF93EF93FF9364
:106C2000E0910602F09107021995FF91EF91BF9153
:106C3000AF919F918F917F916F915F914F913F9114
:106C40002F910F900BBE0F900FBE0F901F901895B5
:106C50001F920F920FB60F9211240BB60F922F9323
:106C60003F934F935F936F937F938F939F93AF93D4
:106C7000BF93EF93FF93E0911002F09111021995E9
:106C8000FF91EF91BF91AF919F918F917F916F9104
:106C90005F914F913F912F910F900BBE0F900FBEC0
:106CA0000F901F9018951F920F920FB60F921124FC
:106CB0000BB60F922F933F934F935F936F937F93F6
:106CC0008F939F93AF93BF93EF93FF93E091120243
:106CD000F09113021995FF91EF91BF91AF919F91A0
:106CE0008F917F916F915F914F913F912F910F9075
:106CF0000BBE0F900FBE0F901F90189508951F9315
:106D0000CF93DF93EC011D821C821F821E821986A5
:106D100081E0888782E28A871F861E86FE01B396FD
:106D2000CE01C1962FEF2193E817F907E1F711E0A3
:106D300018A3CE0113D61F8B188E198E80E48A8F6C
:106D40001B8E8FE79AE39AAB89ABDF91CF911F91AE
:106D50000895DB01ED91FC911994EF92FF921F933E
:106D6000CF93DF931F921F92CDB7DEB77C01DC017A
:106D7000D196ED91FC91D29782E069837A8319953F
:106D800020E030E04AE069817A81C701E2DF182F14
:106D9000D701D196ED91FC91D29783E01995D70157
:106DA000D196ED91FC91D29780E01995812F0F90AB
:106DB0000F90DF91CF911F91FF90EF9008950F9367
:106DC0001F93CF93DF93EC018B01E9A9FAA982E02D
:106DD0001995E9A9FAA981E0199520E030E044E18C
:106DE000B801CE01B6DF9E012D5C3F4F47E1B801EF
:106DF000CE01AFDFE9A9FAA980E0DF91CF911F9121
:106E00000F911994EF92FF921F93CF93DF93EC01B0
:106E10007B01E9A9FAA982E01995E9A9FAA981E01B
:106E2000199520E030E045E1B701CE0192DF182F3F
:106E3000882339F09E012D5C3F4F47E1B701CE0119
:106E400088DFE9A9FAA980E01995812FDF91CF9118
:106E50001F91FF90EF900895CF93DF931F92CDB7CE
:106E6000DEB79E012F5F3F4F46E473DF89810F90AD
:106E7000DF91CF910895CF93DF931F92CDB7DEB707
:106E80009E012F5F3F4F47E464DF89810F90DF91C0
:106E9000CF91089520E030E048E45BCFCF93DF93BB
:106EA000EC016A817B81D8DF88836A817B81CE0196
:106EB000E2DF89836A817B81CE01ECDF8B879E01D3
:106EC0002D5C3F4F6A817B8147E1CE01DF91CF91FD
:106ED00040CFCF93DF93EC016A817B813EDF882333
:106EE00019F0CE01DBDF81E0DF91CF9108958F9221
:106EF0009F92AF92BF92CF92EF920F93CF93DF9377
:106F00001F921F92CDB7DEB74C015B012A834983E4
:106F1000F6DEF401B382A282498147A32A8120A729
:106F200005A3E4A2C3A2C4010F900F90DF91CF91FB
:106F30000F91EF90CF90BF90AF909F908F90C9CF5F
:106F4000FC01628173813BCFCF93DF93EC01EE852F
:106F5000FF85309709F019956A817B81CE01DF9119
:106F6000CF9150CF0F93FC0182819381648F458F25
:106F7000278F068F9F01245E3F4F4BE3BC01CF015B
:106F80000F91E7CEFC0160A30895BF92CF92DF92EC
:106F9000EF92FF920F931F93CF93DF936C01D62F45
:106FA000B42EC22F7801CC2369F0F701049120E0C0
:106FB0004B2D6D2FC601D6DFFFEFEF1AFF0AC15030
:106FC000D85FF1CFDF91CF911F910F91FF90EF909C
:106FD000DF90CF90BF9008958F929F92AF92BF9213
:106FE000CF92DF92EF92FF920F931F93CF93DF9395
:106FF0005C01C62EC42FD22ED02F220F220F220FBB
:107000001ED0882379F0DC0F8D2C912CCD1751F0F8
:1070100087012D2D4C2F6C2DC501B7DFE80CF91C15
:10702000CF5FF4CFDF91CF911F910F91FF90EF9041
:10703000DF90CF90BF90AF909F908F9008950F9367
:10704000FC010150040F84A996A9941718F00817A1
:1070500028F402C0081750F0041740F42150260FFE
:1070600083A995A9961720F4281720F480E007C07B
:10707000281720F481E0261710F0F8CF81E00F9157
:10708000089581E008952EE93FE0009729F0F90185
:107090003197F1F70197F9CF0895FC0112828081B1
:1070A0008150838314820895FC0180819281980F1E
:1070B00092832181921760F494819F5F94839381DE
:1070C000890F821710F08FEF820F838381E008957C
:1070D00080E00895FC0191E08381861708F490E038
:1070E00031E0461708F030E0832F892B21E05281F0
:1070F000451708F420E02823832F8923822B089545
:10710000DC01FB01108212968C91129781831596F7
:107110008C9115978150828313968C918383089567
:10712000FB0141812381213029F0233031F468EFC4
:10713000640F04C0642F485F01C0642FCBCFDC0113
:1071400015962C9115971696ED91FC911797CF01F6
:10715000820F911D820F911D1192E817F907E1F737
:107160000895FC01A681B7818281481B8581483042
:1071700018F0A80FB11D4770382F36953695369503
:10718000562F577080E890E002C0959587955A95E4
:10719000E2F7439F402D1124669566956695E62F8C
:1071A000F0E0E40FF11DEA0FFB1F3081222311F004
:1071B000832B02C08095832380830895FB01418146
:1071C000DC0112962C911297421760F013962C91C5
:1071D0001397241738F0608115962C91621710F4DC
:1071E0002481BFCF0895CF92DF92FF920F931F9318
:1071F000CF93DF936C01EB01FA809B81913051F0CA
:1072000030F0923049F0933051F41FEF09C010E094
:1072100001E007C011E004C010E00FEF02C010E071
:1072200000E0F7FE03C0BE01C601C8DF9881900FE1
:1072300098839981910F9983FF0C99F7DF91CF91F2
:107240001F910F91FF90DF90CF9008950F931F93A0
:10725000CF93DF938901FB01C281D3814233D9F0FF
:1072600058F44531E1F0473109F1443141F5CE019F
:1072700066DFCE0112DF23C04634E1F04734E1F08F
:107280004B33E9F4B901CE014BDF8823C1F0B801DB
:10729000CE01A9DF14C0B901CE0190DF10C0CE012C
:1072A00003DF882369F0CE014ADF09C0B901CE01AE
:1072B00027DF05C08D8101C08981F801808381E0CD
:1072C000DF91CF911F910F910895CF92DF92EF92AE
:1072D000FF920F931F93CF93DF937C01D62FD42E71
:1072E000C22F122FC62EC20E6C2D611B183038F023
:1072F0000FEF20E04D2DC70135DE1850F5CF6C2F74
:10730000687F6D0F2C2F277071F097E029272F5F72
:1073100027700FEF10E001C0000F2A95EAF720E078
:107320004D2DC7011FDEDF91CF911F910F91FF906F
:10733000EF90DF90CF900895CF92DF92EF92FF927F
:107340000F931F93CF93DF937C01D62ED42FC22FA0
:10735000122FC42EC20E4C2D411B183038F00FEFE7
:1073600021E06D2DC701FEDD1850F5CF4C2F487F71
:107370004D0F2C2F277071F097E029272F5F277072
:107380000FEF10E001C0000F2A95EAF721E06D2D04
:10739000C701E8DDDF91CF911F910F91FF90EF9032
:1073A000DF90CF900895EF92FF920F931F93CF93AA
:1073B000DF93EC01162FF42EE22E01E040DE88234D
:1073C00059F02E2D4F2D612FCE01DF91CF911F91BE
:1073D0000F91FF90EF9079CFDF91CF911F910F9197
:1073E000FF90EF900895EF92FF920F931F93CF932A
:1073F000DF93EC01162FF42EE22E022F21E01FDE88
:10740000882359F02E2D4F2D612FCE01DF91CF9182
:107410001F910F91FF90EF908FCFDF91CF911F9130
:107420000F91FF90EF900895DF92EF92FF920F93EC
:107430001F93CF93DF937C01162FC42FD22ED02F12
:10744000FEDD8823F9F02D2D4C2F612FC7013DDF84
:107450002D2F4C2F612FC7016FDF6FEF6D0D610F67
:107460002D2F4C2FC70168DF4FEF4D0F4C0F2D2DE7
:10747000612FC701DF91CF911F910F91FF90EF9086
:10748000DF9023CFDF91CF911F910F91FF90EF906D
:10749000DF900895EF92FF920F931F93CF93DF93A6
:1074A0007C01D62F122FC42F040F212F4C2F6D2FAC
:1074B000C7010BDFCF5F0C13F8CFDF91CF911F9186
:1074C0000F91FF90EF900895DF92EF92FF920F934C
:1074D0001F93CF93DF93EC01162FF42EE22EAFDD36
:1074E000882329F02E2D4F2D612FCE01D3DFDF9180
:1074F000CF911F910F91FF90EF90DF900895089525
:10750000FC01E60FF11D849190E0982F88273196B9
:10751000E4918E0F911D0895FC0184910895FCDF84
:10752000882321F0823011F083E0089586E00895E9
:1075300080E00895FC018081089566E0E1CF68E075
:10754000DFCF0A96FC01849108950B96FC0184918B
:107550000895DC011496ED91FC9115973196849174
:107560000895BF92CF92DF92EF92FF920F931F93F5
:10757000CF93DF938C01E62EDC011496CD91DC9144
:107580001597CE01C9DFF82EF80184819581C7DFF8
:10759000C82EF1E0FF1203C02FE0B22E02C0BB24C0
:1075A000BA94D80114968D919C911597CADFF82E44
:1075B000F80184819581C9DFD82ED80114968D9168
:1075C0009C911597BCDFB0E6BE1538F4009729F002
:1075D000C80FD91F91E6F92E0FC0F801848195815B
:1075E000ACDFF0E4FE1538F4009729F0C80FD91F7E
:1075F00081E4F82E01C06196DE1490F4D801509613
:107600001C92509753961C92539754961C925497E1
:1076100051961C92519752961C9280E090E066C061
:10762000DF1460F38C2D90E0FE0124912F3F11F4C4
:10763000219657C0FE104CC0D80114968D919C9194
:1076400015976ADF9E012F5F3F4FFE01882311F0DF
:107650008230E1F48491D80153968C935397F901C9
:10766000249154962C935497FE013396E4915096AE
:10767000EC935097FE013496E4915196EC93519718
:10768000FE013596E4915296EC9320C08491982F98
:107690009F709250D80152969C93529782958F700A
:1076A00051968C935197F9012491822F8F705496A3
:1076B0008C93549722952F7053962C935397FE01D9
:1076C0003296E491E295EF705096EC93CE010EC0A5
:1076D000FE013296E491EB219C012E0F311DC20F69
:1076E000D31FFD1409F48ACFF3949ECFDF91CF917D
:1076F0001F910F91FF90EF90DF90CF90BF90089572
:107700004F925F926F927F929F92AF92BF92CF9271
:10771000DF92EF92FF920F931F93CF93DF931F920D
:10772000CDB7DEB72C01C62E942E622F1ADF7C0156
:10773000892B09F43AC0F20184819581F0DEB82EDC
:10774000F201138904898189C80E8289981AD92C7B
:10775000D01A212F4D2D6C2DC20171DC882311F11F
:10776000EB0CF11C195F169516951695612E712C70
:10777000D914C1F03C2D57018A2D8E19811770F450
:10778000F501049120E04D2D632FC2013983EADB1E
:10779000FFEFAF1ABF0A3981385FEECFE60CF71C56
:1077A000D394E6CFF201808901C080E00F90DF9191
:1077B000CF911F910F91FF90EF90DF90CF90BF90EE
:1077C000AF909F907F906F905F904F9008950F9330
:1077D0001F93CF93DF9300D0CDB7DEB78C01DC01D0
:1077E0005596ED91FC9156972B834A8369831995A1
:1077F0004A81480F2B816981C8010F900F900F902B
:10780000DF91CF911F910F917BCFAF92BF92DF920B
:10781000EF92FF920F931F93CF93DF931F921F92CC
:10782000CDB7DEB77C01D62E042FDC015596ED9145
:10783000FC91569729833A831995080F2981A22E26
:107840003A81B32E10E0F50121915F01222339F036
:10785000402F6D2DC70154DFD80E180FF4CF812FA4
:107860000F900F90DF91CF911F910F91FF90EF90AC
:10787000DF90BF90AF900895DF92EF92FF920F9349
:107880001F93CF93DF937C01D62FD42E8901DC0187
:107890005596ED91FC9156971995D80EC0E0F801D8
:1078A0002491222349F04D2D6D2FC70129DFD80FD8
:1078B000C80F0F5F1F4FF3CF8C2FDF91CF911F9118
:1078C0000F91FF90EF90DF900895DC0114962D91B9
:1078D0003C9115972115310509F43FC057968C91BD
:1078E0005797F901811108C03596E4915896EC93A9
:1078F0005897F9013C9611C0813041F43F96E491CC
:107900005896EC935897F901709607C03D96E4910C
:107910005896EC935897F9013E96E4915996EC935A
:10792000599758968C915897082E000C990B599698
:107930002C915997821B910927FD93955A962C916A
:107940005A97203441F0829FC001112426E0969579
:1079500087952A95E1F75B968C93089528E93AE399
:10796000FC01368B258B0895CF92DF92EF92FF9228
:107970000F931F93CF93DF938C017B016A01CB019F
:10798000FA011995D82F882311F1682FC801E9DD74
:10799000F801C189C195FFEFEF1AFF0AC701F6018F
:1079A0001995F801882351F08089C80FC701F601A5
:1079B0001995D82F682FC801D4DDEDCFD03221F032
:1079C00091898389890F01C080898C0F01C080E073
:1079D000DF91CF911F910F91FF90EF90DF90CF90AB
:1079E00008954AE95AE3C0CFCF93DF93FC01248185
:1079F00035812617370741F0EC017583648365DF15
:107A000088E99AE39E8B8D8BDF91CF910895CF9378
:107A1000DF9300D01F92CDB7DEB7611571058105E8
:107A2000910579F09B01AC0169833A834B835C83B8
:107A30000F94008829813A814B815C810F9474876F
:107A400003C060E070E0CB010F900F900F900F909B
:107A5000DF91CF910895CF92DF92EF92FF920F9333
:107A60001F9362177307840795077CF489019A01B5
:107A70006B017C01C901B8016C197D098E099F0950
:107A8000C6DF6C0D7D1D8E1D9F1D1F910F91FF90F8
:107A9000EF90DF90CF9008954F925F926F927F9218
:107AA000AF92BF92CF92DF92EF92FF920F931F930C
:107AB000CF93DF93CDB7DEB729013A019B01AC012B
:107AC00024193509460957098A899B89AC89BD89DA
:107AD000BC01CD016A197B098C099D090F9410879F
:107AE000A801970124193509460957090F9474878D
:107AF000CA01B9016A0D7B1D8C1D9D1DDF91CF91BF
:107B00001F910F91FF90EF90DF90CF90BF90AF90BB
:107B10007F906F905F904F90089580E090E008957F
:107B20000895CF92DF92EF92FF920F931F93CF931E
:107B3000DF936C017A018B01C0E0D0E0CE15DF0548
:107B400089F0D8016D918D01D601ED91FC910190E4
:107B5000F081E02DC6011995892B11F47E0102C038
:107B60002196ECCFC701DF91CF911F910F91FF902C
:107B7000EF90DF90CF9008956115710579F0FB01CA
:107B800001900020E9F73197AF01461B570BDC014C
:107B9000ED91FC910280F381E02D199480E090E05A
:107BA0000895DC01ED91FC910190F081E02D199494
:107BB0004F925F926F927F92EF92FF920F931F937B
:107BC000CF93DF93CDB7DEB7A1970FB6F894DEBFA2
:107BD0000FBECDBF7C01FA01CB0119A2223008F4FF
:107BE0002AE08E010F5D1F4F422E512C612C712C0B
:107BF000BF01A30192010F945287F901CA010150FC
:107C000011096A3014F4605D01C0695CD8016C939D
:107C1000232B242B252B61F7B801C701ADDFA196DB
:107C20000FB6F894DEBF0FBECDBFDF91CF911F918D
:107C30000F91FF90EF907F906F905F904F9008951D
:107C4000CF92DF92EF92FF920F931F93CF93DF9328
:107C5000EC016A017B012115310579F4E881F98194
:107C60000190F081E02D642FDF91CF911F910F9152
:107C7000FF90EF90DF90CF9019942A303105D9F41E
:107C800077FF18C06DE28DDF8C0144275527BA01BC
:107C90004C195D096E097F092AE0CE0189DF800F4A
:107CA000911FDF91CF911F910F91FF90EF90DF9087
:107CB000CF9008952AE0B701A601CE01DF91CF91C0
:107CC0001F910F91FF90EF90DF90CF9071CF9A01AD
:107CD000AB01770F660B770BB3CFCF93CFB7F89489
:107CE0008091C004811127C0ECE5F4E08491E6E1C5
:107CF000F4E09491E82FF0E0EE0FFF1FEF55FB4FFB
:107D0000A591B491EC91E92321F461E085E30E940F
:107D1000CE3461E085E30E9492348CB580618CBDE5
:107D20008CB580648CBD61E084E30E94923461E094
:107D300083E30E9492348091C0048F5F8093C004DB
:107D4000CFBFCF910895CF92EF920F93FC0113AE66
:107D500014AE15AE0496CBD80F91EF90CF90089546
:107D6000CF92DF92EF92FF921F93CF93DF93EC01BC
:107D700080E090E00F94A88425ED34E045E352E4E0
:107D80000F94468620E030E04AE754E40F940F84D5
:107D90006B017C012AE037ED43EA5CE369857A8573
:107DA0008B859C850F942F839B01AC01C701B60185
:107DB0000F94468626E636E646EA5EE30F940F8485
:107DC00020E030E040E85FE30F942E830F947C8442
:107DD000162FE881F9810480F581E02D603118F5D6
:107DE00061E0CE0119952AE037ED43EA5CE369854D
:107DF0007A858B859C850F942F839B01AC01C701ED
:107E0000B6010F9446862CEE31E548E35EE30F940D
:107E10000F8420E030E040E85FE30F942E830F945E
:107E20007C84162F03C060E0CE011995612FCE012E
:107E3000C6D2612F70E080E090E00F94AA842D8577
:107E40003E854F8558890F9446860F947C84CE01D9
:107E5000DF91CF911F91FF90EF90DF90CF9092C272
:107E6000FC01258736874787508B7ACFCF92DF92E8
:107E7000EF92FF92CF93DF93EC01DED2682F70E098
:107E80006F5F7F4F072E000C880B990B0F94AA840D
:107E900020E030E040E05DE30F9446866B017C011A
:107EA000E881F9810680F781E02DCE0119958111D5
:107EB00005C026E636E646EA5EE304C02CEE31E570
:107EC00048E35EE3C701B6010F9446866B017C016F
:107ED0002AE037ED43EA5CE369857A858B859C85EA
:107EE0000F942F839B01AC01C701B6010F940F843F
:107EF00025ED34E045EB5FE30F940F8420E030E0A4
:107F00004AE754E40F9446860F947C84CB01DF91BA
:107F1000CF91FF90EF90DF90CF900895DC01ED912D
:107F2000FC910084F185E02D19956115710581059D
:107F3000910539F06F3F7F4F8F4F9F4F21F080E0C9
:107F4000089582E0089581E00895DC01ED91FC91AF
:107F50000484F585E02D199583500895DC01ED9199
:107F6000FC910088F189E02D19958F5F08956031AB
:107F7000710509F441C088F46230710509F454C0F8
:107F800020F4672B09F458C008956430710509F492
:107F900043C068307105C1F1089560347105E1F0A6
:107FA00020F46032710501F108956038710561F0C7
:107FB0006115714009F048C0DC01ED91FC91028827
:107FC000F389E02D60E03FC0DC01ED91FC91028877
:107FD000F389E02D61E037C0DC01ED91FC9102886E
:107FE000F389E02D62E02FC0DC01ED91FC91028865
:107FF000F389E02D63E027C0DC01ED91FC9102885C
:10800000F389E02D64E01FC0DC01ED91FC91028852
:10801000F389E02D65E017C0DC01ED91FC91028849
:10802000F389E02D66E00FC0DC01ED91FC91028840
:10803000F389E02D67E007C0DC01ED91FC91028837
:10804000F389E02D68E019940895DC01ED91FC912D
:108050000488F589E02D1995893048F4E82FF0E07F
:10806000EE0FFF1FE85EFC4F80819181089580E054
:1080700090E00895DC01ED91FC91008CF18DE02DF4
:108080001995843030F4E82FF0E0EC5EFC4F8081ED
:10809000089580E00895DC01ED91FC910280F38168
:1080A000E02D61E01995862F0895FC0185810895E2
:1080B000DC0115966C931597ED91FC91262F30E01D
:1080C00040E050E00190F081E02D61E11994DC0185
:1080D000ED91FC910280F381E02D62E11994FC01A5
:1080E000268137818085482F4F70842FB90190E019
:1080F0000895DC019A01462F4F7016962C9316971F
:1081000017963C931797942F9F7018968C911897F9
:10811000807F892B18968C931897ED91FC9111977D
:1081200050E00190F081E02D63E1CD011994FC0154
:1081300067A170A592A581A591700895DC0197961D
:108140004C93979798965C93989799966C93999778
:108150009A968C919A9770FB80F99A968C939A973D
:10816000ED91FC9111979A01AB0151700190F08152
:10817000E02D6DE6CD011994DC016F7097962C917E
:108180009797207F262B97962C939797ED91FC91AC
:10819000119798963C91989799964C9199979A96A1
:1081A0005C9151700190F081E02D6DE61994DC0135
:1081B0006F7098963C919897307F362B98963C93A9
:1081C0009897ED91FC91119797962C919797999686
:1081D0004C9199979A965C9151700190F081E02DA5
:1081E0006DE61994DC016F7799964C9199974078D8
:1081F000462B99964C939997ED91FC9111979796F0
:108200002C91979798963C9198979A965C9151707B
:108210000190F081E02D6DE61994FC0191A5990F74
:108220009595292F092E000C330B20743327220F2C
:10823000331F892F8F77822B0895DC01ED91FC91FC
:108240000280F381E02D6FE61994DC01ED91FC9141
:108250000084F185E02D1995CB0193700895DC0120
:10826000ED91FC910084F185E02D199577FB88272D
:1082700080F90895DC01ED91FC910084F185E02DF9
:1082800019958F710895DC01ED91FC910084F185C1
:10829000E02D1995892F81700895DC01ED91FC91F5
:1082A0000084F185E02D199591FB882780F90895C8
:1082B000DC01ED91FC910084F185E02D199592FB94
:1082C000882780F90895DC01ED91FC910084F18507
:1082D000E02D199593FB882780F90895DC01ED9135
:1082E000FC910084F185E02D199594FB882780F995
:1082F0000895DC01ED91FC910084F185E02D199544
:1083000095FB882780F90895DC01ED91FC910084AC
:10831000F185E02D199596FB882780F90895DC01F9
:10832000ED91FC910084F185E02D199597FB88274C
:1083300080F90895FC01228133818481482F4F7098
:10834000842FB90190E00895DC019A01462F4F7007
:1083500012962C93129713963C931397942F9F7019
:1083600014968C911497807F892B14968C93149774
:10837000ED91FC91119750E00190F081E02D60E1CA
:10838000CD011994DC016F7112968C911297807E49
:10839000682B12966C931297ED91FC911197262FF2
:1083A00013963C91139714968C911497482F4F7005
:1083B00050E00190F081E02D60E1CD011994DC01E5
:1083C0006F7113968C911397807E682B13966C9324
:1083D0001397ED91FC91119712962C911297362FCD
:1083E00014968C911497482F4F7050E00190F081B3
:1083F000E02D60E1CD011994DC016F7014968C9131
:108400001497807F682B14966C931497ED91FC91D0
:10841000119712962C91129713963C911397462F11
:108420004F7050E00190F081E02D60E1CD01199492
:10843000FC0182818F710895FC0183818F71089501
:10844000DC016770962F9295907F92966C9192972F
:108450006F78692B92966C939297ED91FC9111979E
:1084600092962D913D914D915C9195970190F0815F
:10847000E02D6CE6CD011994DC0192968C919297D7
:1084800060FB87F992968C939297669567709396A6
:108490008C919397887F682B93966C939397ED912B
:1084A000FC91119792962D913D914D915C919597EC
:1084B0000190F081E02D6CE6CD011994DC019396DA
:1084C0008C91939760FB87F993968C93939761FBBC
:1084D000882780F994966C9194976E7F682B949678
:1084E0006C939497ED91FC91119792962D913D91FB
:1084F0004D915C9195970190F081E02D6CE6CD0156
:108500001994DC0194962C91949760FB21F9949630
:108510002C939497ED91FC91119792962D913D910A
:108520004D915C9195970190F081E02D6CE6199446
:108530006F70DC0195962C919597207F622B959614
:108540006C939597ED91FC91119792962D913D9199
:108550004D915C9195970190F081E02D6CE6199416
:10856000CF93DF93EC01E881F9810280F381E02D64
:108570006CE619956AA37BA38CA39DA3DF91CF9191
:108580000895CF93DF93EC01EBDF8AA1829587708A
:10859000DF91CF910895CF93DF93EC01E1DF9AA1B2
:1085A000991F9927991F8BA18770880F892BDF91BD
:1085B000CF910895CF93DF93EC01D2DF9BA1991F58
:1085C0009927991F8CA18170880F892BDF91CF91FA
:1085D0000895CF93DF93EC01C3DF8CA18695817062
:1085E000DF91CF910895CF93DF93EC01B9DF8DA197
:1085F0008F70DF91CF910895DC0192964D935D933A
:108600006D937C939597ED91FC910190F081E02D15
:108610009A01AB016CE619946F70DC0192962C9173
:108620009297207F622B92966C939297ED91FC919A
:10863000119792962D913D914D915C919597019056
:10864000F081E02D6CE61994CF93DF93EC0188DF85
:108650008AA18F70DF91CF910895CF92DF92EF9230
:10866000CF93DF93EC01E881F9810280F381E02D63
:1086700060E019956B01E82E23E0E222CA8ADB8ACA
:108680002E2D23709C899C7F922B9C8B8E2DB60166
:1086900090E0DF91CF91EF90DF90CF900895DC01D3
:1086A0009A01462F437052962C93529753963C93BF
:1086B0005397942F937054968C9154978C7F892B59
:1086C00054968C935497ED91FC91119750E0019042
:1086D000F081E02D60E0CD011994DC0152968C917F
:1086E000529760FB82F952968C935297ED91FC91D0
:1086F0001197282F53963C91539754968C915497E9
:10870000482F437050E00190F081E02D60E0CD01F2
:108710001994DC0152968C91529760FB84F9529621
:108720008C935297ED91FC911197282F53963C9181
:10873000539754968C915497482F437050E0019072
:10874000F081E02D60E0CD011994DC0153968C910D
:10875000539760FB80F953968C935397ED91FC915E
:10876000119752962C915297382F54968C9154977A
:10877000482F437050E00190F081E02D60E0CD0182
:108780001994CF93DF93EC0168DF8A8982FB8827F5
:1087900080F9DF91CF910895FC0123A534A585A52B
:1087A000482F4F73842FB90190E00895DC019A019E
:1087B000462F4F739B962C939B979C963C939C972C
:1087C000942F9F739D968C919D97807C892B9D966D
:1087D0008C939D97ED91FC91119750E00190F08161
:1087E000E02D60E7CD011994CF93DF93EC0161E0B8
:1087F00088810E94923461E08C810E94923462E010
:108800008A810E949234E881F981EF51FC4FE49112
:10881000EE83EA81FB81EF51FC4FE491EF83EC8121
:10882000FD81EF51FC4FE491E887DF91CF910895EE
:108830009F92AF92BF92CF92DF92EF92FF920F93EF
:108840001F93CF93DF938C01942E87E0C82ED12CF9
:10885000E12CF12CC0E0A62EB12CC501911019C05D
:108860000E2C02C0959587950A94E2F780FF02C00E
:1088700061E001C060E0F80180810E94CE3461E0D7
:10888000F80184810E94CE34F8018281911016C0D3
:1088900007C00C2C02C0959587950A94E2F7E6CFA5
:1088A0000E94FD3421E030E0892B11F420E030E01B
:1088B0000E2C01C0220F0A94EAF70DC00E94FD346D
:1088C00021E030E0892B11F420E030E00C2C01C0D5
:1088D000220F0A94EAF7C22B60E0F80184810E941B
:1088E000CE34FFEFEF1AFF0A81E0C81AD108E8E0A2
:1088F000EE16F10409F0B1CF8C2FDF91CF911F91CB
:108900000F91FF90EF90DF90CF90BF90AF909F902E
:1089100008950F931F93CF93DF938C01D62F672F6A
:1089200041E086DFC82F41E06D2FC80181DF2C2F89
:1089300030E0322F2227A901482BCA01DF91CF91C5
:108940001F910F9108950F93FC0130E080E092E1B8
:10895000AAE7B0E0481759076A077B0740F4B695C5
:10896000A795979587953F5F3630A1F737E091E05F
:108970009327222311F020E501C020E7892F869557
:108980000C70082B022B0083917091830F91089536
:108990002091BF04222399F04FB7F8942091BF048F
:1089A000213059F42DB32093BD043DB32091BE0472
:1089B000209523232DBB4FBF02C04093BD048CBD27
:1089C0009DBD08958EBD00000DB407FEFDCF8EB590
:1089D00008950CB405FC0DC09EBD00000DB407FE4B
:1089E000FDCF9EB58EBD00000DB407FEFDCF8EB548
:1089F00008958EBD00000DB407FEFDCF8EB59EBD5F
:108A000000000DB407FEFDCF9EB508958091BF0410
:108A1000882361F09FB7F8942091BF048091BD0432
:108A2000213019F48DBB9FBF08958FBF0895CF9358
:108A3000DF93FC01128213828481807F84831582FC
:108A4000168217828085807F8087218732874387BF
:108A5000548780E090E0A0E0BFE385879687A787F2
:108A6000B08B8EE293E091838083128A138A84898B
:108A70008C7F848B158A168A8789807F878B108EDE
:108A8000118E828D807F828F138E148E158E868D2F
:108A90008E7F868F178E10A281A1807881A3DF013F
:108AA000929685E0ED0119928A95E9F717A210A632
:108AB00011A682A58E7F82A713A614A685A5807C09
:108AC00085A786A58C7F86A770AB67A712AA11AA77
:108AD000DF91CF910895FC0187A50C94CE34AF921D
:108AE000BF92CF92DF92EF92FF920F93CF93DF93DB
:108AF0001F921F92CDB7DEB75C01F62EFC0181A953
:108B000092A9892B09F44EC060E0C501E4DF41E081
:108B10006F2DF50181A992A98BDE60E070E0F5016F
:108B200081A992A9F6DE60E070E0F50181A992A921
:108B3000F0DE61E0C501CFDF60E0C501CCDF41E0E0
:108B40006F2DF50181A992A973DEF501818B41E0BA
:108B500060E081A992A96CDEC82ED12CE12CF12C09
:108B6000FE2CED2CDC2CCC2441E060E0F50181A949
:108B700092A95EDEC82AFE2CED2CDC2CCC2441E030
:108B800060E0F50181A992A953DEC82AFE2CED2CE4
:108B9000DC2CCC2441E060E0F50181A992A948DEFB
:108BA000C82A41C0409114025091150260911602EA
:108BB000709117020CE021E0CE010196C4DE89819C
:108BC0009A81E6DE60E0C50186DF8F2DFBDE80E066
:108BD00090E0FFDE80E090E0FCDE61E0C5017BDF3D
:108BE00060E0C50178DF8F2DEDDEF501818B80E03F
:108BF000E9DEC82ED12CE12CF12CFE2CED2CDC2C46
:108C0000CC2480E0DFDEC82AFE2CED2CDC2CCC242A
:108C100080E0D8DEC82AFE2CED2CDC2CCC2480E0B1
:108C2000D1DEC82AF3DE61E0C50155DFC701B60118
:108C30000F900F90DF91CF910F91FF90EF90DF9009
:108C4000CF90BF90AF9008954F925F926F927F92B6
:108C50008F929F92AF92BF92EF92FF920F931F93CA
:108C6000CF93DF931F921F92CDB7DEB77C014901EE
:108C70005A01162F1068FC0181A992A925016624CA
:108C80007724892BA9F060E0C70125DF41E0612F3F
:108C9000F70181A992A9CCDDF701818BB20181A9ED
:108CA00092A937DEB401F70181A992A932DE1CC076
:108CB00040911402509115026091160270911702B2
:108CC0000CE021E0CE0101963EDE89819A8160DED2
:108CD00060E0C70100DF812F75DEF701818BC201E3
:108CE00078DEC40176DE92DE61E0C701F4DE0F902B
:108CF0000F90DF91CF911F910F91FF90EF90BF9058
:108D0000AF909F908F907F906F905F904F9008955D
:108D1000CF93DF93EC0161E08FA50E94923461E074
:108D2000CE01D9DE89A99AA9009709F05DDD8A896B
:108D30009B892C89A22FA370AC016A2F70E0CE0111
:108D4000AEDC4AA15BA16CA17DA1CE0155DC4FA197
:108D500058A569A57AA57170CE01F0D98BA59CA5FF
:108D60002DA5A22FAF73AC016A2F70E0CE011EDDDE
:108D70008A819B812C81A22FAF70AC016A2F70E099
:108D8000CE01E2DA68E0CE0147DCE881F9810688AD
:108D9000F789E02D61E0CE01DF91CF911994DC01DC
:108DA000ED91FC910280F381E02D64E01994F7DFEE
:108DB00064FB882780F90895CF93DF93EC01F7DFF8
:108DC000811105C0CE0140DC91E0811101C090E02D
:108DD000892FDF91CF910895FC01258936898789F4
:108DE000482F4F70842FB90190E00895DC019A015B
:108DF000462F4F7055962C93559756963C93569701
:108E0000942F9F7057968C915797807F892B5796F8
:108E10008C935797ED91FC91119750E00190F08160
:108E2000E02D64E1CD011994FC01208D318D828DFE
:108E3000482F4F70842FB90190E00895DC01ED9127
:108E4000FC910280F381E02D61E71995862F08954A
:108E500080E090E0089508950E941333FCDF0F94A2
:108E60007182C0E0D0E00F9403832097E1F30E9469
:108E70000000F9CFCF93DF931F92CDB7DEB790916B
:108E8000D004292F2370233041F091609260909399
:108E9000D00489830E948B5589810F90DF91CF91F7
:108EA0000C9499558091D004982F9370913031F0A3
:108EB00081608D7F8093D0040C9492550895CF9358
:108EC000DF93EC018991882319F00E949955FACF1C
:108ED000DF91CF9108950F931F93CF938C01C62FED
:108EE000F80181918F01882331F0CC2321F00E9479
:108EF0009955C150F5CFCF911F910F910895CF9300
:108F0000DF93FC018491EF012196882321F00E94D8
:108F10009955FE01F7CFDF91CF9108950F931F93DD
:108F2000CF93DF93CDB7DEB727970FB6F894DEBFA8
:108F30000FBECDBF6330B1F038F46130B1F06230B4
:108F400049F525E437E113C0653031F040F0663073
:108F500009F525E537E10BC021E537E108C02DE42F
:108F600037E105C029E437E102C021E437E19F93EE
:108F70008F933F932F938E010F5F1F4F1F930F937C
:108F80000F94AA8CC8019BDF0F900F900F900F9049
:108F90000F900F9027960FB6F894DEBF0FBECDBF8F
:108FA000DF91CF911F910F9108951F93CF93DF937E
:108FB0001F92CDB7DEB7182F811102C080E201C029
:108FC00084E2611102C090E001C092E0892B6983C4
:108FD00051DF9091D00410FB92F9892F698160FBD9
:108FE00083F98093D0040F90DF91CF911F91089562
:108FF0006091D00462FB992790F9891721F063FBF7
:10900000662760F9D2CF0895CF93C82F81E0F0DFB3
:10901000C11102C082E001C083E02CDF9091D00436
:10902000C0FB94F99093D004CF9108959091D0040F
:10903000929591708913E8CF0895CF93C82F80E05F
:10904000D7DF8C2F8F738068CF9114CFCF93C82F29
:1090500080E0CEDF8C2F8F738064CF910BCF1F9376
:10906000CF93DF931F92CDB7DEB7182F81E06983CE
:10907000BFDF6981862F8068FDDE812F8F70806859
:109080000F90DF91CF911F91F5CE80E0B1DF81E0AD
:10909000F1DE6FE070E080E090E00C94DA32CF9384
:1090A000DF93C0E06C2F80E0DADFFCDED1E1D1504D
:1090B00039F080E00E94995580E00E949955F7CFE1
:1090C000CF5FC03279F7DF91CF910895CF92DF92D1
:1090D000EF92FF921F93CF93DF931F921F92CDB712
:1090E000DEB769837A83B2DFDDDE6981C62E7A81DD
:1090F000D72E11E1115069F0F601E590F4908F2D13
:109100000E9499558E2D0E94995582E0C80ED11C5F
:10911000F1CF0F900F90DF91CF911F91FF90EF90C3
:10912000DF90CF900895CF92DF92EF92FF920F934E
:109130001F93CF93DF931F92CDB7DEB7982F623086
:1091400010F06250985FC62EC29480EFC8228A0148
:10915000D12C6D2D6C0D892F998381DFA3DEF80151
:10916000E590F4908F2D0E9499558E2D0E9499556F
:10917000D3940E5F1F4F998180E1D812EACF0F90F0
:10918000DF91CF911F910F91FF90EF90DF90CF90E3
:109190000895CF92DF92EF92FF920F931F93CF9398
:1091A000DF93C42E623010F06250805F982F917070
:1091B000D92EC82FC695D62FD295D07F89E3E82E19
:1091C00088E1F82E01E0F7011491602F6D0F8C2FCC
:1091D00046DF68DECC2059F0D11002C0812F01C0DB
:1091E00080E00E949955DD2029F0812F04C080E0A5
:1091F0000E94995580E00E9499550F5FFFEFEF1A8A
:10920000FF0A053001F7DF91CF911F910F91FF9079
:10921000EF90DF90CF9008958F929F92AF92BF9280
:10922000DF92EF92FF920F931F93CF93DF93D82E8D
:1092300069E10F941F8720E1929FC001112469E129
:1092400070E00F943F8780E090E85C0102C0B59425
:10925000A7946A95E2F711E0ED2CF12C612F8CE0D8
:10926000FEDE20DE20E030E000E0490189E1880EEA
:10927000911CE814F90434F42E153F0534F0C0E0D5
:10928000D0E004C0CFEFDFEF01C0E501113051F0B5
:109290001D3041F0033011F4C16006C0011104C05B
:1092A000D06802C0CFEFDFEF8D2F0E9499558C2F31
:1092B0000E9499550F5F940124363105B1F61F5F66
:1092C0001E3061F68CE0B9DEEDDD80E20E9499553A
:1092D00029E02D1530F464E0C70120DE8EE397E12C
:1092E00005C063E0C7011ADE8AE397E1DF91CF9101
:1092F0001F910F91FF90EF90DF90BF90AF909F90E4
:109300008F90FDCDCF93C82F85E097DECBDDC111C7
:1093100002C0C6E001C0C4E080E00E9499558C2FD5
:10932000CF910C94995580E081DE69ED77E180E082
:1093300090E0CCDE69EB77E180E190E0C7DE69E99F
:1093400077E180E290E0C2DE69E777E180E390E0D8
:10935000BDDE49E158E160E080E0E5DE49EF57E13C
:1093600061E080E0E0DE49E557E161E085E0DBDED9
:1093700080E0C8CF1F93CF93DF931F92CDB7DEB7A6
:10938000182F80E1698359DE8DDD6981662351F0F4
:10939000111102C012E001C010E080E00E94995556
:1093A000812F04C080E20E94995580E20F90DF91E6
:1093B000CF911F910C949955CF92DF92EF92FF922B
:1093C0000F93CF93DF93C82F6B017A01D22F813097
:1093D00049F028F0823049F0833039F008C081E04C
:1093E0002CDE05C081E129DE02C089E026DE5ADDDF
:1093F00063E0C60193DDDD2349F08AE10E949955BF
:1094000063E0C7018BDD011106C015C0002399F090
:1094100085E397E174DD41E04D276C2F85E0B9DEEF
:109420004D2F6C2F89E0DF91CF910F91FF90EF903E
:10943000DF90CF90AECEDF91CF910F91FF90EF9064
:10944000DF90CF9008950F93CF936115710589F048
:10945000C1E0681779073CF49C01261B370B2330C9
:10946000310544F406C09B01281B390B233031051C
:109470000CF4C0E02091180221702C1711F001E0CB
:1094800001C0042F2C2FAB01BC0180E095DF80913F
:109490001802C0FB80F980931802CF910F910895B4
:1094A0000F93CF936115710589F0C1E068177907B3
:1094B0003CF49C01261B370B2330310544F406C0D5
:1094C0009B01281B390B233031050CF4C0E020919F
:1094D000180222FB222720F92C1711F001E001C00D
:1094E000042F2C2FAB01BC0181E066DF80911802B4
:1094F000C0FB82F980931802CF910F910895CF930A
:10950000C82F86E09ADDCEDC63E08C2F90E006DD8C
:1095100085E2CF910C949955CF92DF92EF92FF9212
:109520000F931F93CF93DF93CDB7DEB727970FB677
:10953000F894DEBF0FBECDBF8C0188E07EDDF80160
:1095400060817181828193812CE3C22ED12CE12C28
:10955000F12CA70196010F945287CA01B901A70106
:1095600096010F9452878E010F5F1F4F24363105ED
:1095700098F47F936F933F932F938BE297E19F93A0
:109580008F931F930F930F94AA8C0FB6F894DEBF9E
:109590000FBECDBF85E012C07F936F933F932F9393
:1095A00083E297E19F938F931F930F930F94AA8C5D
:1095B0000FB6F894DEBF0FBECDBF86E0F801E80F0E
:1095C000F11D80E280836EDC66E0C80184DC2796B2
:1095D0000FB6F894DEBF0FBECDBFDF91CF911F91C4
:1095E0000F91FF90EF90DF90CF900895CF93DF938E
:1095F000EC0186E122DD56DC63E0CE018FDC85E202
:10960000DF91CF910C949955CF9388E116DD4ADC18
:1096100082E797E00E94EE93C82F65E182E797E02A
:109620005ADCC53128F480E20E949955CF5FF9CF0A
:10963000CF9108950E94A2954091B70D90913E025E
:109640002091C00D3091C10D60916A0270916B0242
:109650002627372760919C0D70919D0D262737276F
:10966000949FA0011124440F452F441F550B519581
:1096700024273527A9014827CA012091C604309123
:10968000C7042817390731F09093C7048093C604A4
:1096900081E0089580E008954F925F926F927F92EB
:1096A0008F929F92AF92BF92CF92DF92EF92FF92F2
:1096B0001F93CF93DF9300D01F92CDB7DEB7F82E64
:1096C000811104C0B7DF882309F467C00E94A29506
:1096D000182F0F94947E69837A838B839C83A09048
:1096E0006A02B0906B026091980D7091990D809113
:1096F0009A0D90919B0D0F9477842B013C01C090A3
:109700009C0DD0909D0D8090C00D9090C10D6091EA
:10971000BC0D7091BD0D8091BE0D9091BF0D0F9449
:109720007784DC01CB014F2DB4018DDE4F2DB601C6
:10973000C201B6DE2091B70DE22EF12C11110DC041
:1097400090913E0297FD09C0929F900111247901EA
:10975000EE0CEF2CEE1CFF08F19424E62E9DC001C8
:109760002F9D900D112481589F4F6FEF70E00F9443
:109770003F87862FC4DECE010196CEDEC50136DFDF
:10978000EF2811F0812FBEDD61E01C141D041CF0D8
:1097900060E080E001C0812FEDDD0F900F900F9011
:1097A0000F90DF91CF911F91FF90EF90DF90CF90BE
:1097B000BF90AF909F908F907F906F905F904F90F1
:1097C0000895E2E7F7E080E09191992311F089276D
:1097D000FBCF9091C80491110BC091E02091C5047A
:1097E000281301C090E09093C40491E09093C804C2
:1097F0009091C40491118093C50481E0911101C03E
:1098000080E008950E94A295982F81E02091C304E2
:10981000291302C080E008959093C3040895811134
:1098200003C0CFDF882311F0EFDEECCF0895CF9394
:10983000C82F0E94759AC11104C09091C204981754
:1098400021F08093C204CF91E7CCCF910895CF93BC
:10985000C82F0E9485558091D0048E7F8093D004BC
:109860008C2F1ADF8C2FDBDF8C2FE1DF0E948555D8
:109870008091D0048E7F8093D004CF91089561E0D1
:1098800081E093DB61E081E090DB80E0BDCB0E9472
:1098900085558091D0048E7F8093D004F0DFF5DB76
:1098A000FEDB41DD81E0D3DF0E9485558091D0044D
:1098B0008E7F8093D00408950E9485558091D004B6
:1098C0008E7F8093D004E1DB61E081E06EDB0E945B
:1098D00085558091D0048E7F8093D00408950E9496
:1098E00085558091D0048E7F8093D004C8DFCDDB76
:1098F00061E081E05ADB0E9485558091D0048E7F23
:109900008093D004089580E0A2CF9091C10498176D
:1099100029F08093C1048111BACFCECF0895EEED26
:10992000F4E083AF64AF08954AE050E0BC018EEDEF
:1099300094E00C94673EEF92FF920F931F93CF93A6
:10994000DF937A016F3F71058105910509F058F4A5
:109950008EED94E00E94D13D82EE94E00E94A93AFF
:10996000282F30E014C0C0911905D0911A054D2F51
:1099700050E0EC2FF0E08B019C01BF0182EE94E0FF
:10998000ADD1C80FC0931905D0931A059C01C90128
:10999000DF91CF911F910F91FF90EF900895EF927B
:1099A000FF920F931F93CF93DF938B01CEEDD4E003
:1099B000FBACECAC4E2D50E06F2D70E09C0182EEC4
:1099C00094E0E4D1F80EFBAEECAEDF91CF911F91A5
:1099D0000F91FF90EF900895EF92FF920F931F93D6
:1099E000CF93DF938B01CEEDD4E0FBACECAC4E2DEE
:1099F00050E06F2D70E09C0182EE94E013D2F80EDF
:109A0000FBAEECAEDF91CF911F910F91FF90EF90E5
:109A100008950F931F93CF93DF93CDB7DEB72897A9
:109A20000FB6F894DEBF0FBECDBF8A0123E0660FEC
:109A3000771F2A95E1F7680F791F48E050E0CE01C3
:109A400001960F94DE8B29813A81F8018081918102
:109A50002817390790F08217930760F09C81828164
:109A6000981758F081E090E03B812381231738F06C
:109A700080E005C081E090E002C08FEF9FEF289664
:109A80000FB6F894DEBF0FBECDBFDF91CF911F910F
:109A90000F910895EF92FF920F931F93CF93DF934F
:109AA000EC018B017A018A859B858617970731F037
:109AB000888199810E94F43C1B870A878885998553
:109AC000019689F00E811F81B701888199810E94DA
:109AD000F13C080F111D888599858017910718F4AE
:109AE00081E090E011C06E818A81680F97014C81FE
:109AF000888199810E94053C2E813F81280F311D6C
:109B00003F832E8380E090E0DF91CF911F910F91F2
:109B1000FF90EF9008954F925F926F927F928F9295
:109B20009F92AF92BF92CF92DF92EF92FF920F93EC
:109B30001F93CF93DF93CDB7DEB72D970FB6F89471
:109B4000DEBF0FBECDBF6C012A013B0149015801A8
:109B50001B861C86CE0101967C0188E0F7011192DC
:109B60008A95E9F7DB01CA0127E0B695A795979595
:109B700087952A95D1F79A838983F42FFF77FD87FC
:109B80008F2F80588B838C831A8619864F3F5105FF
:109B90006105710509F018F460E070E026C060917D
:109BA000D3047091D4048E01075F1F4F970149E0E1
:109BB0005DE48091D1049091D2040E943F9297FD80
:109BC000EBCF69857A8583E0660F771F8A95E1F789
:109BD0008091D1049091D204680F791F48E050E041
:109BE000C7010F94DE8B6F8178856115710519F4BB
:109BF0004B86B60106C0C616D70619F08D8580685B
:109C00008B87AE01455F5F4FC401F50119952D9615
:109C10000FB6F894DEBF0FBECDBFDF91CF911F917D
:109C20000F91FF90EF90DF90CF90BF90AF909F90FB
:109C30008F907F906F905F904F9008956F927F927A
:109C40008F929F92AF92BF92CF92DF92EF92FF924C
:109C50000F931F93CF93DF9300D01F92CDB7DEB742
:109C60006C017B013A015901480119821A821B8259
:109C70001C82AE014F5F5F4FB301C7010E949F92EC
:109C80007C0149815A816B817C81411551056105B7
:109C9000710529F084019501C6013DDFE6CF0F90E3
:109CA0000F900F900F90DF91CF911F910F91FF9028
:109CB000EF90DF90CF90BF90AF909F908F907F906C
:109CC0006F90089521E02093D504E1EDF4E09183B5
:109CD00080837383628380E090E008957F92AF92E7
:109CE000BF92CF92DF92EF92FF920F931F93CF9389
:109CF000DF93CDB7DEB72C970FB6F894DEBF0FBE5B
:109D0000CDBF6C01762EF72F842FE52FB901A80166
:109D1000D6011496AD90BC9015979091D5049111F1
:109D20000AC02DE738E1482F672DC6010E943C3C50
:109D300080E090E019C0DA82C9827B82FC838D8347
:109D4000EE8318861F82FA86E9861C861B860AE443
:109D50001DE49E012F5F3F4FC501DDDEB501C60149
:109D60000E94F43C8F8198852C960FB6F894DEBF44
:109D70000FBECDBFDF91CF911F910F91FF90EF905C
:109D8000DF90CF90BF90AF907F900895CF92DF92F9
:109D9000EF92FF920F931F93CF93DF93CDB7DEB770
:109DA0002C970FB6F894DEBF0FBECDBF7C01C90162
:109DB000F701C480D5802091D504211108C02DE57C
:109DC00038E1C7010E943C3C80E090E01CC0FA8270
:109DD000E9826B837C834D835E8318861F821A879A
:109DE00009871C861B860AE41DE49E012F5F3F4FF6
:109DF00049E352E9BC01C60121DFB601C7010E9457
:109E0000F43C8F8198852C960FB6F894DEBF0FBE78
:109E1000CDBFDF91CF911F910F91FF90EF90DF9019
:109E2000CF900895CF92DF92EF92FF920F931F93FE
:109E3000CF93DF93CDB7DEB72C970FB6F894DEBF84
:109E40000FBECDBF7C01C901F701C480D580209130
:109E5000D504211108C02DE338E1C7010E943C3C24
:109E600080E090E01CC0FA82E9826B837C834D83A2
:109E70005E8318861F821A8709871C861B860AE460
:109E80001DE49E012F5F3F4F4CE352E9BC01C60128
:109E9000D5DEB601C7010E94F43C8F8198852C96CF
:109EA0000FB6F894DEBF0FBECDBFDF91CF911F91EB
:109EB0000F91FF90EF90DF90CF900895CF93DF93B5
:109EC000EC01262F4CAD6BAD04960E94E73B2BAD09
:109ED000082E000C990B820F911D8BAF81E090E052
:109EE000DF91CF9108950F939CE0899F802D1124DD
:109EF00021E0280F2093DD04845F8093DC0490E050
:109F000002964091160550E08417950714F480E0FE
:109F100033C0822F90E02091180530E0821793071C
:109F2000B4F76623A9F061E082EE94E00E94C237A4
:109F30004091DD044E5F0BE020E860E082EE94E0AB
:109F40000E94643A60E082EE94E00E94C23705C04D
:109F500061E082EE94E00E94C2376091DC0480915F
:109F600016056817A0F29091DD04809118058917F5
:109F700070F280E0D4DC81E00F910895CF93DF93FD
:109F8000FC0185ADEF012496811105C081E085AF0C
:109F9000CE010E946937CE01DF91CF910C94A0379A
:109FA0006FEF7FEF19CD6FEF7FEFF9CC4FEF5FEFE2
:109FB000C2CC482F50E02091DB04022E000C330B62
:109FC0004217530781F08093DB04813031F468E558
:109FD00071E282EE94E00C94F43C68E679E182EE62
:109FE00094E00C94F43C0895EF92FF920F938AE171
:109FF000E82E8FE1F82E00E428E040E060E082EEF9
:10A0000094E00E94EC376BEB74E082EE94E00E94E7
:10A01000F43C28E433E041E169E382EE94E00E94FD
:10A02000053C6BE27DE082EE94E00E94F43C2FE47C
:10A0300033E04CE16AE382EE94E00E94053C66E87E
:10A0400070E182EE94E00E94F43C2FE533E049E2B7
:10A050006BE382EE94E00E94053C66E870E182EEDC
:10A0600094E00E94F43C2BE633E04EE36DE382EE95
:10A0700094E00E94053C2DE633E04EE362E482EE7C
:10A0800094E00E94053C68E679E182EE94E00F914D
:10A09000FF90EF900C94F43C8EED94E06FDF61E064
:10A0A00080E0A2DF82EE94E00E94A4378111F7CF16
:10A0B00064EC79E080E090E00C9485B2EF92FF923E
:10A0C0000F9385E9E82E8EE1F82E03E127E047E0C3
:10A0D00064E282EE94E00E94EC3783E06ADF2DE6D2
:10A0E00033E04BE265E282EE94E00E94053C27E714
:10A0F00033E047E367E082EE94E00F91FF90EF904A
:10A100000C94053C8EED94E039DFD8DF82EE94E0CC
:10A110000E94A4378111F9CF64EC79E080E090E0EF
:10A120000C9485B2B9DFEECF60E070E088E591E293
:10A13000C9CD1F93CF93DF93D2DBC091E304C695C3
:10A14000C6958EED94E01ADFDC2FDD0F1D2F1C0F5E
:10A1500083E02FDF6C2F80E0E2DB82E797E023DFF4
:10A160006D2F80E0DCDB8AEA98E11ADF612F80E066
:10A17000D6DB8DE998E114DF82EE94E00E94A437EB
:10A180008111E6CFDF91CF911F9108950895CF936C
:10A19000E62F6CE0869F602D112481E0860F80936E
:10A1A000DD04645F6093DC04462F50E04E5F5F4F38
:10A1B0002091160530E0421753070CF445C090E09B
:10A1C0002091180530E0821793070CF03DC0CE2F88
:10A1D0008EE3A5DB65E470E080E090E0E7DE61E31C
:10A1E0006C0F062E000C770B880B990BDFDE60E2FC
:10A1F00070E080E090E0DADE6091BC0D7091BD0D02
:10A200008091BE0D9091BF0D0F947784CB010E9479
:10A2100090B3C9DE6FE270E080E090E0C7DE0E949C
:10A22000A295811109C085E0C89FF0011124E55570
:10A23000F24F8481811108C08091C00D9091C10DB1
:10A240000E9490B3CF91AFCECF910895CF92DF927D
:10A25000EF92FF920F931F93CF93DF931F921F9262
:10A26000CDB7DEB77B01622F49833DDE498188236C
:10A2700009F440C0442309F101151105F1F4C701A7
:10A280000E940F9425E130E0281B310937FF02C0FE
:10A290002F5F3F4F3595279530E82158822F830F48
:10A2A00087FD0CC060E270E080E090E02A83398393
:10A2B0007DDE398131502A81F1CF30E8C32ED12C97
:10A2C000B601C70189DB7601E81AF90A0115110503
:10A2D00011F41E2D06C0FF24B701C80160DB1E2D3E
:10A2E000181B173038F060E270E080E090E05EDE2E
:10A2F000181BF7CF0F900F90DF91CF911F910F9107
:10A30000FF90EF90DF90CF9008950F93CF93DF935E
:10A31000982F862FEA01692FE6DD882309F162E78D
:10A3200070E0CE0159DBC2E7C81BC73038F060E2ED
:10A3300070E080E090E03ADEC81BF7CF6091DC046B
:10A340008AE7EDDA602F000F770B880B990B2EDE72
:10A3500060E270E080E090E0DF91CF910F9126CE37
:10A36000DF91CF910F910895CF92DF92EF92FF92FC
:10A370000F931F93CF93DF93982F862F6A01790154
:10A38000692FB1DD882309F442C0C701002321F001
:10A390000E940F94182F03C00E94EE93182FC3E160
:10A3A000D0E0C11BD1098C2F880FC80FCC0FD0E093
:10A3B000BE01C60111DBC81B6AE370E080E090E0DB
:10A3C000F5DDC73038F060E270E080E090E0EEDD6F
:10A3D000C81BF7CF8AEF189F802D11246091DC04F1
:10A3E00080589DDAC701002349F0DF91CF911F917A
:10A3F0000F91FF90EF90DF90CF90D2CDDF91CF9172
:10A400001F910F91FF90EF90DF90CF90CCCDDF9117
:10A41000CF911F910F91FF90EF90DF90CF90089513
:10A42000BF92CF92DF92EF92FF920F931F93CF9341
:10A43000DF936C017B010E940F94C82FC7010E941B
:10A44000EE93082F10E08C2F90E023E130E0201BEA
:10A45000310BBB24B394281739071CF0B12CC5E28B
:10A4600001C0CFE12C2F30E0A9014E5F5F4F8091FA
:10A47000160590E04817590744F02950310980919A
:10A48000180590E082179307C4F5D0E0E114F104B9
:10A4900009F43AC06AE370E080E090E087DDBB2019
:10A4A00081F0C45F80911605C81770F12C2F30E041
:10A4B000295031098091180590E0821793071CF408
:10A4C00023C0DD2309F124E130E0201B310B822F72
:10A4D000880F820F6C2F880F22DA60E270E080E034
:10A4E00090E064DDC701DF91CF911F910F91FF9044
:10A4F000EF90DF90CF90BF9056CD6C2F80E00FDAB9
:10A50000C6014EDDD1E0C2CFDF91CF911F910F91F7
:10A51000FF90EF90DF90CF90BF900895CF92DF92A1
:10A52000EF92FF920F931F93CF93DF931F92CDB7BC
:10A53000DEB7182F7A01D22ECA0169830E940F94C8
:10A54000082F812F880F810FC82ECC0C1CE0698149
:10A55000169F100D1124DD20C1F061E082EE94E021
:10A560000E94C237202F220F200F220F2E5F0BE0F8
:10A5700047EF410F6FEF6C0D82EE94E00E94643A5A
:10A5800060E082EE94E00E94C237612F8C2DC7D923
:10A59000C70106DDDD2071F061E082EE94E00F90EE
:10A5A000DF91CF911F910F91FF90EF90DF90CF90AF
:10A5B0000C94C2370F90DF91CF911F910F91FF90B4
:10A5C000EF90DF90CF900895AF92BF92DF92EF921D
:10A5D000FF920F931F93CF93DF93EC015B01D42E77
:10A5E000C901B801A7010E94389591E02D2D2927B6
:10A5F000A50164E081E092DFCE010E940F942D2D31
:10A60000AE0164E094E1981B892FDF91CF911F91F7
:10A610000F91FF90EF90DF90BF90AF907FCFEF92C0
:10A62000FF920F93CF93DF93D82FC62F7901682F16
:10A630008C2F59DC8823D9F0002329F062E070E0E8
:10A6400080E090E0B3DC2D2F4C2F64E1C7010E9425
:10A65000879468E770E0A3D9C8E7C81BC73038F013
:10A6600060E270E080E090E0A1DCC81BF7CFDF91F2
:10A67000CF910F91FF90EF9008958F929F92AF929C
:10A68000BF92CF92DF92EF92FF920F936B017C010A
:10A690008090D7049090D804A090D904B090DA04A8
:10A6A000A50194010F940884882301F120E030E093
:10A6B000A901C701B6010F940884882351F0A501B0
:10A6C0009401C701B6010F94088487FD04C081E09E
:10A6D00003C080E001C08FEF8093D604C092D704FE
:10A6E000D092D804E092D904F092DA048091160551
:10A6F000813128F480911805833008F048C080919A
:10A700001605853128F480911805843108F04FC072
:10A71000809116058F3308F057C0809118058F324D
:10A7200008F452C08091D60440E3481B8EEEE82E18
:10A7300088E1F82E0DE022E06AE582EE94E00E94C6
:10A74000EC378091D60441E3481B94EDE92E98E163
:10A75000F92E22E065E082EE94E00E94EC3728E0DA
:10A76000E22E29E1F22E00E123E04FE262E182EEE7
:10A7700094E00E94EC3738E3E32E39E1F32E23E036
:10A780004FE267E682EE94E00E94EC371DC08091B4
:10A79000D60444E0481B59EBE52E58E1F52E0CE0B9
:10A7A00022E062E482EE94E00E94EC37A8CF41ED13
:10A7B000E42E48E1F42E01E023E044E16CE382EE74
:10A7C00094E00E94EC37A4CF0F91FF90EF90DF90C0
:10A7D000CF90BF90AF909F908F900895CF92EF92BF
:10A7E0000F93CF93DF93CEEDD4E01B821A828FE8D4
:10A7F00093E099838883CC24CA94EE24EA9402E5FA
:10A8000022E143E169E172E0CE010E94A33E8BE9BF
:10A8100093E099838883DF91CF910F91EF90CF9050
:10A8200008955A9887FD52C05B9800000000000010
:10A8300000005A9A5A98282F220F86FD53C05B9821
:10A8400000000000000000005A9A5A98922F990FB9
:10A8500026FD46C05B9800000000000000005A9AE8
:10A860005A98892F880F96FD39C05B980000000028
:10A87000000000005A9A5A98982F990F86FD2CC014
:10A880005B9800000000000000005A9A5A98892F37
:10A89000880F96FD1FC05B980000000000000000BC
:10A8A0005A9A5A98982F990F86FD12C05B9800000B
:10A8B0000000000000005A9A5A9896FD15C05B9857
:10A8C00000000000000000005A9A08955B9AADCF86
:10A8D0005B9AEDCF5B9AE0CF5B9AD3CF5B9AC6CF02
:10A8E0005B9AB9CF5B9AACCF5B9AEACF2F923F923B
:10A8F0005F927F929F92AF92BF92CF92DF92EF9240
:10A90000FF920F931F93CF93DF937C011B01942E33
:10A9100069018AE0481709F47BC0A5E14A134EC0DB
:10A92000DB011296ED91FC9113971281C681D781BC
:10A930005D9A88E28A950000E9F700EE010F80E158
:10A94000582E510E98E2792E88EF6BDF872D8A956D
:10A950000000E9F7103208F046C0812F8077806848
:10A9600060DF812F8295807F5CDF872D8A950000D4
:10A97000E9F780E856DF80E054DF872D8A950000F4
:10A98000E9F78AEF4EDF872D8A950000E9F75E012F
:10A99000B0E1AB0EB11C8881807F43DF8991829545
:10A9A000807F3FDFCA15DB05B1F7872D8A95000050
:10A9B000E9F71F5F0F5F1511C7CF5D989601492D0D
:10A9C000B101C701DF91CF911F910F91FF90EF90DF
:10A9D000DF90CF90BF90AF909F907F905F903F901F
:10A9E0002F900C942639802F807780681ADF802F73
:10A9F0008295807F16DF872D8A950000E9F780E831
:10AA000010DF80E80EDF872D8A950000E9F7B9CFC7
:10AA1000559A5D98539A5B98529A5A9A5D9AC8E2F1
:10AA20008C2F8A950000E9F788E790E00E94433870
:10AA300088EFF7DE8C2F8A950000E9F780E2F1DEDF
:10AA400080E0EFDE8C2F8A950000E9F780E0E9DEF8
:10AA500080E8E7DE8C2F8A950000E9F780E0E1DEF0
:10AA600080E1DFDE8C2F8A950000E9F78FE090E02F
:10AA70000E94433880E2D5DE80E4D3DE8C2F8A95B5
:10AA80000000E9F780E2CDDE80E6CBDECA9500006B
:10AA9000E9F710E0D8E208E2812F80778068C1DE14
:10AAA000812F8295807FBDDE8D2F8A950000E9F78A
:10AAB00080E8B7DE80E0B5DE8D2F8A950000E9F7EB
:10AAC0008AEFAFDE8D2F8A950000E9F7C0E280E0C3
:10AAD000A8DE80E0A6DE9D2F9A950000E9F7C15020
:10AAE000B1F788EF9EDE802F8A950000E9F71F5F9F
:10AAF000103209F0D1CF80E094DE80EC92DE88E263
:10AB00008A950000E9F75D9859CF5D9A88E28A95A9
:10AB10000000E9F7089588EF84DE88E28A95000056
:10AB2000E9F708958AEF7DDE88E28A950000E9F76B
:10AB30000895CF93C82F807F74DE8C2F8295807FFD
:10AB400070DE88E28A950000E9F7CF910895CF93EF
:10AB5000DF931F921F92CDB7DEB789839A830E943D
:10AB6000968720E040E060E070E089819A810F9054
:10AB70000F90DF91CF910C949B890F93CF93DF932C
:10AB800061E081E00E94AA8AD0914007C0E0D11123
:10AB900017C080913F07811104C00E94D194811198
:10ABA00065C080912702882309F457C081E0909105
:10ABB0003F07911180E004E024E04CE65AE24BC0EC
:10ABC000D130C1F480913F07813021F40E94D194AB
:10ABD000811154C080912702882309F43EC081E08E
:10ABE00090913F07913009F080E003E02EE343E6C7
:10ABF0005AE231C0D230B9F480913F07823021F45B
:10AC00000E94D194811143C080912702882329F1A9
:10AC100081E090913F07923009F080E003E02EE35D
:10AC20004AE55AE218C0D330C1F480913F0783301F
:10AC300021F40E94D194811133C08091270288238E
:10AC400061F081E090913F07933009F080E003E0EC
:10AC50002EE344E55AE26C2F58DBCF5FDF5FC5304F
:10AC600009F095CF84E080933E0721C00E94C989F6
:10AC700080910C07882309F494CF19C088E99DE7D7
:10AC800066DF80910C07882309F4A4CF10C087EAFF
:10AC900092E85DDF80910C07882309F4B5CF07C0E7
:10ACA00089E696E854DF80910C07882331F2DF9122
:10ACB000CF910F910895CF92DF92EF92FF920F9371
:10ACC0001F938091CE09811103C080E19AE002C0F8
:10ACD0008EEC99E020EBC22E2AE2D22E7C0103EA10
:10ACE0001AE229EC39E842E856E56CE97AE286E9AD
:10ACF0009AE20E94A38B1F910F91FF90EF90DF903B
:10AD0000CF90089580E19AE00E94D89E0E94C28967
:10AD10000C94559A0E9474A321E030E0811102C086
:10AD200020E030E0309367072093660710924007D9
:10AD300081E080930C0783E0809327020895CF92EF
:10AD4000DF92EF92FF920F931F93CF93DF930E94B6
:10AD500072A46C0161E081E00E94AA8AC091400760
:10AD6000D0E081E0C81AD108C11117C080913F0717
:10AD7000811104C00E94D194811195C08091270255
:10AD8000882359F081E090913F07911180E004E021
:10AD900024E041E95AE26D2FB8DA60E17AE087E910
:10ADA00099E00E9466AA8091100A8F3201F1809189
:10ADB0001D0A83FF1CC0C130C1F480913F07813060
:10ADC00021F40E94D194811176C0809127028823BA
:10ADD00061F081E090913F07913009F080E000E25E
:10ADE0002EE34DE85AE26D2F90DA92E001C091E037
:10ADF00080912702882309F44EC0760111E01C0FD0
:10AE00008FEFE816F80609F446C0C9133FC060E0AA
:10AE100070E0C7010E944DA090911D0A80913F07EC
:10AE200094FF1CC08C134EC00E94D194882309F457
:10AE300049C080E19AE00E941EA31092400782E080
:10AE400090E0909367078093660781E080930C07FA
:10AE50001092690783E08093270252C08C1304C0CC
:10AE60000E94D19481113DC080912702882361F016
:10AE700081E090913F079C1380E000E027EC39E1EE
:10AE800041E75AE26D2FCBDB912F01C09F5F81E03C
:10AE9000E81AF108B5CFDF5FCF5FD53009F064CF96
:10AEA00090933E072DC00E94C98980910C0788238A
:10AEB00009F464CF25C02EDF80910C07882309F4A4
:10AEC00084CF1EC0809127028823F1F281E0909107
:10AED0003F079C1380E001E027EC39E14FE75AE29D
:10AEE000D1CF0E94968720E040E060E070E08BE5E3
:10AEF00096E50E949B8980910C07882309F4B4CFC2
:10AF0000DF91CF911F910F91FF90EF90DF90CF9045
:10AF10000895CF93DF93EC01CB01BA010F94AA847B
:10AF20000F947C846883DF91CF910895CF93DF9352
:10AF3000EC01CB01BA010F94AA842FE632E143E879
:10AF40005AE30F944686688379838A839B83DF91D3
:10AF5000CF91089569E877E586EB97E50C94DE8953
:10AF600066E977E583ED97E50C94DE890F94AA8472
:10AF70000F947C84862F0C94C9B2CF93DF9300D0BA
:10AF80001F92CDB7DEB769837A838B839C8360E29F
:10AF9000CE0101960E94CEB50F900F900F900F90AA
:10AFA000DF91CF9108950F94AA842FE632E143E810
:10AFB0005AE30F944686E1CF2F923F924F925F92D1
:10AFC0006F927F928F929F92AF92BF92CF92DF92B9
:10AFD000EF92FF920F931F93CF93DF93CDB7DEB71E
:10AFE00029970FB6F894DEBF0FBECDBF1C0179873D
:10AFF0006887CA01B901E982FA820B831C83DE8269
:10B00000CD82AF8220E030E04AE754E40F944686D8
:10B010006B017C0120E030E040E057EC0F940B86A0
:10B0200018162CF0C12CD12CE12C27ECF22EC701E4
:10B03000B6010F9477842B013C0120E030E04AE711
:10B0400054E469817A818B819C810F9446864B01FF
:10B050005C0120E03EEF4FEF56E40F94088487FD3B
:10B0600007C0812C9EEF992EAA24AA9496E4B92EAB
:10B0700020E030E04AE754E4E885F9856081718199
:10B08000828193810F9446866B017C01C301B201DA
:10B090000F94AA849B01AC01C701B6010F942E83C3
:10B0A0000F947C8469837A838B839C83C501B4016C
:10B0B0000F9477847B018C01E418F50806091709C1
:10B0C000FF81FF938D809E8080EBA82E87E5B82EB0
:10B0D000C980DA80A301920168857985C1010E9447
:10B0E000BD870F9029960FB6F894DEBF0FBECDBF77
:10B0F000DF91CF911F910F91FF90EF90DF90CF9054
:10B10000BF90AF909F908F907F906F905F904F9087
:10B110003F902F9008958F929F92AF92BF92CF92BF
:10B12000DF92EF92FF920F931F93CF93DF9361E033
:10B1300081E00E94AA8AD0914007C0E0D11119C0D5
:10B1400080913F07811104C00E94D1948111C4C035
:10B1500080912702882309F4B6C081E090913F07CF
:10B16000911180E004E024E048EE5AE26C2FCDD843
:10B17000AAC0D130E1F480913F07813021F40E94D0
:10B18000D1948111B1C080912702882309F49BC01A
:10B1900011E080913F07813009F010E08091290D86
:10B1A0000E94C9B200E09C0142ED5AE289C0D2304F
:10B1B00009F580913F07823021F40E94D1948111DA
:10B1C000B4C080912702882309F47DC011E08091EA
:10B1D0003F07823009F010E060912A0D70912B0D2D
:10B1E00080912C0D90912D0DC8DE00E09C014EEC5D
:10B1F0005AE266C0D33009F580913F07833021F4CD
:10B200000E94D1948111AAC080912702882309F459
:10B210005AC011E080913F07833009F010E060913F
:10B220002E0D70912F0D8091300D9091310DA5DE76
:10B2300000E09C014AEC5AE243C0D43001F5809111
:10B240003F07843021F40E94D1948111A0C08091E5
:10B2500027028823C1F111E080913F07843009F073
:10B2600010E06091320D7091330D8091340D90910A
:10B27000350D83DE00E09C0146EC5AE221C0D5305A
:10B2800011F580913F07853021F40E94D1948111FE
:10B2900097C0809127028823B1F011E080913F0789
:10B2A000853009F010E060912B0270912C028091A2
:10B2B0002D0290912E0261DE00E09C0142EB5AE2E9
:10B2C0006C2F812F51D8CF5FDF5FC53009F036CFAB
:10B2D00086E080933E078CC00E94C98980910C074C
:10B2E000882309F435CF84C081E00E94C694C090C1
:10B2F000290DD12C1F92812C912C4AEAA42E47E5CE
:10B30000B42EE12CF12C8701EA9420E030E0A90171
:10B3100069E27DE08DED9AE20E94BD870F908091F9
:10B320000C07882309F42FCF63C081E00E94C694E4
:10B33000A12CC12CD12C16E6E12EFE2C0EE111E43D
:10B3400020E030E0A9016AE27DE080ED9AE234DE9F
:10B3500080910C07882309F434CF4AC081E00E9411
:10B36000C694A12CC12CD12C16E6E12EFE2C0EE1A8
:10B3700011E420E030E0A9016EE27DE08CEC9AE27D
:10B380001BDE80910C07882309F43ECF31C081E099
:10B390000E94C694A12CC12CD12C16E6E12EFE2CC5
:10B3A0000EE111E420E030E0A90162E37DE088ECE9
:10B3B0009AE202DE80910C07882309F448CF18C076
:10B3C00081E00E94C694A12CC12CD12C16E6E12E5E
:10B3D000FE2C0EE111E420E030E0A9016BE272E006
:10B3E0008CEB9AE2E9DD80910C07882309F451CFB8
:10B3F000DF91CF911F910F91FF90EF90DF90CF9051
:10B40000BF90AF909F908F900895CF93DF93EC0102
:10B41000CB01BA010F94AA842AE037ED43E25CE342
:10B420000F944686688379838A839B83DF91CF91CB
:10B430000895CF93DF93EC01CB01BA010F94AA8456
:10B44000688379838A839B83DF91CF910895CF931B
:10B45000DF93EC01CB01BA010F94AA8420E030E025
:10B4600048EC51E40F944686688379838A839B83F2
:10B47000DF91CF910895CF93DF93EC01CB01BA0117
:10B480000F94AA8420E030E048EC52E40F94468602
:10B49000688379838A839B83DF91CF910895CF93CB
:10B4A000DF93EC01CB01BA010F94AA8420E030E0D5
:10B4B00048EC51E40F9446860F947C84688379832A
:10B4C0008A839B83DF91CF910895CF93DF93EC0123
:10B4D000CB01BA010F94AA8420E030E048EC52E49A
:10B4E0000F9446860F947C84688379838A839B8338
:10B4F000DF91CF910895CF93DF93EC01CB01BA0197
:10B500000F94AA842AE037ED43E25CE30F94468669
:10B51000688379838A839B83DF91CF910895CF934A
:10B52000DF93EC01CB01BA010F94AA842DEC3CEC23
:10B530004CEC5DE30F944686688379838A839B8312
:10B54000DF91CF91089565E07AE584EF9AE50C9458
:10B55000DE8969E17AE58CEA9BE50C94DE896BE390
:10B560007AE58EE29BE50C94DE8967E27AE581E17B
:10B570009BE50C94DE896FE47AE58FEE9EE50C94F2
:10B58000DE8965E67AE588E69BE50C94DE896BE763
:10B590007AE58BE49BE50C94DE896FE87AE587ED2C
:10B5A0009AE50C94DE890D9449360D949036CF932C
:10B5B000DF9300D01F92CDB7DEB70F94AA842DEC95
:10B5C0003CEC4CEC5DE30F94468669837A838B8375
:10B5D0009C83CE0101960E9470B80F900F900F903F
:10B5E0000F90DF91CF910895CF93DF9300D01F92FA
:10B5F000CDB7DEB70F94AA842AE037ED43E25CE3CF
:10B600000F94468669837A838B839C83CE0101964F
:10B610000E9490B40F900F900F900F90DF91CF91F8
:10B620000895CF93DF9300D01F92CDB7DEB70F946C
:10B63000AA8420E030E048EC51E40F944686698308
:10B640007A838B839C83CE0101960E9417B70F905B
:10B650000F900F900F90DF91CF910895CF93DF93CC
:10B6600000D01F92CDB7DEB70F94AA8420E030E05F
:10B6700048EC52E40F94468669837A838B839C83DB
:10B68000CE0101960E9417B70F900F900F900F9068
:10B69000DF91CF910895CF93DF9300D01F92CDB764
:10B6A000DEB70F94AA842AE037ED43E25CE30F94FF
:10B6B000468669837A838B839C83CE0101960E94A0
:10B6C000CFB70F900F900F900F90DF91CF9108950B
:10B6D000CF93DF9300D01F92CDB7DEB70F94AA842B
:10B6E00020E030E048EC52E40F9446860F947C84CE
:10B6F0000F94A88469837A838B839C83CE010196FF
:10B700000E9417B70F900F900F900F90DF91CF917D
:10B710000895CF92DF92EF92FF926B017C0120E0BF
:10B7200030E0A9010F94088487FD05C020E030E0D7
:10B7300040E05FE304C020E030E040E05FEBC701A1
:10B74000B6010F942F830F947784CB01FF90EF9075
:10B75000DF90CF900C9490B30F94AA84DACFCF935C
:10B76000DF9300D01F92CDB7DEB70F947C840F9487
:10B77000A88469837A838B839C83CE0101960E947F
:10B7800017B70F900F900F900F90DF91CF91089502
:10B790006F927F928F929F92AF92BF92CF92DF92E1
:10B7A000EF92FF920F931F93CF93DF9300D01F92DE
:10B7B000CDB7DEB761E081E00E94AA8A60904007C1
:10B7C000712C61101AC080913F07811104C00E9442
:10B7D000D194811159C180912702882309F44BC16A
:10B7E00081E090913F07911180E004E024E04BE577
:10B7F0005CE2672D0E9485513EC181E068122CC039
:10B8000080913F07813021F40E94D194811144C17D
:10B8100080912702882309F42EC111E080913F070F
:10B82000813009F010E080915A1090915B10A09146
:10B830005C10B0915D1089839A83AB83BC83CE0189
:10B8400001960E9417B700E09C014FE45CE2672D6F
:10B85000812F0E94B4510FC182E068122CC08091E8
:10B860003F07823021F40E94D19481114DC1809113
:10B870002702882309F4FFC011E080913F0782303E
:10B8800009F010E080915E1090915F10A09160101F
:10B89000B091611089839A83AB83BC83CE010196FA
:10B8A0000E9417B700E09C014BE35CE2672D812FFB
:10B8B0000E94B451E0C083E068122CC080913F0721
:10B8C000833021F40E94D194811156C180912702C6
:10B8D000882309F4D0C011E080913F07833009F03C
:10B8E00010E08091621090916310A0916410B0916B
:10B8F000651089839A83AB83BC83CE0101960E9435
:10B9000017B700E09C0149E25CE2672D812F0E949D
:10B91000B451B1C084E0681227C080913F078430E1
:10B9200021F40E94D19481115FC180912702882364
:10B9300009F4A1C011E080913F07843009F010E0C4
:10B9400060912610709127108091281090912910F5
:10B950000F94A88404DF00E09C014BE15CE2672DBA
:10B96000812F0E94B45187C085E0681227C0809162
:10B970003F07853021F40E94D194811171C18091DB
:10B980002702882309F477C011E080913F078530B2
:10B9900009F010E060912A1070912B1080912C100A
:10B9A00090912D100F94A884DADE00E09C014DE008
:10B9B0005CE2672D812F0E94B4515DC086E0681261
:10B9C00027C080913F07863021F40E94D1948111D5
:10B9D00083C180912702882309F44DC011E0809132
:10B9E0003F07863009F010E060912E1070912F1003
:10B9F00080913010909131100F94A884B0DE00E057
:10BA00009C014FEF5BE2672D812F0E94B45133C040
:10BA100087E0681230C080913F07873021F40E9490
:10BA2000D19481118EC180912702882321F111E0E8
:10BA300080913F07873009F010E0609132107091DB
:10BA4000331080913410909135100F94A8840F9486
:10BA50007C840F94A88469837A838B839C83CE0132
:10BA600001960E9417B700E09C0141EF5BE2672D51
:10BA7000812F0E94B4517394639485E07812A1CE13
:10BA800088E080933E0798C10E94C98980910C0785
:10BA9000882309F4A0CE90C181E00E94C6942AE0D8
:10BAA00037ED43E25DE360915A1070915B10809135
:10BAB0005C1090915D100F94468620E030E040E8E5
:10BAC0005FE30F942E830F947C841F92812C912C22
:10BAD00055EBA52E5AE5B52E6B0117E7E12E1FE0B9
:10BAE000F12E00E010E021E030E040E050E06AE5B7
:10BAF00070E185E59CE20E94BD870F9080910C0764
:10BB0000882309F485CE58C181E00E94C6942AE0BA
:10BB100037ED43E25CE360915E1070915F108091BD
:10BB20006010909161100F94468620E030E040E86C
:10BB30005FE30F942E830F947C841F92812C912CB1
:10BB40003FEAA32E3AE5B32E6B011DEDE12E13E083
:10BB5000F12E00E010E021E030E040E050E06EE542
:10BB600070E185E49CE20E94BD870F9080910C07F4
:10BB7000882309F47CCE20C181E00E94C6942AE08B
:10BB800037ED43E25DE36091621070916310809144
:10BB90006410909165100F94468620E030E040E8F4
:10BBA0005FE30F942E830F947C841F92812C912C41
:10BBB00095EBA92E9AE5B92E6B0117E7E12E1FE050
:10BBC000F12E00E010E021E030E040E050E062E6DD
:10BBD00070E182E39CE20E94BD870F9080910C0788
:10BBE000882309F473CEE8C081E00E94C694609176
:10BBF00026107091271080912810909129100F9491
:10BC0000A8842AE037ED43E25DE30F94468620E006
:10BC100030E040E850E40F942E830F947C841F9210
:10BC2000B3ED8B2EBAE59B2E1BEBA12E1AE5B12EA0
:10BC30006B0114E7E12E1FE0F12E00E010E024E09C
:10BC400030E040E050E066E270E182E29CE20E9477
:10BC5000BD870F9080910C07882309F466CEACC095
:10BC600081E00E94C69460912A1070912B108091FF
:10BC70002C1090912D100F94A8842AE037ED43E208
:10BC80005DE30F94468620E030E040E850E40F94F6
:10BC90002E830F947C841F92E3ED8E2EEAE59E2E78
:10BCA000FBEBAF2EFAE5BF2E6B0114E7E12E1FE090
:10BCB000F12E00E010E024E030E040E050E06AE2E5
:10BCC00070E184E19CE20E94BD870F9080910C0797
:10BCD000882309F454CE70C081E00E94C69460911C
:10BCE0002E1070912F1080913010909131100F9480
:10BCF000A8842AE037ED43E25DE30F9446860F9473
:10BD00007C841F9233ED832E3AE5932E4BEBA42EC9
:10BD10004AE5B42E6B0118E7E12E1FE0F12E00E09A
:10BD200010E020E030E0A9016EE270E186E09CE2E4
:10BD30000E94BD870F9080910C07882309F449CE9B
:10BD40003BC081E00E94C694609132107091331024
:10BD500080913410909135100F94A8842AE037ED2B
:10BD600043E25CE30F94468620E030E040E85FE386
:10BD70000F942E830F947C841F9283ED882E8AE586
:10BD8000982E91ECA92E9AE5B92E6B011DEDE12EAE
:10BD900013E0F12E00E010E021E030E040E050E060
:10BDA00062E370E188EF9BE20E94BD870F90809173
:10BDB0000C07882309F437CE0F900F900F900F9047
:10BDC000DF91CF911F910F91FF90EF90DF90CF9077
:10BDD000BF90AF909F908F907F906F9008950F9439
:10BDE000AA8420E030E048EC51E40F944686B7CCBA
:10BDF0000F931F93CF93DF9361E081E00E94AA8AA3
:10BE0000C0914007D0E0C1111AC080913F07811155
:10BE100004C00E94D1948111E8C080912702882338
:10BE200009F461C081E090913F07911180E004E046
:10BE300024E04FE25BE26D2F0E94855154C0C13077
:10BE4000D9F480913F07813021F40E94D19481116F
:10BE5000D4C080912702882309F445C081E09091E5
:10BE60003F07913009F080E003E02EE346E25BE219
:10BE70006D2F0E94855137C0C230D1F480913F07A9
:10BE8000823021F40E94D1948111C1C08091270297
:10BE9000882349F181E090913F07923009F080E0DA
:10BEA00003E02EE349E15BE26D2F0E9485511BC048
:10BEB000C330C9F480913F07833021F40E94D194AC
:10BEC0008111AFC080912702882369F081E09091B1
:10BED0003F07933009F080E003E02EE344E15BE2AA
:10BEE0006D2F0E9485510E94848981111DC0C4302C
:10BEF000E9F480913F07843021F40E94D1948111AC
:10BF00009AC080912702882309F49FC081E0909114
:10BF10003F07943009F080E003E02EE34BE05BE262
:10BF20006D2F0E94855191C014E001C015E0C1132E
:10BF30001BC080913F078C1304C00E94D1948111D3
:10BF400086C080912702882371F081E090913F079D
:10BF50009C1380E003E02EE342E05BE26D2F0E9441
:10BF600085511C2F01C01C2F81E0810FC81318C000
:10BF700080913F078C1304C00E94D194811171C03D
:10BF800080912702882361F081E090913F079C1304
:10BF900080E003E02EE346EF5AE26D2F0E948551C8
:10BFA00082E0810FC81318C080913F078C1304C032
:10BFB0000E94D19481115FC080912702882361F093
:10BFC00081E090913F079C1380E003E02EE34DEE6B
:10BFD0005AE26D2F0E948551DF5FCF5FD53009F0A7
:10BFE00012CF1D5F10933E074FC00E94C9898091F8
:10BFF0000C07882309F411CF47C087E092E60E941E
:10C00000A75580910C07882309F423CF3DC088EC05
:10C010009BE50E94A75580910C07882309F436CF31
:10C0200033C08FEC93E60E94A75580910C078823BC
:10C0300009F448CF29C083E096E60E94A755809175
:10C040000C07882309F45DCF1FC015E08DCF8BE866
:10C0500098E50E94A75580910C07882309F471CFB9
:10C0600013C083E89FE80E94A75580910C0788239E
:10C0700009F486CF09C084ED90E60E94A75580910F
:10C080000C07882309F498CFDF91CF911F910F916E
:10C0900008952F923F924F925F926F927F928F926C
:10C0A0009F92AF92BF92CF92DF92EF92FF920F9347
:10C0B0001F93CF93DF9300D000D0CDB7DEB71C0124
:10C0C0007E836D8329013A01460120E030E040E0A3
:10C0D00057ECB201C3010F940B8618162CF0412CBB
:10C0E000512C612C27EC01C0272DB201862D922FF7
:10C0F0000F9477842B013C0120E03EEF4FEF56E494
:10C10000B701C8010F94088487FD06C0B12C9EEFCB
:10C11000F92E0FEF16E401C0BE2CC301B2010F943B
:10C12000AA849B01AC01ED81FE81608171818281D5
:10C1300093810F942E830F947C8469837A838B83FD
:10C140009C836B2D7F2DC8010F9477847B018C011C
:10C15000E418F50806091709AF9289EAA82E8AE5BE
:10C16000B82EC980DA80A30192016D817E81C10160
:10C170000E94BD870F9026960FB6F894DEBF0FBEC3
:10C18000CDBFDF91CF911F910F91FF90EF90DF9086
:10C19000CF90BF90AF909F908F907F906F905F9067
:10C1A0004F903F902F9008956F927F928F929F9221
:10C1B000AF92BF92CF92DF92EF92FF920F931F93B5
:10C1C000CF93DF9300D01F92CDB7DEB761E081E05F
:10C1D0000E94AA8A60904007712C61101AC0809159
:10C1E0003F07811104C00E94D194811198C08091B1
:10C1F0002702882309F48AC081E090913F079111BA
:10C2000080E004E024E04DE05DE2672D0E9485516E
:10C210007DC081E068122CC080913F07813021F4FD
:10C220000E94D194811183C080912702882309F450
:10C230006DC011E080913F07813009F010E08091DE
:10C24000980F9091990FA0919A0FB0919B0F8983AD
:10C250009A83AB83BC83CE0101960E9490B400E028
:10C260009C0149EF5CE2672D812F0E94B4514EC0C2
:10C2700082E0681225C080913F07823021F40E943D
:10C28000D194811182C080912702882309F43EC095
:10C2900011E080913F07823009F010E06091F30CCB
:10C2A0007091F40C8091F50C9091F60C32DA00E06C
:10C2B0009C0145EE5CE2672D812F0E94B45126C09F
:10C2C00083E0681223C080913F07833021F40E94ED
:10C2D000D194811172C0809127028823B9F011E0B6
:10C2E00080913F07833009F010E06091F70C709166
:10C2F000F80C8091F90C9091FA0C0BDA00E09C019B
:10C3000045ED5CE2672D812F0E94B45173946394D4
:10C3100085E0781262CF84E080933E0765C00E947A
:10C32000C98980910C07882309F461CF5DC020E0A2
:10C3300030E048EC52E46091980F7091990F809131
:10C340009A0F90919B0F0F9446860F947C841F92B6
:10C35000812C912C23EAA22E2AE5B22E6B01EE2429
:10C36000EA941FE7F12E00E010E020E030E0A901A0
:10C3700068E97FE083E09DE20E94BD870F90809195
:10C380000C07882309F450CF2FC081E00E94C69487
:10C39000A12CC12CD12CE12CF12C08E413E420E0D9
:10C3A00030E0A90163EF7CE08FEE9CE272DE8091C9
:10C3B0000C07882309F467CF17C081E00E94C69458
:10C3C000A12CC12CD12CE12CF12C08E413E420E0A9
:10C3D00030E0A90167EF7CE08DED9CE25ADE8091B0
:10C3E0000C07882309F477CF0F900F900F900F90D0
:10C3F000DF91CF911F910F91FF90EF90DF90CF9041
:10C40000BF90AF909F908F907F906F900895AF9264
:10C41000CF92DF92EF92FF920F931F93CF93DF9310
:10C4200061E081E00E94AA8AD0914007C0E0D1116A
:10C430001AC080913F07811104C00E94D1948111DC
:10C4400003C180912702882309F4F5C081E090910F
:10C450003F07911180E004E024E043EC5CE26C2FA4
:10C460000E948551E8C0D13029F580913F07813085
:10C4700021F40E94D1948111EFC08091270288237A
:10C4800009F4D9C011E080913F07813009F010E034
:10C4900060914A1070914B1080914C1090914D100A
:10C4A00038D900E09C0145EB5CE26C2F812F0E94A3
:10C4B000B451C1C0D23029F580913F07823021F4B8
:10C4C0000E94D1948111E2C080912702882309F44F
:10C4D000B2C011E080913F07823009F010E0609116
:10C4E0004E1070914F10809150109091511011D9B1
:10C4F00000E09C0147EA5CE26C2F812F0E94B4515E
:10C500009AC0D33029F580913F07833021F40E94EF
:10C51000D1948111D5C080912702882309F48BC062
:10C5200011E080913F07833009F010E060915210D4
:10C53000709153108091541090915510EAD800E0FA
:10C540009C0149E95CE26C2F812F0E94B45173C0B9
:10C55000D43029F580913F07843021F40E94D19492
:10C560008111C8C080912702882309F464C011E0BA
:10C5700080913F07843009F010E06091561070916F
:10C5800057108091581090915910C3D800E09C0129
:10C590004BE85CE26C2F812F0E94B4514CC0D53027
:10C5A00029F580913F07853021F40E94D1948111B3
:10C5B000BBC080912702882309F43DC011E080911F
:10C5C0003F07853009F010E06091661070916710A8
:10C5D00080916810909169109CD800E09C0141E81E
:10C5E0005CE26C2F812F0E94B45125C0D63019F522
:10C5F00080913F07863021F40E94D1948111ADC013
:10C60000809127028823B9F011E080913F0786309E
:10C6100009F010E060916A1070916B1080916C10BD
:10C6200090916D1076D800E09C014DE65CE26C2F95
:10C63000812F0E94B451CF5FDF5FC53009F0F7CE84
:10C6400087E080933E07A1C00E94C98980910C07B2
:10C65000882309F4F6CE99C081E00E94C694A12CEB
:10C66000C12CD12CE12C10ECF12E09E714E420E0D0
:10C6700030E040E85FE36AE470E18CEB9CE209DDC6
:10C6800080910C07882309F4F8CE7FC081E00E94D6
:10C69000C694A12CC12CD12CE12C10ECF12E09E771
:10C6A00014E420E030E040E85FE36EE470E18EEAFD
:10C6B0009CE2EFDC80910C07882309F405CF65C06C
:10C6C00081E00E94C694A12CC12CD12CE12C10EC4D
:10C6D000F12E09E714E420E030E040E85FE362E592
:10C6E00070E180EA9CE2D5DC80910C07882309F494
:10C6F00012CF4BC081E00E94C694A12CC12CD12C3A
:10C70000E12C10ECF12E09E714E420E030E040E8E1
:10C710005FE366E570E182E99CE2BBDC80910C0797
:10C72000882309F41FCF31C081E00E94C694A12C58
:10C73000C12CD12CE12C10ECF12E09E714E420E0FF
:10C7400030E0A90166E670E186E89CE2A2DC809117
:10C750000C07882309F42DCF18C081E00E94C694ED
:10C76000A12CC12CD12CE12C10ECF12E09E714E402
:10C7700020E030E0A9016AE670E187E79CE289DC0D
:10C7800080910C07882309F43BCFDF91CF911F9153
:10C790000F91FF90EF90DF90CF90AF9008956F9240
:10C7A0007F928F929F92AF92BF92CF92DF92EF9241
:10C7B000FF920F931F93CF93DF9300D01F92CDB7BB
:10C7C000DEB761E081E00E94AA8A60904007712C88
:10C7D00061101AC080913F07811104C00E94D1945A
:10C7E0008111C2C080912702882309F4B5C081E07D
:10C7F00090913F07911180E004E024E04FED5BE26F
:10C80000672D0E948551A8C081E0681226C08091E2
:10C810003F07813021F40E94D1948111ADC08091F5
:10C820002702882309F498C011E080913F078130E6
:10C8300009F010E06091F60F7091F70F8091F80FFA
:10C840009091F90F0E94895B00E09C014FEC5BE244
:10C85000672D812F0E94B4517FC082E0681226C0EC
:10C8600080913F07823021F40E94D19481119EC0B3
:10C8700080912702882309F46FC011E080913F075F
:10C88000823009F010E06091FA0F7091FB0F8091F7
:10C89000FC0F9091FD0F0E94895B00E09C014FEB23
:10C8A0005BE2672D812F0E94B45156C083E068126D
:10C8B0002CC080913F07833021F40E94D1948111D4
:10C8C0008FC080912702882309F446C011E080912F
:10C8D0003F07833009F010E08091FE0F9091FF0F29
:10C8E000A0910010B091011089839A83AB83BC831F
:10C8F000CE0101960E94CFB700E09C014FEA5BE2B7
:10C90000672D812F0E94B45127C084E0681224C093
:10C9100080913F07843021F40E94D194811198C006
:10C92000809127028823C1F011E080913F07843075
:10C9300009F010E0609102107091031080910410D2
:10C94000909105100E94895B00E09C014FE95BE239
:10C95000672D812F0E94B4517394639485E07812FF
:10C9600037CF70923E078DC00E94C98980910C0715
:10C97000882309F437CF85C081E00E94C694A12C9A
:10C98000C12CD12CE12C10E8F12E07E714E420E0B3
:10C9900030E040E85FE366EF7FE087ED9BE279DB24
:10C9A00080910C07882309F43ACF6BC081E00E9484
:10C9B000C694A12CC12CD12CE12C10E8F12E07E754
:10C9C00014E420E030E040E85FE36AEF7FE087ECCA
:10C9D0009BE25FDB80910C07882309F449CF51C0AB
:10C9E00081E00E94C69420E030E048EC52E460917F
:10C9F000FE0F7091FF0F80910010909101100F9425
:10CA0000468620E030E040E251E40F942E830F94FC
:10CA10007C841F92812C912C97ECA92E9AE5B92E3B
:10CA20006B0115EFE12E1FE7F12E00E010E02AE088
:10CA300030E040E050E06EEF7FE087EB9BE20E9449
:10CA4000BD870F9080910C07882309F43ACF19C055
:10CA500081E00E94C694A12CC12CD12CE12C10E8BD
:10CA6000F12E07E714E420E030E040E85FE362E005
:10CA700070E187EA9BE20DDB80910C07882309F4C3
:10CA80004FCF0F900F900F900F90DF91CF911F918C
:10CA90000F91FF90EF90DF90CF90BF90AF909F905D
:10CAA0008F907F906F9008952F923F924F925F9258
:10CAB0006F927F928F929F92AF92BF92CF92DF92AE
:10CAC000EF92FF920F931F93CF93DF93CDB7DEB713
:10CAD00029970FB6F894DEBF0FBECDBF1C01798732
:10CAE0006887CA01B901E982FA820B831C83DE825E
:10CAF000CD82AF8220E030E040E251E40F944686E0
:10CB00006B017C0120E030E040E057EC0F940B8695
:10CB100018162CF0C12CD12CE12C27ECF22EC701D9
:10CB2000B6010F9477842B013C0120E030E040E215
:10CB300051E469817A818B819C810F9446864B01F7
:10CB40005C0120E03EEF4FEF56E40F94088487FD30
:10CB500007C0812C9EEF992EAA24AA9496E4B92EA0
:10CB600020E030E040E251E4E885F98560817181A0
:10CB7000828193810F9446866B017C01C301B201CF
:10CB80000F94AA849B01AC01C701B6010F942E83B8
:10CB90000F947C8469837A838B839C83C501B40161
:10CBA0000F9477847B018C01E418F50806091709B6
:10CBB000FF81FF938D809E808DECA82E8AE5B82E94
:10CBC000C980DA80A301920168857985C1010E943C
:10CBD000BD870F9029960FB6F894DEBF0FBECDBF6C
:10CBE000DF91CF911F910F91FF90EF90DF90CF9049
:10CBF000BF90AF909F908F907F906F905F904F907D
:10CC00003F902F9008959F92AF92BF92CF92DF9264
:10CC1000EF92FF920F931F93CF93DF9300D01F9259
:10CC2000CDB7DEB761E081E00E94AA8A909040070C
:10CC3000B12C91101AC080913F07811104C00E944D
:10CC4000D1948111D4C080912702882309F4C7C0F0
:10CC500081E090913F07911180E004E024E04DE8ED
:10CC60005BE26B2D0E948551BAC081E098122CC006
:10CC700080913F07813021F40E94D1948111BFC07F
:10CC800080912702882309F4AAC011E080913F0710
:10CC9000813009F010E080913A1090913B10A09102
:10CCA0003C10B0913D1089839A83AB83BC83CE0145
:10CCB00001960E9470B800E09C0149E75BE26B2D91
:10CCC000812F0E94B4518BC082E098122CC08091B9
:10CCD0003F07823021F40E94D1948111ACC0809131
:10CCE0002702882309F47BC011E080913F0782303E
:10CCF00009F010E080913E1090913F10A0914010FB
:10CD0000B091411089839A83AB83BC83CE01019695
:10CD10000E9470B800E09C0145E65BE26B2D812F1C
:10CD20000E94B4515CC083E098122CC080913F07F0
:10CD3000833021F40E94D194811199C080912702FF
:10CD4000882309F44CC011E080913F07833009F03B
:10CD500010E08091421090914310A0914410B09146
:10CD6000451089839A83AB83BC83CE0101960E94D0
:10CD700070B800E09C0141E55BE26B2D812F0E94C1
:10CD8000B4512DC084E098122AC080913F078430AE
:10CD900021F40E94D194811186C0809127028823BA
:10CDA000F1F011E080913F07843009F010E08091AC
:10CDB000461090914710A0914810B0914910898376
:10CDC0009A83AB83BC83CE0101960E9470B800E0C9
:10CDD0009C014DE35BE26B2D812F0E94B451B39413
:10CDE000939485E0B81225CFB0923E0777C00E9499
:10CDF000C98980910C07882309F425CF6FC081E091
:10CE00000E94C694A12C65EDC62E6AE5D62EE12CB3
:10CE10001CE3F12E0CE116E420E030E040EA50E49F
:10CE20006AE370E183E89BE23FDE80910C07882390
:10CE300009F426CF53C081E00E94C694A12C45ED91
:10CE4000C42E4AE5D42EE12C1CE3F12E0CE116E4AD
:10CE500020E030E040EA50E46EE370E18FE69BE2D0
:10CE600023DE80910C07882309F439CF37C081E095
:10CE70000E94C694A12C25EDC22E2AE5D22EE12CCB
:10CE80001CE3F12E0CE116E420E030E040EA50E42F
:10CE900062E470E18BE59BE207DE80910C0788235A
:10CEA00009F44CCF1BC081E00E94C694A12C85EDF3
:10CEB000C82E8AE5D82EE12C1CE3F12E0CE116E4F5
:10CEC00020E030E040EA50E466E470E187E49BE271
:10CED000EBDD80910C07882309F45FCF0F900F9052
:10CEE0000F900F90DF91CF911F910F91FF90EF90D6
:10CEF000DF90CF90BF90AF909F9008950F93CF9306
:10CF0000DF9361E081E00E94AA8AC0914007D0E0EF
:10CF1000C11118C080913F07811104C00E94D194B3
:10CF20008111B5C080912702882361F081E0909142
:10CF30003F07911180E004E024E043E45FE26D2FBD
:10CF40000E94855180917B0F8770873009F058C00F
:10CF5000C130D9F480913F07813021F40E94D194EF
:10CF600081119DC080912702882309F4C0C081E00F
:10CF700090913F07913009F080E003E02EE34CE30D
:10CF80005FE26D2F0E948551B2C0C230D9F480910A
:10CF90003F07823021F40E94D19481118AC0809190
:10CFA0002702882309F4A3C081E090913F079230C3
:10CFB00009F080E003E02EE345E35FE26D2F0E947D
:10CFC000855195C0C330D1F580913F07833021F45E
:10CFD0000E94D194811177C080912702882309F49F
:10CFE00086C081E090913F07933009F080E003E034
:10CFF0002EE34EE25FE26D2F0E94855184E03EC039
:10D00000C130F1F480913F07813021F40E94D19426
:10D01000811163C080912702882309F46AC081E0EE
:10D0200090913F07913009F080E000E22EE340E26A
:10D030005FE26D2F0E94855182E020C084E001C034
:10D0400082E0C8131BC080913F078C1304C00E946C
:10D05000D194811150C080912702882371F081E022
:10D0600090913F079C1380E003E02EE346E15FE2EE
:10D070006D2F0E9485518C2F01C08C2FDF5FCF5FF9
:10D08000D53009F045CF8F5F80933E073DC00E94A9
:10D09000C98980910C07882309F444CF35C085E104
:10D0A0009CE60E94A75580910C07882309F45ACF6B
:10D0B0002BC08AE19CE60E94A75580910C0788232B
:10D0C00009F46DCF21C08FE19CE60E94A7558091A5
:10D0D0000C07882309F480CF17C08AE29FE20E94E0
:10D0E000BB8780910C07882309F494CF0DC084E09E
:10D0F000C5CF82E0C3CF84E29CE60E94A755809111
:10D100000C07882309F4A7CFDF91CF910F910895E1
:10D11000CF92DF92EF92FF92CF93C82F0E94A93255
:10D120006B017C0124EA30E74DE75FE3609157072C
:10D13000709158078091590790915A070F9408846D
:10D1400087FD05C04AEF50E060E070E003C040E0BA
:10D1500050E0BA01C40ED51EE61EF71EC09253075A
:10D16000D0925407E0925507F0925607C0932802D8
:10D17000CF91FF90EF90DF90CF9008952F923F9244
:10D180004F925F926F927F928F929F92AF92BF92D7
:10D19000CF92DF92EF92FF921F93CF93DF93CDB7A1
:10D1A000DEB728970FB6F894DEBF0FBECDBF1C01C7
:10D1B000162F0E94D194882329F010926E070E94A6
:10D1C000C989DAC020916607309167073E832D83B5
:10D1D000232B09F49DC0E4E01E9FC0011124988711
:10D1E0008F83FC01E059FD4F80809180A280B38045
:10D1F00020E030E04AE754E4C501B4010F942E83E7
:10D200002B013C0120E030E04AE754E4C501B401C1
:10D210000F942F836B017C01809165028823B9F103
:10D22000113029F198F0123091F540905D02509044
:10D230005E0260905F0270906002C0906102D090C8
:10D240006202E0906302F090640221C040904D02BF
:10D2500050904E0260904F0270905002C090510268
:10D26000D0905202E0905302F090540210C04090CF
:10D270005502509056026090570270905802C0902C
:10D280005902D0905A02E0905B02F0905C022D812E
:10D290003E81B901330F880B990B0F94AA8420911A
:10D2A0005707309158074091590750915A070F94EA
:10D2B00046869B01AC01C501B4010F942F83EF8119
:10D2C000F885E059FD4F5F0160837183828393830A
:10D2D0002D813E8137FF0CC0A30192010F94088479
:10D2E00087FF11C0F50140825182628273820BC0B8
:10D2F000A70196010F940B8618162CF4F501C08235
:10D30000D182E282F382812F03DF81E080932702C2
:10D31000109267071092660780912702882361F1B7
:10D3200024E0129FF0011124E059FD4F808191818A
:10D33000A281B38189839A83AB83BC832DEC3CECBF
:10D340004CEC5DE360915707709158078091590745
:10D3500090915A070F940B8687FD05C0CE01019668
:10D360000E9456B505C060E2CE0101960E94CEB57E
:10D37000BC01C1010E94105228960FB6F894DEBF7E
:10D380000FBECDBFDF91CF911F91FF90EF90DF9047
:10D39000CF90BF90AF909F908F907F906F905F9055
:10D3A0004F903F902F90089560E08BEB9FE2E6CE88
:10D3B00061E084EB9FE2E2CE62E08DEA9FE2DECEA6
:10D3C000CF93DF9300D01F92CDB7DEB70E94D194E8
:10D3D000882329F010926E070E94C98957C0609176
:10D3E0006607709167076115710569F1072E000CDA
:10D3F000880B990B0F94AA842091570730915807F6
:10D400004091590750915A070F9446869B01AC01F1
:10D4100060917C0270917D0280917E0290917F02EA
:10D420000F942F8360937C0270937D0280937E0221
:10D4300090937F0283E06CDE81E08093270210925C
:10D44000670710926607809127028823F9F02091E0
:10D450001E0630911F0640912006509121066091D2
:10D460007C0270917D0280917E0290917F020F94E8
:10D470002E8369837A838B839C83CE0101960E94DD
:10D4800056B5BC018CE49FE20E9410520F900F90A1
:10D490000F900F90DF91CF91089521E020936E07B8
:10D4A00060935707709358078093590790935A07D2
:10D4B00020E040E060E070E080911C0690911D0645
:10D4C0000C949B8960E070E080E291E4E6CF60E03C
:10D4D00070E080E89FE3E1CF6DEC7CEC8CEC9DE3A9
:10D4E000DCCFFF920F931F93CF93DF93F82E7093AF
:10D4F0001D0660931C0661E081E00E94AA8AD0911B
:10D500004007C0E091E081E0F81659F1F81628F0E4
:10D5100082E0F81609F449C06CC0D111D3C0992338
:10D5200089F080913F0718166CF0209166073091C2
:10D5300067072F5F3F4F30936707209366078F5F22
:10D5400080933F0780912702882309F42CC100E0D3
:10D5500010E021E041E066EA7FE28C2F0E94265134
:10D5600022C1D111AFC0992389F080913F071816CD
:10D570006CF020916607309167072F5F3F4F309323
:10D580006707209366078F5F80933F07809127028C
:10D59000882309F408C100E010E021E041E06FE9D0
:10D5A0007FE28C2F0E942651FEC0D1118BC099239F
:10D5B00089F080913F0718166CF020916607309132
:10D5C00067072F5F3F4F30936707209366078F5F92
:10D5D00080933F0780912702882309F4E4C000E08C
:10D5E00010E021E041E068E97FE28C2F0E942651A3
:10D5F000DAC040917C0250917D0260917E02709170
:10D600007F0240931E0650931F066093200670937E
:10D610002106D11122C0992389F080913F07181665
:10D620006CF020916607309167072F5F3F4F309372
:10D630006707209366078F5F80933F0780912702DB
:10D64000882309F4E8C000E010E021E041E06EE842
:10D650007FE28C2F0E942651DEC083E0F81232C098
:10D660006091BC0D7091BD0D8091BE0D9091BF0D6C
:10D670002091860D211126C00F94778420913A02C3
:10D6800030913B0262177307ECF4D130C9F48091FA
:10D690003F07813021F40E94D19481118EC0809186
:10D6A0002702882369F081E090913F07913009F0CB
:10D6B00080E004E024E04EE75FE26C2F0E94855199
:10D6C00082E072C0D130D9F480913F07813021F4DB
:10D6D0000E94D194811179C080912702882309F496
:10D6E00062C081E090913F07913009F080E004E052
:10D6F00024E044E75FE26C2F0E94855154C0D23091
:10D70000D9F480913F07823021F40E94D194811195
:10D7100064C080912702882309F445C081E090917C
:10D720003F07923009F080E003E02EE34AE65FE233
:10D730006C2F0E94855137C0D330D1F480913F07C0
:10D74000833021F40E94D194811151C0809127022D
:10D75000882349F181E090913F07933009F080E000
:10D7600003E02EE341E65FE26C2F0E9485511BC06F
:10D77000D430C9F480913F07843021F40E94D194C1
:10D7800081113FC080912702882369F081E0909148
:10D790003F07943009F080E003E02EE346E55FE2C6
:10D7A0006C2F0E94855185E0CF5FDF5F90E0C53030
:10D7B00009F0A9CE80933E0732C00E94C9898091AA
:10D7C0000C07882309F46BCF2AC00E94C989809175
:10D7D0000C07882309F480CF22C082E69AE60E94D3
:10D7E000A75580910C07882309F493CF18C087E6CA
:10D7F0009AE60E94A75580910C07882309F4A6CFCA
:10D800000EC08CE69AE60E94A75580910C078823EB
:10D8100009F4B8CF04C083E0F812C5CF21CFDF915F
:10D82000CF911F910F91FF9008954FEF64ED79E62E
:10D8300080E057CE4FEF68ED79E681E052CE4FEFB2
:10D840006CED79E682E04DCE4FEF60EE79E683E055
:10D8500048CE0F93CF93DF9361E081E00E94AA8AC4
:10D86000D0914007C0E0D1111AC080913F078111CB
:10D8700004C00E94D1948111A9C0809127028823FD
:10D8800009F49BC081E090913F07911180E004E092
:10D8900024E041E15FE26C2F0E9485518EC0D130BF
:10D8A000D9F480913F07813021F40E94D1948111F5
:10D8B00095C080912702882309F47FC081E0909170
:10D8C0003F07913009F080E003E02EE347E05FE29C
:10D8D0006C2F0E94855171C0D230D9F480913F07DE
:10D8E000823021F40E94D194811182C0809127025C
:10D8F000882309F462C081E090913F07923009F0DB
:10D9000080E000E22EE349EF5EE26C2F0E94855139
:10D9100054C0D330D9F480913F07833021F40E9462
:10D92000D19481116FC080912702882309F445C0EA
:10D9300081E090913F07933009F080E000E22EE310
:10D9400042E55EE26C2F0E94855137C0D430D1F49D
:10D9500080913F07843021F40E94D19481115CC0F2
:10D9600080912702882349F181E090913F0794300C
:10D9700009F080E000E22EE344E35DE26C2F0E94B8
:10D9800085511BC0D530C9F480913F07853021F403
:10D990000E94D19481114AC080912702882369F0A6
:10D9A00081E090913F07953009F080E000E22EE39E
:10D9B0004FE15DE26C2F0E948551CF5FDF5FC53084
:10D9C00009F051CF86E080933E0739C00E94C98993
:10D9D00080910C07882309F450CF31C08EE797E679
:10D9E0000E94A75580910C07882309F462CF27C0B5
:10D9F00083E09FE20E94BB8780910C07882309F493
:10DA000075CF1DC08FE59EE20E94BB8780910C07F9
:10DA1000882309F488CF13C083E49DE20E94BB876A
:10DA200080910C07882309F49BCF09C080E39DE215
:10DA30000E94BB8780910C07882309F4ADCFDF914A
:10DA4000CF910F910895CF93DF93EC01CB01BA01F1
:10DA50000F94AA840F94778479836883DF91CF91A0
:10DA6000089563E27DE68AEB9DE60C94DE890F93D0
:10DA70001F93CF93DF9361E081E00E94AA8AC09157
:10DA80004007D0E081E0C11122C0882389F0809155
:10DA90003F0718166CF020916607309167072F5FDB
:10DAA0003F4F30936707209366078F5F80933F0750
:10DAB00080912702882309F441C000E010E020E0B3
:10DAC00041E065E271E38D2F0E94265137C0C130DD
:10DAD000D1F480913F07813021F40E94D1948111CB
:10DAE00037C080912702882349F181E090913F0758
:10DAF000913009F080E000E22EE34AE151E36D2F1E
:10DB00000E9485511BC0C230C9F480913F0782300A
:10DB100021F40E94D194811122C080912702882390
:10DB200069F081E090913F07923009F080E000E2D7
:10DB30002EE346E051E36D2F0E948551DF5FCF5FFA
:10DB400080E0D53009F09FCF83E080933E070DC081
:10DB5000C093FB0C80910C07882319F206C0C09378
:10DB6000FB0C80910C078823C1F2DF91CF911F91AC
:10DB70000F9108950F94AA840F947784CB010C948D
:10DB800090B3EF92FF920F931F93CF93DF93CDB794
:10DB9000DEB72B970FB6F894DEBF0FBECDBF7C016A
:10DBA00040912306842F042E000C990B209124060B
:10DBB000223051F0233019F024E531E30AC047FF49
:10DBC00006C020E631E305C022E731E302C029E6C2
:10DBD00031E39F934F933F932F938E010F5F1F4F1E
:10DBE0001F930F930F94AA8C4091380250913902E1
:10DBF0004F50510997010F900F900F900F900F9079
:10DC00000F904E155F050CF49A013093C10D2093CF
:10DC1000C00D80E00E9462E2C8010E94958B2B96A5
:10DC20000FB6F894DEBF0FBECDBFDF91CF911F912D
:10DC30000F91FF90EF900895E091230687E1E802AD
:10DC4000F0011124E854F24F808591859ACF7F929C
:10DC50008F929F92AF92BF92CF92DF92EF92FF92FC
:10DC60000F931F93CF93DF93782E809324066093B6
:10DC7000230661E081E00E94AA8AD0914007C0E0BB
:10DC800081E0D1112EC0882389F080913F071816BA
:10DC90006CF020916607309167072F5F3F4F3093FC
:10DCA0006707209366078F5F80933F078091270265
:10DCB000882309F494C022E0721649F033E073120D
:10DCC00003C066E371E305C066E271E302C066E487
:10DCD00071E300E010E021E041E08C2F0E9426512A
:10DCE0007EC0D130D9F480913F07813021F40E9469
:10DCF000D19481117DC080912702882309F46FC0DF
:10DD000081E090913F07913009F080E004E024E049
:10DD100041EB51E36C2F0E94855161C0D230D9F4A0
:10DD200080913F07823021F40E94D194811168C014
:10DD300080912702882309F452C081E090913F0727
:10DD4000923009F080E000E22EE345EA51E36C2FC7
:10DD50000E94855144C0D330D1F480913F07833075
:10DD600021F40E94D194811156C08091270288230A
:10DD7000B1F181E090913F07933009F080E000E23B
:10DD80002EE349E951E36C2F0E94855128C0D4301D
:10DD900031F580913F07843021F40E94D1948111A4
:10DDA00045C0809127028823D1F011E080913F0780
:10DDB000843009F010E02091230637E12303F001BD
:10DDC0001124E854F24F808591850E9490B300E0C1
:10DDD0009C014BE751E36C2F812F0E94B451CF5F20
:10DDE000DF5F80E0C53009F04CCFC0933E075BC0D9
:10DDF0000E94C98980910C07882309F47CCF53C005
:10DE000080912B0690912C06BCDE80910C07882314
:10DE100009F48ECF48C080912D0690912E06B1DE78
:10DE200080910C07882309F4A0CF3DC081E00E94B7
:10DE3000C6940091230627E1020380011124F80112
:10DE4000E854F24F60857185072E000C880B990B02
:10DE50000F94AA8420E030E040EF52E40F942E8328
:10DE60000F947C84F801E054F24F1F928CE1882ECD
:10DE70008EE6982E91E3A92E9DE6B92E6B011AEA43
:10DE8000E12EF12C00E010E028E730E040E050E027
:10DE9000BF018AE891E30E94BD870F9080910C0733
:10DEA000882309F47ECFDF91CF911F910F91FF90CE
:10DEB000EF90DF90CF90BF90AF909F908F907F902A
:10DEC000089560E081E0C3CE8F929F92AF92BF929F
:10DED000CF92DF92EF92FF920F931F93CF93DF9336
:10DEE0004C015B016A0160E085E00E94AA8AD09142
:10DEF0004007F12C82E0E82ED1111AC08091270250
:10DF0000882321F180912A02823041F0833019F474
:10DF10006BED70E305C069EC70E302C06BEE70E37B
:10DF200000E010E021E041E08F2D0E9426510EC05C
:10DF3000D13061F480912702882341F000E010E0A5
:10DF400020E041E0B4018F2D0E942651A114B104BC
:10DF500081F0D23081F480912702882309F46EC0C9
:10DF600000E010E020E041E0B5018F2D0E94265135
:10DF700065C0C2E001C0C3E0C114D10491F0DC135C
:10DF80000FC080912702882351F000E010E020E0CC
:10DF900041E0B6018F2D0E942651CD2F01C0CD2F1B
:10DFA000CF5F21E030E0A114B10411F420E030E0B3
:10DFB00081E090E0C114D10411F480E090E0820F80
:10DFC000931F029781F0DC130DC0809127028823F4
:10DFD00049F000E010E020E041E064E071E38F2DC3
:10DFE0000E942651CF5FDC1314C080912702882342
:10DFF00071F000E010E021E040E069EF70E38F2D68
:10E000000E942651609122068F2D0E94C750E092F7
:10E010002702F394DF5F85E0F8126ECFCF5FC093E5
:10E020003E07DF91CF911F910F91FF90EF90DF900E
:10E03000CF90BF90AF909F908F900895C3E0C11490
:10E04000D10409F0ADCFADCF40E050E060E070E02A
:10E050008EEB90E339CF45EB50E365EA70E38CE952
:10E0600090E332CF40E050E06CE870E383E890E367
:10E070002BCF40E050E064E770E385E690E324CFE7
:10E0800040E050E066E570E389E490E31DCF4DE3A6
:10E0900050E36CE270E38CE190E316CF40E050E097
:10E0A0006EE070E385E090E30FCF40E050E065EF75
:10E0B0007FE288EE9FE208CF40E050E06BED7FE228
:10E0C0008AED9FE201CF40E050E06BEC7FE282EC12
:10E0D0009FE2FACE611160932A0240932206082E35
:10E0E000000C990BAA0BBB0B8C309105A0F5FC0121
:10E0F0008827EA56FF4F8F4F0D9490878BE290E769
:10E100001FC082E390E71CC085E590E719C087E453
:10E1100090E716C08EE490E713C083E690E710C046
:10E120008CE590E70DC080E490E70AC089E390E7B2
:10E1300007C01092FB0C87E39DE602C084E290E7E3
:10E14000009749F021E020936E0720E040E060E076
:10E1500070E00C949B890C94C2891092C61910929D
:10E16000920280911D0A806280931D0A0E942DDD1B
:10E170006FEF87E892E30E9444970C94C289CF9294
:10E18000DF92EF92FF920F931F9385E8C82E82E3F0
:10E19000D82EE12CF12C0AE712E329EC39E84DEAFC
:10E1A00050E765E772E380E792E30E94A38B1F913B
:10E1B0000F91FF90EF90DF90CF90089590911D0AFE
:10E1C00093FB882780F993FF06C081E090914D086A
:10E1D000911101C080E00895F1DF882339F080912A
:10E1E0001D0A82FB882780F991E08927089583EA38
:10E1F00092E30E94A18A40E061E080E06BDF89E960
:10E2000092E30D94BD72E8DF882321F085E992E363
:10E210000F94BD720C9425DDEF92FF920F931F9324
:10E22000CF93DF9361E081E00E94AA8AC09140070A
:10E2300010E0C11118C080913F07811104C00E94F5
:10E24000D1948111AAC180912702882361F081E0D5
:10E2500090913F07911180E004E024E044E652E30E
:10E26000612F0E94855180911D0A82FBDD27D0F924
:10E2700082FD06C0D1E09091B919913009F0D0E04B
:10E2800083FBEE24E0F883FF03C098DFF82E01C083
:10E29000F12CDD2309F458C0C130D9F480913F0737
:10E2A000813021F40E94D19481117FC18091270295
:10E2B000882309F48BC181E090913F07913009F0E8
:10E2C00080E000E22EE348E552E3612F0E94855191
:10E2D0007DC1C230D9F480913F07823021F40E9481
:10E2E000D194811169C180912702882309F46EC1FC
:10E2F00081E090913F07923009F080E003E02EE347
:10E300004DE452E3612F0E94855160C1C33009F092
:10E3100047C080913F07833021F40E94D19481113E
:10E3200057C180912702882309F450C181E0909160
:10E330003F07933009F080E003E02EE348E452E326
:10E34000612F0E94855142C18091B919823029F014
:10E3500043DF811102C0D1E004C0C13009F442C1E1
:10E36000D2E0CD131BC080913F078C1304C00E94E4
:10E37000D194811159C180912702882371F081E0E5
:10E3800090913F079C1380E003E02EE342E352E3C9
:10E39000612F0E948551DC2F01C0DC2FDF5F01C09F
:10E3A000D4E0CD131BC080913F078C1304C00E94A2
:10E3B000D194811143C180912702882371F081E0BB
:10E3C00090913F079C1380E003E02EE346E252E386
:10E3D000612F0E948551DC2F01C0DC2F81E08D0F61
:10E3E000C81318C080913F078C1304C00E94D194B9
:10E3F00081112EC180912702882361F081E09091E4
:10E400003F079C1380E003E02EE348E152E3612FD5
:10E410000E94855182E08D0F4091C00D5091C10D39
:10E420009091860D911107C020913A0230913B02E4
:10E4300042175307DCF0C81333C080913F078C1399
:10E4400004C00E94D19481110DC1809127028823BC
:10E4500039F181E090913F079C1380E000E22EE3C8
:10E4600040E052E3612F0E9485511AC0C81318C0C2
:10E4700080913F078C1304C00E94D1948111FCC08D
:10E4800080912702882361F081E090913F079C13DF
:10E4900080E003E02EE340EF51E3612F0E948551BD
:10E4A000DD5FCD1318C080913F078C1304C00E941C
:10E4B000D1948111EBC080912702882361F081E023
:10E4C00090913F079C1380E003E02EE342EE51E37E
:10E4D000612F0E94855191E09D0FEE2009F43BC011
:10E4E000F11053C0C91318C080913F078C1304C0AA
:10E4F0000E94D1948111D4C080912702882361F0B9
:10E5000081E090913F079C1380E000E22EE34FEC06
:10E5100051E3612F0E94855182E08D0FC81318C00E
:10E5200080913F078C1304C00E94D1948111C2C016
:10E5300080912702882361F081E090913F079C132E
:10E5400080E003E02EE341EC51E3612F0E9485510E
:10E5500093E09D0F1AC0C91316C080913F078C131A
:10E5600002C00E94D19480912702882361F081E04B
:10E5700090913F079C1380E000E22EE346EB51E3CD
:10E58000612F0E94855192E09D0F1F5FCF5F153074
:10E5900009F04FCE90933E0796C00E94C9898091A2
:10E5A0000C07882309F44FCE8EC021DE80910C0722
:10E5B000882309F47BCE87C08FEB90E70E94A75594
:10E5C00080910C07882309F48ECE7DC0D4E006CF5D
:10E5D00081EC94E70E94A75580910C07882309F4E9
:10E5E000A0CE71C080913F07813021F40E94D19468
:10E5F000811112C0809127028823A1F081E09091BF
:10E600003F07913009F080E000E22EE34BE352E354
:10E61000612F0E94855106C0F6DD80910C0788238A
:10E6200049F351C0D2E0BACE89E29CE60E94A755D8
:10E6300080910C07882309F49ECE45C082E599E7B6
:10E640000E94A75580910C07882309F4B4CE3BC0E3
:10E650008FE696E80E94A75580910C07882309F45D
:10E66000C9CE31C080E192E30E94BB8780910C0744
:10E67000882309F4EACE27C081E69FE60E94A755C9
:10E6800080910C07882309F4FBCE1DC087EA98E728
:10E690000E94A75580910C07882309F40CCF13C062
:10E6A0008EED91E30E94BB8780910C07882309F4CB
:10E6B00023CF09C08FE996E50E94A75580910C07EA
:10E6C000882309F435CFDF91CF911F910F91FF90EF
:10E6D000EF9008956091B60D70E080E00C94A8DD95
:10E6E0006091840270918502072E000C880B990BB3
:10E6F0000F94AA842AE037ED43E25CE30F94468648
:10E7000060938002709381028093820290938302CF
:10E710000895CF93DF93EC01CB01BA010F94AA8443
:10E720000F947C846883DF91CF91089580E00C94EE
:10E7300062E269E873E78FE993E70C94DE890F944E
:10E74000AA840F947C84862F0C94F8B2EF92FF92E7
:10E750000F931F93CF93DF9300D01F92CDB7DEB7F7
:10E76000082F7B010E94D194882329F010926E0714
:10E770000E94C9893BC06091660770916707611567
:10E78000710551F0109267071092660781E080933F
:10E790002702802F0E9413C180912702882331F124
:10E7A00084E0089F800111240A5F1F4E6091E50CF0
:10E7B0007091E60C072E000C880B990B0F94AA841D
:10E7C0009B01AC01F80160817181828193810F947A
:10E7D000468669837A838B839C8360E2CE010196AF
:10E7E0000E9466B6BC01C7010E9410520F900F90A4
:10E7F0000F900F90DF91CF911F910F91FF90EF90AD
:10E80000089564E273E380E0A1CF69E173E381E0FE
:10E810009DCF20E040E060E070E00E949B8981E0B5
:10E8200080936E071092E60C1092E50C089581E03B
:10E8300094E7EFCF85E094E7ECCF2F923F924F9291
:10E840005F926F927F928F929F92AF92BF92CF9280
:10E85000DF92EF92FF920F931F93CF93DF93CDB789
:10E86000DEB729970FB6F894DEBF0FBECDBF1C01EF
:10E870007987688769011A830983EB82BA01550F8A
:10E88000880B990B0F94AA844B015C0120E030E0C7
:10E8900040E057EC0F940B8618162CF0812C912C2D
:10E8A000A12C27ECB22EC501B4010F9477842B0163
:10E8B0003C01B601DD0C880B990B0F94AA844B0127
:10E8C0005C0120E03EEF4FEF56E40F94088487FD93
:10E8D00007C0812C9EEF992EAA24AA9496E4B92E03
:10E8E000E885F98560817181072E000C880B990BF2
:10E8F0000F94AA846B017C01C301B2010F94AA8416
:10E900009B01AC01C701B6010F942E830F947C8448
:10E910006C837D838E839F83C501B4010F947784BC
:10E920007B018C01E418F50806091709FB81FF93A8
:10E9300089809A8081E3A82E8DE6B82ECC80DD8078
:10E94000A301920168857985C1010E94BD870F905E
:10E9500029960FB6F894DEBF0FBECDBFDF91CF91E1
:10E960001F910F91FF90EF90DF90CF90BF90AF90ED
:10E970009F908F907F906F905F904F903F902F90DF
:10E9800008958F929F92AF92BF92CF92DF92EF92B3
:10E99000FF920F931F93CF93DF9361E081E00E947A
:10E9A000AA8AD0914007C0E0D1111AC080913F07D8
:10E9B000811104C00E94D194811121C1809127024C
:10E9C000882309F413C181E090913F07911180E001
:10E9D00004E024E044E153E36C2F0E94855106C11A
:10E9E000D13011F580913F07813021F40E94D194FC
:10E9F00081110DC180912702882309F4F7C011E02D
:10EA000080913F07813009F010E080916A02909177
:10EA10006B020E9490B300E09C0148E053E36C2F2E
:10EA2000812F0E94B451E2C0D23011F580913F078E
:10EA3000823021F40E94D1948111FBC08091270281
:10EA4000882309F4D3C011E080913F07823009F098
:10EA500010E08091C00D9091C10D0E9490B300E034
:10EA60009C014AEF52E36C2F812F0E94B451BEC02B
:10EA7000D33011F580913F07833021F40E94D19467
:10EA80008111ECC080912702882309F4AFC011E006
:10EA900080913F07833009F010E080919C0D9091A8
:10EAA0009D0D0E9490B300E09C0142EF52E36C2F59
:10EAB000812F0E94B4519AC0D43001F580913F0754
:10EAC000843021F40E94D1948111DDC0809127020D
:10EAD000882309F48BC011E080913F07843009F04E
:10EAE00010E08091B60D0E94F8B200E09C014EED5E
:10EAF00052E36C2F812F0E94B45178C0D53011F5AC
:10EB000080913F07853021F40E94D1948111DEC0AD
:10EB100080912702882309F469C011E080913F07A2
:10EB2000853009F010E080918402909185020E9466
:10EB300090B300E09C0144ED52E36C2F812F0E94C2
:10EB4000B45154C0D630D9F480913F07863021F4B7
:10EB50000E94D1948111CCC080912702882309F4AE
:10EB600045C081E090913F07963009F080E003E0D6
:10EB70002EE349EC52E36C2F0E94855137C0D73009
:10EB8000D1F480913F07873021F40E94D194811104
:10EB9000B9C080912702882349F181E090913F0715
:10EBA000973009F080E003E02EE34EEB52E36C2F48
:10EBB0000E9485511BC0D830C9F480913F0788302E
:10EBC00021F40E94D1948111A7C08091270288234B
:10EBD00069F081E090913F07983009F080E003E010
:10EBE0002EE34FEA52E36C2F0E948551CF5FDF5F27
:10EBF000C53009F0D9CE89E080933E0796C00E94C7
:10EC0000C98980910C07882309F4D8CE8EC0E12CE5
:10EC100000E010E027EE33E04AE050E06AE672E000
:10EC20008EE093E30ADE80910C07882309F4E2CE9C
:10EC30007CC081E00E94C694E12C06E913E722E241
:10EC400031E040E050E060EC7DE081E093E3F5DD11
:10EC500080910C07882309F4F1CE67C081E00E94FF
:10EC6000C694E12C0FEA12EE2CE830E040E050E0D0
:10EC70006CE97DE086EF92E3E0DD80910C0788236C
:10EC800009F400CF52C081E00E94C694C090B60D36
:10EC9000D12C1F928AE6882E83E7982E99E9A92E17
:10ECA00093E7B92EE12CF12C8701EA9420E030E0C3
:10ECB000A90166EB7DE088EE92E30E94BD870F908C
:10ECC00080910C07882309F401CF2FC0E12C00E7C5
:10ECD00013E727EE33E04AE050E064E872E089EDA4
:10ECE00092E3ABDD80910C07882309F411CF1DC09E
:10ECF00087E194E70E94A75580910C07882309F4C7
:10ED00002BCF13C08AE194E70E94A75580910C078E
:10ED1000882309F43ECF09C080E19BE80E94A755F3
:10ED200080910C07882309F450CFDF91CF911F9178
:10ED30000F91FF90EF90DF90CF90BF90AF909F909A
:10ED40008F9008950E94D194882321F010926E072D
:10ED50000E94C9890C945E500E94D194882341F08E
:10ED600020E040E060E070E082EA96E70E949B8944
:10ED700061E080E00C94F44F4F925F926F927F922B
:10ED8000AF92BF92CF92DF92EF92FF92CF93DF9339
:10ED9000EB01FC0160817181828193812CE3C22EA1
:10EDA000D12CE12CF12CA70196010F945287B62E9D
:10EDB000A72ECA01B901A70196010F9452876B01D2
:10EDC0007C01CA01B90128E130E040E050E00F9435
:10EDD00052872B013C01C9016DE671E00F942B872E
:10EDE00061157105D9F0AF92BF92DF92CF925F9219
:10EDF0004F929F938F937F936F9381E893E39F93B9
:10EE00008F93DF93CF930F94AA8C8DB79EB70E96F6
:10EE10000FB6F8949EBF0FBE8DBF61C00097C9F0BA
:10EE2000AF92BF92DF92CF925F924F929F938F9358
:10EE300081E793E39F938F93DF93CF930F94AA8CF3
:10EE4000EDB7FEB73C960FB6F894FEBF0FBEEDBF10
:10EE500046C04114510461047104B9F0AF92BF92ED
:10EE6000DF92CF925F924F9285E693E39F938F93C9
:10EE7000DF93CF930F94AA8C8DB79EB70A960FB6E7
:10EE8000F8949EBF0FBE8DBF2AC0C114D104E10407
:10EE9000F104A9F0AF92BF92DF92CF928DE593E398
:10EEA0009F938F93DF93CF930F94AA8CEDB7FEB708
:10EEB00038960FB6F894FEBF0FBEEDBF10C0AF92EC
:10EEC000BF9289E593E39F938F93DF93CF930F9442
:10EED000AA8C0F900F900F900F900F900F90DF91D2
:10EEE000CF91FF90EF90DF90CF90BF90AF907F9049
:10EEF0006F905F904F9008952F923F924F925F9244
:10EF00006F927F928F929F92AF92BF92CF92DF9239
:10EF1000EF92FF920F931F93CF93DF93CDB7DEB79E
:10EF20006F970FB6F894DEBF0FBECDBF0E94D1948D
:10EF3000882319F00E94C989F1C02090E30D309018
:10EF4000E40D8091E50D9091E60D9F8F8E8F80915D
:10EF5000E70D9091E80DA091E90DB091EA0D8A8F2F
:10EF60009B8FAC8FBD8F4090EB0D5090EC0D60905F
:10EF7000ED0D7090EE0D8090EF0D9090F00DA09043
:10EF8000F10DB090F20D60E085E00E94AA8AE09059
:10EF90004007F12CDE0111966D01E1100DC080914A
:10EFA00027028823E1F0C1010E94C6B38C0120E052
:10EFB00040E066EE73E310C0B1E0EB1210C0809148
:10EFC0002702882361F08E8D9F8D0E94C6B38C012D
:10EFD00020E040E06AED73E38F2D0E9426518A8D78
:10EFE0009B8DAC8DBD8D8E8B9F8BA88FB98FB601FD
:10EFF000CE014696C1DE92E0E9120BC08091270255
:10F000008823B1F000E010E020E040E068EC73E31A
:10F010000CC0A3E0EA120CC080912702882341F0C3
:10F02000860120E040E065EC73E38F2D0E942651BD
:10F030004E8A5F8A688E798EB601CE0146969CDE36
:10F04000B4E0EB120BC0809127028823B1F000E0FE
:10F0500010E020E040E063EB73E30CC085E0E812D1
:10F060000CC080912702882341F0860120E040E017
:10F0700060EB73E38F2D0E94265120E030E048ECD6
:10F0800052E4C501B4010F940F840F947784CB012F
:10F090006AE070E00F943F879F938F9320E030E009
:10F0A0004AE754E4C501B4010F940F840F947784A8
:10F0B0009F938F937F936F93A8EAB3E3BF93AF932C
:10F0C000DF92CF920F94AA8C0FB6F894DEBF0FBEDA
:10F0D000CDBFB6E0EB120BC0809127028823B1F0C0
:10F0E00000E010E020E040E068E973E30CC087E056
:10F0F000E8120CC080912702882341F0860120E0AD
:10F1000040E065E973E38F2D0E942651F394E39468
:10F1100095E0F91242CF88E080933E076F960FB6D4
:10F12000F894DEBF0FBECDBFDF91CF911F910F913D
:10F13000FF90EF90DF90CF90BF90AF909F908F9017
:10F140007F906F905F904F903F902F9008950F9316
:10F15000CF93DF9361E081E00E94AA8AD0914007BB
:10F16000C0E0D11117C080913F07811104C00E94F7
:10F17000D194811166C080912702882309F458C078
:10F1800081E090913F07911180E004E024E044E5A4
:10F1900053E34BC0D130C1F480913F07813021F45B
:10F1A0000E94D194811155C080912702882309F4CF
:10F1B0003FC081E090913F07913009F080E003E08B
:10F1C0002EE343E453E331C0D230B9F480913F07DA
:10F1D000823021F40E94D194811145C08091270290
:10F1E000882331F181E090913F07923009F080E06F
:10F1F00003E02EE345E353E318C0D530C9F4809112
:10F200003F07853021F40E94D194811136C080914E
:10F210002702882369F081E090913F07953009F03B
:10F2200080E003E02EE34FE253E36C2F0E94855110
:10F23000CF5FDF5FC53009F094CF86E080933E0753
:10F2400024C00E94C98980910C07882309F493CFB8
:10F250001CC08CEA96E70E94A75580910C07882372
:10F2600009F4A2CF12C08CE797E70E94A7558091BE
:10F270000C07882309F4B2CF08C08DEB95E50E94F6
:10F28000A75580910C07882311F2DF91CF910F9140
:10F29000089560E070E080E00E94A8DD0E94FCE23A
:10F2A0000C94C2898F929F92AF92BF92CF92DF92BD
:10F2B000EF92FF920F931F93CF93DF9361E081E072
:10F2C0000E94AA8AD0914007C0E0D1111AC0809153
:10F2D0003F07811104C00E94D1948111ABC080917D
:10F2E0002702882309F474C081E090913F079111AF
:10F2F00080E004E024E047E254E36C2F0E94855153
:10F3000067C0D13011F580913F07813021F40E9410
:10F31000D194811197C080912702882309F458C0A5
:10F3200011E080913F07813009F010E08091C00D1D
:10F330009091C10D0E9490B300E09C0149E154E31B
:10F340006C2F812F0E94B45143C0D23009F58091B7
:10F350003F07823021F40E94D194811199C080919D
:10F3600027028823A9F111E080913F07823009F03C
:10F3700010E080919C0D90919D0D0E9490B300E053
:10F380009C0141E154E36C2F812F0E94B45120C0B5
:10F39000D330F1F480913F07833021F40E94D1945F
:10F3A00081119BC080912702882391F011E0809108
:10F3B0003F07833009F010E08091B60D0E94C9B27A
:10F3C00000E09C014DEF53E36C2F812F0E94B4515C
:10F3D0008091C00D9091C10D20919C0D30919D0D9B
:10F3E000232B11F4892BE9F0D430C9F480913F0725
:10F3F000843021F40E94D194811192C0809127021F
:10F40000882369F081E090913F07943009F080E013
:10F4100000E22EE344EF53E36C2F0E94855185E018
:10F4200001C084E0CF5FDF5FC53009F04ECF80932D
:10F430003E077CC00E94C98980910C07882309F48B
:10F440004ECF74C081E00E94C694C090C00DD09091
:10F45000C10D1F9266E9862E63E7962E71E3A72EF3
:10F460007DE6B72E12E2E12EFF24F39400E010E0D7
:10F4700020E030E0A90160EC7DE080E294E30E94AE
:10F48000BD870F9080910C07882309F444CF4EC0AC
:10F4900081E00E94C694C0909C0DD0909D0D1F925B
:10F4A0003FEA832E32EE932E41E3A42E4DE6B42E96
:10F4B0001CE8E12EF12C00E010E020E030E0A90192
:10F4C0006CE97DE085E194E30E94BD870F90809117
:10F4D0000C07882309F443CF29C081E00E94C69419
:10F4E000C090B60DD12C1F928AE6882E83E7982E05
:10F4F0009AEAA92E97E5B92EE12CF12C8701EA941E
:10F5000020E030E0A90166EB7DE087E094E30E9413
:10F51000BD870F9080910C07882309F443CF06C064
:10F52000B8DE80910C07882309F468CFDF91CF9172
:10F530001F910F91FF90EF90DF90CF90BF90AF9011
:10F540009F908F90089580E095E290933406809389
:10F5500033068CE491E09093300680932F0680EC84
:10F560009EEF90933206809331069091380680E2A8
:10F57000890F863740F080EF890F20E431E0309327
:10F5800032062093310610923506809336068FEFAF
:10F590008093370608958F929F92BF92CF92DF9209
:10F5A000EF92FF920F931F93CF93DF931F92CDB7EC
:10F5B000DEB7E1D7882309F4D6C180916607863289
:10F5C00014F085E202C087FD80E0282F082E000C91
:10F5D000330B3093670720936607982F990F890F95
:10F5E0008093380680918806882309F4BCC1209155
:10F5F0003106309132060091350610913606020F21
:10F60000131FE0903306F090340680912F069091FE
:10F610003006E80EF91E01304FE7140768F0319507
:10F620002195310930933206209331066CED70E05C
:10F6300085E090E00F94087EF7FE15C080912F06BC
:10F640009091300691958195910990933006809321
:10F650002F0668E171E085E090E00F94087E81E07C
:10F660008093370617C081E0E81680E4F80694F02E
:10F670006BE470E084EF91E00F94087E8091420685
:10F68000815080934206882311F05DDF6CC1109297
:10F69000880669C120912F0630913006C7019A5023
:10F6A0008130934108F098C08F2D992787FD9A9556
:10F6B0000A9765E070E00F943F87812F17FF02C023
:10F6C00087E0810F482F45954595459581E090E06D
:10F6D000A0E0B0E004C0880F991FAA1FBB1F4A9585
:10F6E000D2F7FB01EE0FFF1FE75CF94F408151811C
:10F6F0008A0108231923012B09F419C180959095DB
:10F70000842395239183808384E090E0861B970B6C
:10F710004091890650918A06840F951F90938A061E
:10F720008093890680914106815080934106811122
:10F7300003C082E080938806932F9095991F9927A4
:10F74000991F80913706881F8827881F9817F1F026
:10F750003195219531093093300620932F0620E111
:10F7600030E040E050E060EF7FEF8FEF9FEF0E94CE
:10F770002B3D2091310630913206620F731F70933A
:10F7800032066093310660E773E021C08091310654
:10F7900090913206919581959109909332068093CC
:10F7A000310620E130E040E050E060EF7FEF8FEF86
:10F7B0009FEF0E942B3D20912F0630913006620F63
:10F7C000731F7093300660932F0660E872E085E047
:10F7D00090E00F94087EABC0121613060CF0A7C081
:10F7E000FDE3FF1A41E0E41642E0F40608F09FC092
:10F7F00080913806181B103108F099C03195219579
:10F8000031093093300620932F0660E773E083E0E0
:10F8100090E00F94087E8FEF8093370621E012303E
:10F820000CF020E08EEF810F8C30A0F0809131063B
:10F830009091320641E050E01816190614F040E0AD
:10F8400050E030E04217530709F055C0919581957B
:10F85000910927C0143050F520E030E0A90160EC98
:10F860007FEF8FEF9FEF0E942B3D2091310630916B
:10F870003206620F731F7093320660933106611572
:10F880007E4F34F480E09EEF9093320680933106F1
:10F8900080913106909132068130924064F180E08F
:10F8A00092E0909332068093310625C01C301CF103
:10F8B00020E430E040E050E060E070E0CB010E94E6
:10F8C0002B3D2091310630913206620F731F7093E9
:10F8D00032066093310661157E4F34F480E09EEF6E
:10F8E00090933206809331068091310690913206D2
:10F8F00081309240A4F6809188068230C1F480E481
:10F90000809341068FEF9FEF90933A0680933906DC
:10F9100090933C0680933B0690933E0680933D0671
:10F920009093400680933F0681E080938806209163
:10F930003506309136068091310690913206820F5D
:10F94000931F9093360680933506209133063091AD
:10F95000340680912F0690913006820F931F90936A
:10F9600034068093330661E082EE94E00E94C23751
:10F97000809116058E3130F0809116058E3308F493
:10F9800056C05AC0809118058A30B0F389E3E82E3A
:10F9900086E0F82E9AE0892E912CB82C80911605DD
:10F9A00090E094012C5F3F4F281739075CF442E048
:10F9B000E40EF11C85E0880E911CEEE18E16910498
:10F9C00061F7DACF80911805881588F330E0C12CF3
:10F9D000D12CF70180819181A0E0B0E00C2C04C013
:10F9E000B695A795979587950A94D2F780FD07C09D
:10F9F000FFEFCF1ADF0A385F303859F7D8CF00E071
:10FA000010E0A801480D591D8091160590E0481797
:10FA100059073CF08091180590E0841795070CF089
:10FA200055C00F5F1F4F0430110559F7E1CF80918A
:10FA300018058C3308F055C0809188068823B1F0F2
:10FA400080913406482F582F550F550B9A013327B4
:10FA50002F5F3F4F8091160590E0281739073CF043
:10FA600080911805841708F04DC001C09DD5809184
:10FA700016058B30D0F469E080E00E948F4C8091B5
:10FA8000890690918A060E94944C69E08EE60E9455
:10FA90008F4C2091420683E090E0821B91096FEF2A
:10FAA0007FEF845D9B4C0E94EC4C0E94D194882394
:10FAB00091F10F90DF91CF911F910F91FF90EF90F7
:10FAC000DF90CF90BF909F908F90ABC527E04B2DDC
:10FAD000400F632F82EE94E039830E94D33939813D
:10FAE000A0CF20E14DE36091380682EE94E00E94C1
:10FAF000D33920E14CE36091380682EE94E00E9415
:10FB0000D3399ACF6091360602E022E082EE94E08B
:10FB10000E94143AACCF0F90DF91CF911F910F91BB
:10FB2000FF90EF90DF90CF90BF909F908F900895BF
:10FB30006BEC7AE782E064D588E38093380683E053
:10FB40008093420680E480934106E9E3F6E0118267
:10FB50001082138212821582148217821682F3DCBD
:10FB600082E190E0909367078093660708958F92F3
:10FB70009F92AF92BF92CF92DF92EF92FF92CF937C
:10FB800070915B06A6E5B6E020E030E090E080E012
:10FB9000622FCD902F5F3F4FC110722F8C2962953D
:10FBA000607F40E050E0D12CE12CF12C4601570160
:10FBB000042E04C0B694A794979487940A94D2F71D
:10FBC00080FE08C0E92FF0E0E95BF94FC62FC42B97
:10FBD000C0839F5F4F5F5F4F4530510539F723303A
:10FBE0003105B1F670935B0640E050E020E090E014
:10FBF000A0E0B0E06C017D01042E04C0F694E7940F
:10FC0000D794C7940A94D2F7C0FE05C020935D062E
:10FC10002AE335E007C02E504F5F5F4F4530510556
:10FC200049F7F4CF422F3150A0F0225F6C017D01E3
:10FC3000032E04C0F694E794D794C7940A94D2F79D
:10FC4000C0FEF0CF40935C0680915A06823069F482
:10FC500003C020935C06F8CF80915E06181614F05E
:10FC60008CEF01C084E080935E06CF91FF90EF900F
:10FC7000DF90CF90BF90AF909F908F90089580E0DD
:10FC800090E0FC01EF59F94F128203968E319105F5
:10FC9000C1F70895109260068AE080935F0683E0C2
:10FCA00080935E068FE080935A06E6E5F6E08FE1EA
:10FCB0008083818382835BDFE2CF1F93CF93DF93C7
:10FCC000EC01162FDCDF809185068093820687E3A6
:10FCD0008093830686E0809384066AE070E088EE75
:10FCE00093E00F94087E909186069150909386063B
:10FCF000992351F010928106188310928506109274
:10FD000067071092660701C01882DF91CF911F919B
:10FD100008955F926F927F928F929F92AF92BF925F
:10FD2000CF92DF92EF92FF920F931F93CF93DF93C7
:10FD300084E08093270280916807882309F467C2D2
:10FD400080916607909167078E31910514F08DE1DF
:10FD500090E097FF02C080E090E090936707809367
:10FD60006607880F991F880F991F20918506422FDB
:10FD7000022E000C550B4817590774F42D5FAC0187
:10FD8000421B510927FD5395423051051CF0209329
:10FD9000850602C08093850620918506422F022E9B
:10FDA000000C550B841795077CF42350422F022E2C
:10FDB000000C550B481B590B423051051CF0209389
:10FDC000850602C08093850680918806882309F401
:10FDD0001EC220914506222349F090914606920FBB
:10FDE00090934606933F14F410924506823070F0CB
:10FDF000815080938806823011F44CDF08C284362B
:10FE000009F005C281E08093880601C28091440612
:10FE10008F5F8093440640915A0690E0242F30E093
:10FE200035952795281739070CF0ACC090914306FB
:10FE300081E089278093430610924406442309F405
:10FE4000A1C090915E0680916006890F20915D06A9
:10FE5000821724F020915C062817D4F49195909392
:10FE60005E0620915F062B5F20935F0680936006FD
:10FE700080915B063AE08302C0011124820F911D3C
:10FE800027FD9A95C99724F064E188E896E015DF8C
:10FE90009091600680915E06890F80936006809144
:10FEA0005A06882309F46EC024E130E040E050E0B7
:10FEB00060E070E0CB010E942B3D672B682B692B23
:10FEC00009F060C0E3E6F6E0C0E0D0E08081811197
:10FED00053C0CE01880F991FC80FD91FCF59D94FD2
:10FEE000209709F44FC020915A0630E02F5F3F4F12
:10FEF000032E000C440B550B60E070E0CB010E9418
:10FF00002B3DFB01E95BF94F4081242F30E0B4E049
:10FF100035952795BA95E1F7F901E755FC4F8081B2
:10FF200090E04F70509160066EE0469F500D112496
:10FF3000452FFC01EA55FC4F5081450FFC01ED5562
:10FF4000FC4F90819695842F890F888380915F065E
:10FF500082502F5F3F4F9AE0299F800D11248983A3
:10FF600022E030E040E050E060E070E0CB010E9431
:10FF70002B3D6E5F6A8306C021963396CA30D10549
:10FF800009F0A4CF90918106992341F080918006D9
:10FF9000890F8093800687FD1092810680918106EB
:10FFA000882309F4A2C020918006E0915F062E17F5
:10FFB0000CF49BC0022E000C330B0E2E000CFF0B1A
:10FFC000CF014D96821793070CF48FC0E0907F0607
:10FFD000CE2D0E2C000CDD0B10916006CE01811B86
:10FFE000910917FD93956EE070E00F943F87F62E10
:10FFF000653008F07AC02E1B3F0BC90102966AE0FB
:020000021000EC
:1000000070E00F943F87062F633008F06EC0812C9C
:10001000912C540183940F2C04C0880C991CAA1CA9
:10002000BB1C0A94D2F7A62F660FBB0BBD016A5A00
:10003000794FFB019081892F882109F456C0FD0179
:10004000E755FC4FE0814E2F50E0812FFEE0FF9EF0
:10005000800D11249A012A553C4FF901F080F80EC9
:10006000EF140CF442C0FA01ED55FC4F1081412F02
:1000700050E04F0D511DF7FC5A95C417D507ACF54C
:1000800010928106282D20952923FB01208323E04F
:1000900030E02A1B3B0B8091890690918A06280F3D
:1000A000391F30938A06209389066AE070E088E25F
:1000B00090E00F94087E20915F06FAE00F9F200DDC
:1000C0001124912F96958F2D890F8550809382064C
:1000D0002093830684E08093840680915A068150A1
:1000E00080935A06882321F042DDC3E6D6E011C092
:1000F00084E180938806C3DDF8CFFE018291890FE9
:100100008083803454F01882239626E0C138D207C9
:10011000E1F098819923C1F3F0CF8733ACF3FE016E
:100120003297208180918506281774F3022E000CE7
:10013000330B082E000C990B0A968217930724F3B1
:1001400068E788E896E0B9DDDFCF80914506811148
:1001500024C024EF31E040E050E060E070E0CB01EB
:100160000E942B3D672B682B692BB9F422E030E00D
:1001700040E050E060E070E0CB010E942B3D672B37
:10018000682B692B09F091C18FEF80934506813070
:1001900009F48DC18FE780934606809181068823FC
:1001A000B1F180914506882391F1809180068730D6
:1001B00074F520917F0680914606281744F1022E9F
:1001C000000C330B082E000C990B0C96821793072A
:1001D000F4F0109245061092810680918906909164
:1001E0008A060A9690938A06809389066AE070E0F0
:1001F00088E290E00F94087E809146068F5F80939E
:10020000820681E08093830684E080938406809157
:10021000700782FF04C080915906815001C08AE0B6
:10022000809359060E94D1948823C1F0809188065A
:10023000811103C01092590611C0813079F4809168
:10024000810681110BC0809185068B5F80937F06AC
:1002500084E3809380068CEF809381068091590619
:10026000811101C0DED161E082EE94E00E94C237CC
:10027000C0915F064C2F0C2E000C550B80915B0635
:100280009A016AE08602200D311D112422503109A5
:100290008091160590E0821793072CF08091450617
:1002A000811165C069C08091180590E08417950799
:1002B000ACF379EA672E73E0772EE6E58E2EE6E062
:1002C0009E2EFEE15F2E5C0EF301C1903F012C2FAC
:1002D0000C2E000C330BA901495F5F4F809116056E
:1002E00090E0481759073CF4C65FFFEF8F1A9F0A4A
:1002F000C511EACFD3CF8091180590E082179307FC
:100300009CF3D091600616E41D0FA12CB12CD12CCA
:10031000CC0CDD1CF401808190E0A0E0B0E00A2C60
:1003200004C0B695A795979587950A94D2F780FF54
:1003300017C0809143067601E80EF11CC70164E006
:10034000880F991F6A95E1F79C01215A3B4C79016E
:1003500008E022E04C2F6D2F82EE94E00E94EC37F3
:10036000D25F3FEFA31AB30AD113D4CFBDCF809190
:100370001605883008F49DC080918806882369F0AE
:10038000909116059F3348F490911805973328F003
:10039000823008F49CC081FD9AC080918106882338
:1003A000B1F040918006242F042E000C330BB901CC
:1003B0006D5F7F4F8091160590E0681779073CF0DC
:1003C0008091180590E0821793070CF08EC0C0E072
:1003D000D0E0FE01EF59F94F8281882399F04181E5
:1003E000842F042E000C990B2091160530E0821703
:1003F000930744F002972091180530E02817390739
:100400000CF07BC02396CE31D10519F7809184067C
:100410008823B1F040918306242F042E000C330B67
:10042000B9016A5F7F4F8091160590E068177907E0
:100430003CF08091180590E0821793070CF065C09E
:1004400080918806811101C0AFD0809116058A3055
:1004500008F06DC069E080E00E948F4C80918906B1
:1004600090918A060E94944C80918606882309F414
:100470005EC0C1E040E1C42ED12C809186068C176D
:1004800008F455C0B6016C1B7109660F660F660F44
:100490005AE4E52E54E3F52E05E021E041E082EE3A
:1004A00094E00E94EC37CF5FE8CF81E06ECE83EF1F
:1004B00072CE22E3E22E24E3F22E05E022E042E0B7
:1004C0006091460682EE94E00E94EC3755CF9FE49F
:1004D000E92E94E3F92E08E022E047E360918506D7
:1004E00082EE94E00E94EC3758CF24E060917F06C2
:1004F00082EE94E00E94F3396ACF425023E060819B
:1005000082EE94E00E94F3397DCF8CE3E82E84E301
:10051000F82E07E022E06091820682EE94E00E94CD
:10052000EC378091840681508093840689CFDF91D7
:10053000CF911F910F91FF90EF90DF90CF90BF90E0
:10054000AF909F908F907F906F905F90089569E833
:100550007EE784E155D083E0809386068AE080932D
:1005600059061092810696DB109285061092670755
:1005700010926607089580916807882319F082E039
:100580008093870684E080932702809188068823E1
:1005900049F0909187068FEF890F8093870681E05D
:1005A00019160CF080E008950F938091160585329E
:1005B00028F5809118058B3108F160E082EE94E017
:1005C0000E94C23709E028E34BE164E282EE94E046
:1005D0000E94643A61E082EE94E00E94C2370E9479
:1005E000A295882359F063E285E20E948F4C6FEF59
:1005F0007FEF8FEB94E30F910C94EC4C0F910895E7
:10060000FB0110928A06109289068093880620E0EA
:1006100040E060E070E0CF018ED681E080936E070D
:10062000089510926E07B5C680918B0690918D0645
:1006300089130DC080918C0690918E06891714F055
:100640002FEF01C021E0820F80938C0608C089172C
:1006500014F02FEF01C021E0820F80938B068913E5
:1006600019C02091EF0621502093EF0630E0832F30
:1006700090E0DC01AA0FBB1FA557B94F880F991F47
:10068000FC01E357F94F808191818D939C933F5FEB
:10069000231768F70895EF92FF921F93CF93DF938C
:1006A0001091EF062091F606E22E022E000CFF08B4
:1006B0003091F706C32F032E000CDD0BEEE8F6E0B9
:1006C00040E0411709F446C0CF010397DC019C913B
:1006D000BF0161507109DB018C9198131DC0692F16
:1006E000092E000C770B61507109C617D70711F05E
:1006F00039132DC09081BF0162507109DB018C91CB
:10070000582F98170CF4592F25170CF189170CF452
:10071000892F8217E4F020C0BF0162507109DB010C
:100720005C91652F052E000C770B61507109E61660
:10073000F70611F025130BC0582F98170CF4592FFA
:1007400035172CF089170CF4892F83172CF44F5F81
:100750003296B7CF80E001C081E0DF91CF911F9149
:10076000FF90EF90089528E130E040E050E060E035
:1007700070E0CB010E942B3D6093F7062AE030E049
:1007800040E050E060E070E0CB010E942B3D6093C0
:10079000F60681DF8111E7CF08959091F806811167
:1007A00002C08FEF01C081E0980F93709093F8061C
:1007B000E091EF06EF5FE093EF06F0E0EE0FFF1F32
:1007C000E557F94F8091F30680838091F10681838C
:1007D0000895CF9380E091E09093F3068093F20622
:1007E00080E095E09093F1068093F0061092F80671
:1007F0001092EF06EBE8F6E01082C5E0C18381E0DD
:10080000CCDFC093F506109267071092660710922E
:10081000F406CF910895EF92FF920F931F93CF9319
:10082000DF938091EF06843008F4B1C090E0FC01C2
:10083000EE0FFF1FE757F94F2081EC01CC0FDD1FB2
:10084000C557D94F68810297261719F0F12C3196B8
:100850006BC0E12C219631964E2D50E04817590778
:100860000CF095C0BA01660F771F8B010557194F21
:10087000D801FC90DB01A357B94F3C91F316E9F086
:10088000432FF3160CF44F2D24179CF13F150CF455
:100890003F2D321774F1DB01A557B94F11965C91CA
:1008A00041E0308153170CF040E031E0688165177A
:1008B0000CF430E04317E9F06CC02F111AC06881C6
:1008C000408111965C91D80111963C91A42F641738
:1008D0000CF4A62F732F35170CF4752F7A174CF0E4
:1008E00046170CF4462F53170CF4352F43170CF012
:1008F00050C0E394B1CFEA01CC0FDD1F8E01055744
:10090000194FD80111967C91DE01A357B94F11966A
:100910003C911197731709F14081532F73170CF411
:10092000572F45173CF4F3944F2D50E048175907C3
:1009300014F32DC037170CF4372F3417A4F3C55711
:10094000D94F588141E052170CF040E031E0651773
:100950000CF430E0431739F31CC030813713E3CF78
:100960004C91D8013C91762F26170CF4722F532FFF
:1009700034170CF4542F5717B4F2562F62170CF497
:10098000522F43170CF4342F53176CF202C080E03F
:1009900001C081E0DF91CF911F910F91FF90EF9007
:1009A0000895CF92DF92EF92FF920F931F93CF9310
:1009B000DF931F92CDB7DEB7DEDD882309F480C058
:1009C0008091F2069091F306392F4091F0065091F4
:1009D000F1062091F806213061F02CF4211116C0A7
:1009E000CA01C3970AC0223031F0233079F4C3978B
:1009F00009C0C39607C0CA01C3969093F1068093BD
:100A0000F00604C09093F3068093F2061091F3066B
:100A10000091F106311303C0051709F451C01831D4
:100A200010F40A3048F01092880668E270E080E91D
:100A300091E00F94087E44C0E091EF06F0E0EE0FE5
:100A4000FF1FE557F94F108301838091660790914E
:100A5000F406282F291B39F08093F40681E0121642
:100A60000CF080E09ADE8091F506882321F0815019
:100A70008093F50601C0D8DDCEDE8111D4CF809100
:100A8000F70618131DC08091F606081319C06CED07
:100A900070E085E090E00F94087E68E171E085E009
:100AA00090E00F94087E8091890690918A060196C5
:100AB00090938A068093890682E08093F50653DE40
:100AC00061E082EE94E00E94C23780911605893081
:100AD00050F467E080E00E948F4C809189069091ED
:100AE0008A060E94944C06E32CE749E062E082EE1D
:100AF00094E00E94143AF12C8091EF0620911605A3
:100B0000F81608F071C0EF2DF0E0AF01440F551F4B
:100B1000DA01A557B94F9C91FA01E357F94F80814B
:100B2000981345C091811196EC901E2DE9160CF496
:100B3000192F85E01802B0011124625F7F4F30E069
:100B4000621773070CF44EC09E150CF4E92E9E2D0F
:100B5000E5E09E0290011124265F3F4F8091180529
:100B600090E028173907F4F58E2D880F880F8E0D29
:100B70007BE0780FCA018557994F6C011E1594F1DF
:100B8000272F072E000C330BA9014D5F5F4F80917B
:100B9000160590E0481759073CF08091180590E041
:100BA000821793070CF04DC0E3947B5FE7CF11965B
:100BB0003C91432F440F440F340F4BE0D42ED30EFF
:100BC0004D2D0D2C000C550BBA016D5F7F4F30E0A1
:100BD000621773073CF02091180530E024173507A1
:100BE0000CF040C0F39488CF4091F606842F880F14
:100BF000880F480F455F642F042E000C770BFB0114
:100C00003396822F90E0E817F9073CF080911805A1
:100C100090E0861797070CF044C0809188068111F8
:100C200001C0C2DC0E94D194882309F448C00F900F
:100C3000DF91CF911F910F91FF90EF90DF90CF90B8
:100C4000F0CCF6016081862F880F880F680F6C5FEB
:100C500004E024E0472F82EE94E079830E94643A16
:100C60007981A2CFE82E98170CF4E92EC82E8917A7
:100C70000CF4C92E1E2D110F110F1E0D50E01C5F1C
:100C8000CE140CF4AFCF612F650F04E024E04D2D9E
:100C900082EE94E059830E94643AE39459815B5F49
:100CA000EFCF6091F706862F880F880F680F6C5F73
:100CB00004E024E082EE94E00E94143AAECF0F905C
:100CC000DF91CF911F910F91FF90EF90DF90CF9028
:100CD000089561ED74E881E093DC7BDD44CD0F93F2
:100CE0001F93CF93DF9361E081E034D4D09140072C
:100CF000C0E0D11117C080913F07811104C00E944C
:100D0000D19481119EC080912702882309F43EC0AE
:100D100081E090913F07911180E004E024E048E1F8
:100D200055E331C0D130B9F480913F07813021F4CF
:100D30000E94D19481118CC080912702882331F1C7
:100D400081E090913F07913009F080E003E02EE3CD
:100D500046E055E318C0D230C9F480913F07823095
:100D600021F40E94D19481117DC0809127028823B3
:100D700069F081E090913F07923009F080E003E054
:100D80002EE347EF54E36C2F0E948551BDD2182FFC
:100D9000D330D9F480913F07833021F40E94D1945D
:100DA00081116AC080912702882309F478C081E00C
:100DB00090913F07933009F080E000E22EE348EE87
:100DC00054E36C2F0E9485516AC081116AC0D430EF
:100DD000B9F480913F07843021F40E94D1948111AD
:100DE00052C080912702882319F181E090913F073A
:100DF000943009F080E000E22EE34AED54E315C0A0
:100E0000D530B1F480913F07853009F443C080911B
:100E10002702882369F081E090913F07953009F01F
:100E200080E000E22EE349EC54E36C2F0E948551F0
:100E300086E0CF5FDF5FC53009F05BCF80933E0770
:100E40003BC0A7D280910C07882309F45CCF34C043
:100E500088EF9EE50E94A75580910C07882309F42E
:100E60006BCF2AC080E19BE80E94A75580910C07B8
:100E7000882309F47ACF20C060D480910C0788239E
:100E800009F490CF19C05CD480910C07882309F431
:100E9000A8CF12C00E94D194811105C0B8CF1123F0
:100EA00039F284E0C6CF0F94600481E0A5D380912D
:100EB0000C07882309F4ABCFDF91CF911F910F91DD
:100EC0000895CF93DF93EC01CB01BA010F94AA846C
:100ED0000F9477846883DF91CF910895CF93DF9348
:100EE000EC01CB01BA010F94AA8420E030E040E28B
:100EF00051E40F9446860F947C8479836883DF9154
:100F0000CF9108950F94AA840F947784862F0C9420
:100F10001EB30F94AA8420E030E040E251E40F9425
:100F200046860F947C84CB010C944DB3E0910D0761
:100F3000E63000F581E08E0F80930D078091660703
:100F400090916707A0E0B0E03091400720913E0704
:100F500048E0E49FF0011124E25FF84F40916107FF
:100F6000509162075183408382839383A483B58326
:100F70003683278308950D94BD722F923F924F922E
:100F80005F926F927F928F929F92AF92BF92CF9219
:100F9000DF92EF92FF920F931F93CF93DF9300D0D6
:100FA00000D0CDB7DEB71C012B833C834D835E831D
:100FB00069837A83BBDF83E08093270230920B073B
:100FC00020920A0769817A81709309076093080764
:100FD0002B813C814D815E8120930407309305076E
:100FE0004093060750930707E0920007F09201072D
:100FF0000093020710930307D0926707C092660719
:10100000B0926207A09261079092FF068092FE065E
:101010008C8D8093FD0626960FB6F894DEBF0FBE2A
:10102000CDBFDF91CF911F910F91FF90EF90DF9097
:10103000CF90BF90AF909F908F907F906F905F9078
:101040004F903F902F9008952F923F924F925F9232
:101050006F927F928F929F92AF92BF92CF92DF92C8
:10106000EF92FF920F931F93CF93DF93CDB7DEB72D
:1010700029970FB6F894DEBF0FBECDBF1C0179874C
:101080006887F22E1A830983EB82642F70E080E078
:1010900090E00F94A8844B015C0120E030E040E038
:1010A00057EC0F940B8618162CF0812C912CA12C48
:1010B00027ECB22EC501B4010F9477842B013C01BB
:1010C0006F2D70E080E090E00F94A8844B015C01EC
:1010D00020E03EEF4FEF56E40F94088487FD07C0F1
:1010E000812C9EEF992EAA24AA9496E4B92EE88525
:1010F000F985608170E080E090E00F94A8846B0136
:101100007C01C301B2010F94AA849B01AC01C70109
:10111000B6010F942E830F947C846C837D838E8321
:101120009F83C501B4010F9477847B018C01E4187F
:10113000F50806091709FB81FF9389809A8089E9E0
:10114000A82E83E7B82ECC80DD80A30192016885AC
:101150007985C10112DF0F9029960FB6F894DEBF92
:101160000FBECDBFDF91CF911F910F91FF90EF90F8
:10117000DF90CF90BF90AF909F908F907F906F90B7
:101180005F904F903F902F9008952F923F924F92F3
:101190005F926F927F928F929F92AF92BF92CF9207
:1011A000DF92EF92FF920F931F93CF93DF93CDB710
:1011B000DEB729970FB6F894DEBF0FBECDBF1C0176
:1011C0007987688769011A830983EB82BA0180E015
:1011D00090E00F94A8842DEC3CEC4CEC5DE30F9474
:1011E00046864B015C0120E030E040E057EC0F9474
:1011F0000B8618162CF0812C912CA12C27ECB22EEA
:10120000C501B4010F9477842B013C01B60180E045
:1012100090E00F94A8842DEC3CEC4CEC5DE30F9433
:1012200046864B015C0120E03EEF4FEF56E40F9401
:10123000088487FD07C0812C9EEF992EAA24AA94CA
:1012400096E4B92EE885F9856081718180E090E0AF
:101250000F94A8842DEC3CEC4CEC5DE30F94468697
:101260006B017C01C301B2010F94AA849B01AC0104
:10127000C701B6010F942E830F947C846C837D8309
:101280008E839F83C501B4010F9477847B018C0109
:10129000E418F50806091709FB81FF9389809A80F5
:1012A00084E6A82E8AE8B82ECC80DD80A3019201C6
:1012B00068857985C10161DE0F9029960FB6F89493
:1012C000DEBF0FBECDBFDF91CF911F910F91FF9079
:1012D000EF90DF90CF90BF90AF909F908F907F90D6
:1012E0006F905F904F903F902F900895FB019081F9
:1012F00081E08927808383E080932702411551058F
:1013000011F0FA0119940895809174109091711060
:10131000891B8F7071F490911D0A92FB882780F9C8
:1013200092FD08C081E09091B919913019F080E0E8
:10133000089581E00895E0916107F0916207E81750
:10134000F907F9F09093620780936107709367073C
:10135000609366074093400720933E07805394496B
:1013600021F410926E0710920D070E94C65082E081
:101370008093270281E080930C07109269071092F6
:10138000F906089520E040E060E070E080E394E931
:10139000D2CFE0910D07EE2381F0E150E0930D07ED
:1013A00088E0E89FF0011124E25FF84F2781468131
:1013B00060E070E080819181BECFE4CFCF93DF9376
:1013C000FC01EB01809166079091670797FF04C0CD
:1013D000109267071092660740910007509101072D
:1013E00060910207709103078091660790916707EB
:1013F000092E000CAA0BBB0B481759076A077B077D
:1014000024F450936707409366078091270288234E
:10141000D1F0209166073091670780910407909181
:101420000507A0910607B0910707BC01CD01620F27
:10143000731F811D911D1995BC0180910A07909120
:101440000B070E94105280915B07811108C08091A8
:10145000FD06882389F180912702882369F1809114
:10146000080790910907009791F020916607309145
:101470006707409104075091050760910607709136
:101480000707420F531F611D711DFE011995E09161
:10149000FE06F091FF06309741F08091FD06811124
:1014A00003C080915B07811119950E94D194882314
:1014B00019F0DF91CF916DCFDF91CF91089561E663
:1014C00077E882E897E87ACF6EE677E889E897E8E8
:1014D00075CF0F931F93CF93DF93809127028823BB
:1014E00059F06091FA067091FB0600E010E020E0F0
:1014F00041E081E00E9426518091FC0681111CC0D0
:1015000081E08093FC06C0916107D091620720E0E2
:1015100040E060E070E089E69AE80DDF0F94FA267B
:101520001092FC0620E040E060E070E0CE01DF9128
:10153000CF911F910F91FFCEDF91CF911F910F910E
:101540000895009711F48CE295E39093FB06809345
:10155000FA06BFCF282F10926007809166079091FE
:1015600067078130904820F0109267071092660755
:1015700080916807882331F08091660780933F0748
:1015800010920C0780913E071816BCF4082E000C30
:10159000990B821B910920913F07022E000C330BFF
:1015A0002817390754F097FF02C080E090E080933D
:1015B0003F07909367078093660780913F076623F4
:1015C000C1F090914007891714F48093400720914F
:1015D0004007022E000C330B2C5F3F4F482F082E84
:1015E000000C550B2417350734F4845080934007C2
:1015F0000895809340070895882361F063E972E0BD
:1016000084E690E00F94087E6AEB72E084E690E056
:101610000D94087E68EB71E084E190E00D94087E03
:10162000CF92DF92EF92FF92CF93DF930E94D194FB
:10163000882359F00F94250410926E07DF91CF9103
:10164000FF90EF90DF90CF90A4CE81E080936E0763
:10165000C0916607D0916707209709F442C01092A5
:10166000670710926607BE010D2E000C880B990BC0
:101670000F94AA8420910E1030910F1040911010F9
:10168000509111100F9446862091530F3091540FB2
:101690004091550F5091560F0F942F836B017C0191
:1016A00020E030E040E050EC0F940B8687FD19C03D
:1016B00020E030E040EA50E4C701B6010F9408840E
:1016C00018167CF0BE0182E00E9413C1C092530F35
:1016D000D092540FE092550FF092560F82E0809313
:1016E0002702809127028823C9F083E59FE00E94AA
:1016F000F2B3BC018DE195E30E9410526091530F4B
:101700007091540F8091550F9091560FDF91CF91AA
:10171000FF90EF90DF90CF900C943D53DF91CF91ED
:10172000FF90EF90DF90CF90089521E02093FC068A
:101730000F94C2721092FC0608950F9410075CCFAC
:101740000F94C61659CF4F925F926F927F928F92ED
:101750009F92AF92BF92CF92DF92EF92FF920F9340
:101760001F93CF93DF931F921F92CDB7DEB72C014B
:101770004A013901580187017601209166073091AD
:1017800067072115310559F081E0121613060CF098
:1017900080E08093F90610926707109266076983CC
:1017A0007A830E94D194D82E69817A81811104C0F4
:1017B00080912702882311F195014091F906C20119
:1017C0000E94E452DD20D1F08091F906882311F0C7
:1017D000F40101C0F3010F900F90DF91CF911F91A1
:1017E0000F91FF90EF90DF90CF90BF90AF909F90C0
:1017F0008F907F906F905F904F9019940F900F9003
:10180000DF91CF911F910F91FF90EF90DF90CF90DC
:10181000BF90AF909F908F907F906F905F904F9010
:1018200008956091D70E7091D80E84EA9EE00C94D2
:10183000B03E60919C0E70919D0E89E69EE00C94E6
:10184000B03E6091610E7091620E8EE29EE00C944B
:10185000B03E6091260E7091270E83EF9DE00C94B0
:10186000B03E8F929F92AF92BF92CF92DF92EF9253
:10187000FF921F93CF93DF93C4EADEE019AD60912E
:101880003A1070913B1080913C1090913D100F9454
:101890007C844B015C01CE010E942540DC0120E1EB
:1018A00036E041EC50E00F94A7876B017C01A12F3B
:1018B000B0E0A50194010F94A7872227362F472F68
:1018C000582FC701B6010F945287BA01A9016627A4
:1018D0007727CE010E94794019AFDF91CF911F91F8
:1018E000FF90EF90DF90CF90BF90AF909F908F9040
:1018F00008958F929F92AF92BF92CF92DF92EF9214
:10190000FF921F93CF93DF93C9E6DEE019AD60919C
:101910003E1070913F1080914010909141100F94B3
:101920007C844B015C01CE010E942540DC0120E15A
:1019300036E041EC50E00F94A7876B017C01A12FAA
:10194000B0E0A50194010F94A7872227362F472FD7
:10195000582FC701B6010F945287BA01A901662713
:101960007727CE010E94794019AFDF91CF911F9167
:10197000FF90EF90DF90CF90BF90AF909F908F90AF
:1019800008958F929F92AF92BF92CF92DF92EF9283
:10199000FF921F93CF93DF93CEE2DEE019AD60910B
:1019A00042107091431080914410909145100F9413
:1019B0007C844B015C01CE010E942540DC0120E1CA
:1019C00036E041EC50E00F94A7876B017C01A12F1A
:1019D000B0E0A50194010F94A7872227362F472F47
:1019E000582FC701B6010F945287BA01A901662783
:1019F0007727CE010E94794019AFDF91CF911F91D7
:101A0000FF90EF90DF90CF90BF90AF909F908F901E
:101A100008958F929F92AF92BF92CF92DF92EF92F2
:101A2000FF921F93CF93DF93C3EFDDE019AD609179
:101A300046107091471080914810909149100F9472
:101A40007C844B015C01CE010E942540DC0120E139
:101A500036E041EC50E00F94A7876B017C01A12F89
:101A6000B0E0A50194010F94A7872227362F472FB6
:101A7000582FC701B6010F945287BA01A9016627F2
:101A80007727CE010E94794019AFDF91CF911F9146
:101A9000FF90EF90DF90CF90BF90AF909F908F908E
:101AA00008951F93CF93DF93C4EADEE01AAD612F50
:101AB000CE010E94F2401AAFDF91CF911F9108959D
:101AC0001F93CF93DF93C9E6DEE01AAD612FCE01FD
:101AD0000E94F2401AAFDF91CF911F91089560915B
:101AE000DC0E84EA9EE00C946D436091A10E89E6C1
:101AF0009EE00C946D436091660E8EE29EE00C9425
:101B00006D4360912B0E83EF9DE00C946D430F931A
:101B10001F93CF93DF9361E081E01CDDD0914007FC
:101B2000C0E081E0D11122C0882389F080913F0775
:101B300018166CF020916607309167072F5F3F4FB2
:101B400030936707209366078F5F80933F078091EC
:101B50002702882309F4AAC000E010E020E041E059
:101B600060EC75E38C2F0E942651A0C0D130D1F4D7
:101B700080913F07813019F414D78111A1C0809161
:101B80002702882309F492C081E090913F079130A9
:101B900009F080E004E024E044EB55E36C2F0E9460
:101BA000855184C0D230F9F480913F07823019F416
:101BB000F8D681118CC080912702882309F476C061
:101BC0008091DC0E811103C02BEA35E302C02FEABD
:101BD00035E381E090913F07923009F080E001E029
:101BE00049EA55E360C0D330F9F480913F07833070
:101BF00019F4D7D6811178C080912702882309F47F
:101C000055C08091A10E811103C020EA35E302C0C6
